:020000040800F2
:1000000000060020E1010008E3010008E301000808
:10001000E3010008E3010008E3010008E301000830
:10002000E3010008E3010008E30100086D2F000868
:10003000E3010008E3010008E3010008E301000810
:10004000E3010008E3010008E3010008E301000800
:10005000E3010008E3010008153200083D32000802
:10006000653200088D320008B5320008E30100084F
:10007000E3010008E3010008E3010008E3010008D0
:10008000E3010008E3010008E3010008E3010008C0
:10009000E3010008E3010008E3010008DD32000885
:1000A000E3010008E3010008E3010008E3010008A0
:1000B000B1330008E3010008E3010008E301000890
:1000C000E3010008E3010008E3010008E301000880
:1000D000E3010008E3010008E3010008E301000870
:1000E00041330008E3010008E3010008E3010008D0
:1000F000E3010008E3010008E3010008E301000850
:10010000E3010008E3010008E3010008E30100083F
:10011000E3010008E3010008E3010008E30100082F
:10012000E3010008E3010008E3010008E30100081F
:10013000E3010008E3010008E3010008E30100080F
:10014000E3010008E3010008E3010008212700089B
:10015000E3010008E3010008E3010008E3010008EF
:10016000E3010008E3010008E3010008E3010008DF
:10017000E3010008E3010008E3010008E3010008CF
:10018000E3010008E3010008E3010008E3010008BF
:10019000E3010008E3010008E3010008E3010008AF
:1001A000E3010008E3010008E3010008E30100089F
:1001B000E3010008E3010008E3010008E30100088F
:1001C000E3010008E3010008E3010008E30100087F
:1001D000E3010008E3010008E3010008E30100086F
:1001E00002E000F000F8FEE772B6374880F30888B6
:1001F000364880F3098836483649086040F20000E6
:10020000CCF200004EF63471CEF200010860BFF36C
:100210004F8FBFF36F8F40F20000C0F2F0004EF638
:100220008851CEF200010860BFF34F8FBFF36F8F8C
:100230004FF00000E1EE100A4EF63C71CEF20001E4
:100240000860062080F31488BFF36F8F01F030FF41
:1002500002F02AFE4FF055301F491B4A91423CBF25
:1002600041F8040BFAE71D49184A91423CBF41F896
:10027000040BFAE71A491B4A1B4B9A423EBF51F83E
:10028000040B42F8040BF8E700201849184A914281
:100290003CBF41F8040BFAE701F00EFF02F058FEF4
:1002A000144C154DAC4203DA54F8041B8847F9E7A7
:1002B00000F042F8114C124DAC4203DA54F8041B22
:1002C0008847F9E701F0F6BE000600200022002072
:1002D0000000000808ED00E00000002000060020FB
:1002E0007837000800220020402200204022002011
:1002F000602E0020E0010008E0010008E001000895
:10030000E00100082DE9F04F2DED108AC1F80CD066
:10031000C3689D46BDEC108ABDE8F08F002383F3CF
:1003200011882846A047002001F074FAFEE701F08A
:1003300003FA00DFFEE7000038B500F0BFFB01F074
:1003400087FE054601F0AAFE0446C8B90E4B9D4241
:1003500018D001339D4218BF044641F2883504BFCE
:1003600001240025002001F07DFE0CB100F074F89E
:1003700000F002FD284600F0C3F800F06DF8F9E740
:100380000025EFE70546EDE7010007B008B500F0EE
:1003900067FBA0F120035842584108BD07B541F260
:1003A0001203022101A8ADF8043000F077FB03B07E
:1003B0005DF804FB38B5302383F3118817480368D0
:1003C0000BB101F0F3FA164A144800234FF47A7186
:1003D00001F0E2FA002383F31188124C236813B171
:1003E0002368013B2360636813B16368013B63606A
:1003F0000D4D2B7833B963687BB9022000F026FCE1
:10040000322363602B78032B07D163682BB902205A
:1004100000F01CFC4FF47A73636038BD402200206A
:10042000B50300086023002058220020084B1870F4
:1004300003280CD8DFE800F008050208022000F0CD
:10044000FDBB022000F0F0BB024B00225A60704757
:100450005822002060230020244B254A10B51C465A
:100460001968013140D004339342F9D16268214BBD
:100470009A4239D9204B9B6803F1006303F580331E
:100480009A4231D2002000F033FB0220FFF7CEFF6A
:100490001A4B1A6C00221A64196E1A66196E596C7E
:1004A0005A64596E5A665A6E5A6942F080025A610D
:1004B0005A6922F080025A615A691A6942F0005260
:1004C0001A611A6922F000521A611B6972B64FF064
:1004D000E0233021C3F8084DD4E9003281F31188BC
:1004E0009D4683F30888104710BD00BF0000010837
:1004F00020000108FFFF0008002200200038024011
:100500002DE9F04F93B0AA4B00902022FF210AA8BA
:100510009D6800F0DBFBA74A1378A3B9A648012128
:1005200003601170302383F3118803680BB101F06D
:100530003DFAA24AA04800234FF47A7101F02CFA48
:10054000002383F31188009B13B19D4B009A1A601E
:100550009C4A009C1378032B1EBF00231370984AFB
:100560004FF0000A18BF5360D3465646D1460120CB
:1005700000F064FB24B1924B1B68002B00F0118249
:10058000002000F06DFA0390039B002BF2DB0120AA
:1005900000F04AFB039B213B162BE8D801A252F83E
:1005A00023F000BF0106000829060008BD06000868
:1005B0006F0500086F0500086F0500084707000871
:1005C000170900083108000893080008BB08000854
:1005D000E10800086F050008F30800086F0500082F
:1005E00065090008A10600086F050008A9090008B0
:1005F0000D060008A10600086F0500089308000812
:100600000220FFF7C3FE002840F0F581009B022185
:10061000BAF1000F08BF1C4605A841F21233ADF82D
:10062000143000F03BFAA2E74FF47A7000F018FAA9
:10063000071EEBDB0220FFF7A9FE0028E6D0013FF2
:10064000052F00F2DA81DFE807F0030A0D101336F8
:1006500005230593042105A800F020FA17E054486B
:100660000421F9E758480421F6E758480421F3E744
:100670004FF01C08404600F03DFA08F104080590D0
:10068000042105A800F00AFAB8F12C0FF2D10120DC
:1006900000FA07F747EA0B0B5FFA8BFB4FF00009F4
:1006A00000F060FB26B10BF00B030B2B08BF0024FE
:1006B000FFF774FE5BE746480421CDE7002EA5D086
:1006C0000BF00B030B2BA1D10220FFF75FFE0746B7
:1006D00000289BD0012000F00BFA0220FFF7A6FEB5
:1006E00000261FFA86F8404600F012FA044690B140
:1006F0000021404600F01CFA01360028F1D1BA462C
:10070000044641F21213022105A8ADF814303E460A
:1007100000F0C4F92BE70120FFF788FE2546244BA3
:100720009B68AB4207D9284600F0E4F9013040F05D
:1007300067810435F3E7234B00251D70204BBA4633
:100740005D603E46ACE7002E3FF460AF0BF00B035C
:100750000B2B7FF45BAF0220FFF768FE322000F026
:100760007FF9B0F10008FFF651AF18F003077FF4EE
:100770004DAF0F4A926808EB050393423FF646AF30
:10078000B8F5807F3FF742AF124B0193B84523DDA8
:100790004FF47A7000F064F90390039A002AFFF690
:1007A00035AF019B039A03F8012B0137EDE700BF3A
:1007B000002200205C23002040220020B503000816
:1007C000602300205822002004220020082200205C
:1007D0000C2200205C220020C820FFF7D7FD07462E
:1007E00000283FF413AF1F2D11D8C5F12002424558
:1007F0000AAB25F0030028BF424683490192184402
:1008000000F03EFA019A8048FF2100F05FFA4FEABB
:10081000A8037D490193C8F38702284600F05EFAD9
:10082000064600283FF46DAF019B05EB830537E7D3
:100830000220FFF7ABFD00283FF4E8AE00F0A4F97A
:1008400000283FF4E3AE0027B846704B9B68BB42DC
:1008500018D91F2F11D80A9B01330ED027F003039C
:1008600012AA134453F8203C05934046042205A9DC
:1008700000F0ACFA04378046E7E7384600F03AF972
:100880000590F2E7CDF81480042105A800F006F9E0
:1008900006E70023642104A8049300F0F5F800287B
:1008A0007FF4B4AE0220FFF771FD00283FF4AEAE36
:1008B000049800F051F90590E6E70023642104A8AC
:1008C000049300F0E1F800287FF4A0AE0220FFF7C7
:1008D0005DFD00283FF49AAE049800F04DF9EAE778
:1008E0000220FFF753FD00283FF490AE00F05CF9C2
:1008F000E1E70220FFF74AFD00283FF487AE05A993
:10090000142000F057F904210746049004A800F0D1
:10091000C5F83946B9E7322000F0A2F8071EFFF605
:1009200075AEBB077FF472AE384A926807EB0903D5
:1009300093423FF66BAE0220FFF728FD00283FF4FC
:1009400065AE27F003074F44B9453FF4A9AE4846CA
:1009500000F0D0F80421059005A800F09FF809F1F7
:100960000409F1E74FF47A70FFF710FD00283FF417
:100970004DAE00F009F9002844D00A9B01330BD09A
:1009800008220AA9002000F0A9F900283AD0202264
:10099000FF210AA800F09AF9FFF700FD1C4800F0BB
:1009A0003FFF13B0BDE8F08F002E3FF42FAE0BF0E9
:1009B0000B030B2B7FF42AAE0023642105A80593BB
:1009C00000F062F8074600287FF420AE0220FFF70F
:1009D000DDFC804600283FF419AEFFF7DFFC41F252
:1009E000883000F01DFF059800F0EEF9464600F053
:1009F000B9F93C46BBE5064652E64FF0000905E66C
:100A0000BA467EE637467CE65C22002000220020C3
:100A1000A086010070B50F4B1B780133DBB2012BB0
:100A20000C4611D80C4D29684FF47A730E6AA2FB5C
:100A30000332014622462846B047844204D1074B80
:100A400000221A70012070BD4FF4FA7000F0E8FE29
:100A50000020F8E710220020082600209423002020
:100A600007B50023024601210DF107008DF807307C
:100A7000FFF7D0FF20B19DF8070003B05DF804FB3D
:100A80004FF0FF30F9E700000A4608B50421FFF7F0
:100A9000C1FF80F00100C0B2404208BD30B4054C37
:100AA0002368DD69044B0A46AC460146204630BC4B
:100AB000604700BF08260020A086010070B501F045
:100AC000CDF9094E094D30800024286833888342CF
:100AD00008D901F0BDF92B6804440133B4F5803F17
:100AE0002B60F2D370BD00BF962300206823002046
:100AF00001F062BA00F1006000F5803000687047D4
:100B000000F10060920000F5803001F0EDB90000C6
:100B1000054B1A68054B1B889B1A834202D9104467
:100B200001F096B90020704768230020962300202A
:100B300038B5084D044629B128682044BDE838403E
:100B400001F0A6B92868204401F08AF90028F3D002
:100B500038BD00BF6823002010F003030AD1B0F5B0
:100B6000047F05D200F10050A0F51040D0F8003805
:100B7000184670470023FBE700F10050A0F5104035
:100B8000D0F8100A70470000064991F8243033B1BC
:100B90000023086A81F824300822FFF7B1BF012042
:100BA000704700BF6C230020014B1868704700BFDE
:100BB000002004E070B5194B1D68194B0138C5F3CE
:100BC0000B0408442D0C04221E88A6420BD15C683D
:100BD0000A46013C824213460FD214F9016F4EB10E
:100BE00002F8016BF6E7013A03F10803ECD1814208
:100BF0000B4602D22C2203F8012B0A4A0524168840
:100C0000AE4204D1984284BF967803F8016B013C50
:100C100002F10402F3D1581A70BD00BF002004E0B5
:100C20009434000880340008022802BF024B4FF4BD
:100C300000129A61704700BF00040240022802BF00
:100C4000014B20229A61704700040240022801BF34
:100C5000024A536983F02003536170470004024045
:100C600070B504464FF47A764CB1412C254628BF26
:100C7000412506FB05F000F0D3FD641BF4E770BDD1
:100C800010B50023934203D0CC5CC4540133F9E780
:100C900010BD000010B5013810F9013F3BB191F9CA
:100CA00000409C4203D11AB10131013AF4E71AB174
:100CB00091F90020981A10BD1046FCE70346024641
:100CC000D01A12F9011B0029FAD1704702440346D9
:100CD000934202D003F8011BFAE770472DE9F8436D
:100CE0001F4D144695F824200746884652BBDFF86E
:100CF00070909CB395F824302BB92022FF214846F0
:100D00002F62FFF7E3FF95F82400C0F10802A2422A
:100D100028BF2246D6B24146920005EB8000FFF77D
:100D2000AFFF95F82430A41B1E44F6B2082E1744DA
:100D30009044E4B285F82460DBD1FFF725FF00285A
:100D4000D7D108E02B6A03EB82038342CFD0FFF7B1
:100D50001BFF0028CBD10020BDE8F8830120FBE772
:100D60006C230020024B1A78024B1A70704700BFA8
:100D7000942300201022002010B5104C104800F0E1
:100D8000B5F821460E4800F0DDF82468626DD2F80F
:100D9000043843F00203C2F804384FF47A70FFF7C6
:100DA0005FFF0849204600F0D3F9626DD2F804389D
:100DB00023F00203C2F8043810BD00BF60350008FC
:100DC00008260020683500087047000030B5094D3E
:100DD0000A4491420DD011F8013B5840082340F3DA
:100DE0000004013B2C4013F0FF0384EA5000F6D1CD
:100DF000EFE730BD2083B8ED02684368114301601E
:100E000003B118477047000013B5446BD4F894340D
:100E10001A681178042915D1217C022912D1197977
:100E2000128901238B4013420CD101A904F14C001B
:100E300001F0F6FED4F89444019B21790246206823
:100E400000F0D0F902B010BD143001F079BE0000FE
:100E50004FF0FF33143001F073BE00004C3001F04E
:100E60004BBF00004FF0FF334C3001F045BF000096
:100E7000143001F047BE00004FF0FF31143001F094
:100E800041BE00004C3001F017BF00004FF0FF32B0
:100E90004C3001F011BF00000020704710B5D0F8B1
:100EA00094341A6811780429044617D1017C022968
:100EB00014D15979528901238B4013420ED1143039
:100EC00001F0DAFD024648B1D4F894444FF480733F
:100ED00061792068BDE8104000F072B910BD0000D3
:100EE000406BFFF7DBBF0000704700007FB5124B7F
:100EF000036000234360C0E90233012502260F4B43
:100F0000057404460290019300F18402294600967C
:100F10004FF48073143001F08BFD094B0294CDE93E
:100F2000006304F523724FF48073294604F14C00EA
:100F300001F052FE04B070BDB4340008E10E0008A8
:100F4000090E00080B68302282F311880A7903EB3E
:100F5000820290614A79093243F822008A7912B1FB
:100F600003EB820398610223C0F8941403740020F9
:100F700080F311887047000038B5037F044613B131
:100F800090F85430ABB9201D01250221FFF734FF42
:100F900004F1140025776FF0010100F069FC84F87A
:100FA000545004F14C006FF00101BDE8384000F0EE
:100FB0005FBC38BD10B5012104460430FFF71CFFAB
:100FC0000023237784F8543010BD000038B5044660
:100FD0000025143001F044FD04F14C00257701F0A8
:100FE00013FE201D84F854500121FFF705FF204611
:100FF000BDE83840FFF752BF90F8443003F060037B
:10100000202B07D190F84520212A4FF0000303D868
:101010001F2A06D800207047222AFBD1C0E90E33D0
:1010200003E0034A82630722C2630364012070471E
:101030001122002037B5D0F894341A6811780429A9
:1010400004461AD1017C022917D11979128901238A
:101050008B40134211D100F14C05284601F094FE5B
:1010600058B101A9284601F0DBFDD4F89444019B56
:1010700021790246206800F0B5F803B030BD0000C9
:10108000F0B500EB810385B09E6904460D46FEB1C4
:10109000302383F3118804EB8507301D0821FFF707
:1010A000ABFEFB685B691B6806F14C001BB101904D
:1010B00001F0C4FD019803A901F0B2FD024648B158
:1010C000039B2946204600F08DF8002383F3118806
:1010D00005B0F0BDFB685A691268002AF5D01B8A7A
:1010E000013B1340F1D104F14402EAE7093138B57C
:1010F00050F82140DCB1302383F31188D4F89424D4
:101100001368527903EB8203DB689B695D6845B124
:1011100004216018FFF770FE294604F1140001F065
:10112000B5FC2046FFF7BAFE002383F3118838BDD3
:101130007047000001F014B8012303700023C0E9D8
:101140000133C36183620362C36243620363704716
:1011500038B50446302383F311880025C0E90355D0
:10116000C0E90555416001F00BF80223237085F3B7
:101170001188284638BD000070B500EB8103054694
:101180005069DA600E46144618B110220021FFF7AC
:101190009DFDA06918B110220021FFF797FD31468F
:1011A0002846BDE8704001F0B5B80000826802F042
:1011B000011282600022C0E90422826101F036B986
:1011C000F0B400EB81044789E4680125A4698D40EF
:1011D0003D43458123600023A2606360F0BC01F0C1
:1011E00051B90000F0B400EB81040789E4680125DF
:1011F00064698D403D43058123600023A2606360E4
:10120000F0BC01F0CBB9000070B502230025044604
:101210000370C0E90255C0E90455C564856180F8D2
:10122000345001F013F863681B6823B12946204647
:10123000BDE87040184770BD0378052B10B5044613
:101240000AD080F850300523037043681B680BB147
:10125000042198470023A36010BD000001780529F0
:1012600006D190F85020436802701B6803B11847FC
:101270007047000070B590F83430044613B1002375
:1012800080F8343004F14402204601F0F1F863683C
:101290009B68B3B994F8443013F0600535D0002151
:1012A000204601F091FB0021204601F083FB63689A
:1012B0001B6813B1062120469847062384F8343072
:1012C00070BD204698470028E4D0B4F84A30E26B5D
:1012D0009A4288BFE36394F94430E56B002B4FF0EA
:1012E000300380F20381002D00F0F280092284F89F
:1012F000342083F311880021D4E90E232046FFF720
:1013000071FF002383F31188DAE794F8452003F096
:101310007F0343EA022340F20232934200F0C58089
:1013200021D8B3F5807F48D00DD8012B3FD0022BB8
:1013300000F09380002BB2D104F14C02A263022290
:10134000E2632364C1E7B3F5817F00F09B80B3F5CE
:10135000407FA4D194F84630012BA0D1B4F84C3092
:1013600043F0020332E0B3F5006F4DD017D8B3F568
:10137000A06F31D0A3F5C063012B90D8636894F8B7
:1013800046205E6894F84710B4F848302046B047CD
:10139000002884D04368A3630368E3631AE0B3F5CD
:1013A000106F36D040F6024293427FF478AF5C4B28
:1013B000A3630223E3630023C3E794F84630012BC1
:1013C0007FF46DAFB4F84C3023F00203C4E90E553E
:1013D000A4F84C30256478E7B4F84430B3F5A06F36
:1013E0000ED194F8463084F84E30204600F086FF47
:1013F00063681B6813B101212046984703232370BB
:101400000023C4E90E339CE704F14F03A3630123D7
:10141000C3E72378042B10D1302383F311882046AF
:10142000FFF7C4FE85F311880321636884F84F50E9
:1014300021701B680BB12046984794F84630002B6A
:10144000DED084F84F300423237063681B68002BC0
:10145000D6D0022120469847D2E794F848301D069E
:1014600003F00F0120460AD500F0F4FF012804D054
:1014700002287FF414AF2B4B9AE72B4B98E700F030
:10148000DBFFF3E794F84630002B7FF408AF94F8C5
:10149000483013F00F01B3D01A06204602D501F0F0
:1014A000A7FAADE701F09AFAAAE794F84630002BC4
:1014B0007FF4F5AE94F8483013F00F01A0D01B066E
:1014C000204602D501F080FA9AE701F073FA97E717
:1014D000142284F8342083F311882B462A462946A7
:1014E0002046FFF76DFE85F31188E9E65DB1152210
:1014F00084F8342083F311880021D4E90E23204698
:10150000FFF75EFEFDE60B2284F8342083F311889A
:101510002B462A4629462046FFF764FEE3E700BF34
:10152000E4340008DC340008E034000838B590F8F2
:1015300034300446002B3ED0063BDAB20F2A34D8B2
:101540000F2B32D8DFE803F0373131082232313146
:101550003131313131313737C56BB0F84A309D42C6
:1015600014D2C3681B8AB5FBF3F203FB12556DB9A5
:10157000302383F311882B462A462946FFF732FE93
:1015800085F311880A2384F834300EE0142384F89C
:101590003430302383F3118800231A46194620463D
:1015A000FFF70EFE002383F3118838BD036C03B1EF
:1015B00098470023E7E70021204601F005FA0021C3
:1015C000204601F0F7F963681B6813B10621204635
:1015D00098470623D7E7000010B590F83430142B55
:1015E000044629D017D8062B05D001D81BB110BD51
:1015F000093B022BFBD80021204601F0E5F9002130
:10160000204601F0D7F963681B6813B10621204614
:101610009847062319E0152BE9D10B2380F83430C5
:10162000302383F3118800231A461946FFF7DAFDA9
:10163000002383F31188DAE7C3689B695B68002B9A
:10164000D5D1036C03B19847002384F83430CEE73A
:1016500000230375826803691B6899689142FBD275
:101660005A68036042601060586070470023037539
:10167000826803691B6899689142FBD85A680360C5
:10168000426010605860704708B50846302383F305
:1016900011880B7D032B05D0042B0DD02BB983F3C0
:1016A000118808BD8B6900221A604FF0FF338361F7
:1016B000FFF7CEFF0023F2E7D1E9003213605A6052
:1016C000F3E70000FFF7C4BF054BD9680875186839
:1016D00002681A60536001220275D860FEF712BEDC
:1016E0009823002030B50C4BDD684B1C87B00446B6
:1016F0000FD02B46094A684600F04EF92046FFF706
:10170000E3FF009B13B1684600F050F9A86907B0E9
:1017100030BDFFF7D9FFF9E79823002089160008AC
:10172000044B1A68DB6890689B68984294BF00205D
:101730000120704798230020084B10B51C68D8681A
:1017400022681A60536001222275DC60FFF78EFF69
:1017500001462046BDE81040FEF7D4BD9823002086
:1017600038B5074C074908480123002523706560F8
:1017700001F042FB0223237085F3118838BD00BFBE
:1017800000260020EC3400089823002000F044B923
:10179000034A516853685B1A9842FBD8704700BFF0
:1017A000001000E08B60022308618B8208467047BE
:1017B0008368A3F1840243F8142C026943F8442C93
:1017C000426943F8402C094A43F8242CC26843F884
:1017D000182C022203F80C2C002203F80B2C044ACC
:1017E00043F8102CA3F12000704700BF1D03000830
:1017F0009823002008B5FFF7DBFFBDE80840FFF79E
:1018000061BF0000024BDB6898610F20FFF75CBFEF
:1018100098230020302383F31188FFF7F3BF0000E3
:1018200008B50146302383F311880820FFF75AFFDB
:10183000002383F3118808BD064BDB6839B1426889
:1018400018605A60136043600420FFF74BBF4FF0ED
:10185000FF307047982300200368984206D01A682A
:101860000260506099611846FFF72CBF7047000076
:1018700038B504460D462068844200D138BD03685F
:1018800023605C608561FFF71DFFF4E710B5036816
:101890009C68A2420CD85C688A600B604C60216036
:1018A000596099688A1A9A604FF0FF33836010BDBF
:1018B0001B68121BECE700000A2938BF0A2170B52B
:1018C00004460D460A26601901F090FA01F07CFAF0
:1018D000041BA54203D8751C2E460446F3E70A2EC6
:1018E00004D9BDE87040012001F0C6BA70BD000007
:1018F000F8B5144B0D46D96103F1100141600A2A75
:101900001969826038BF0A22016048601861A8180E
:10191000144601F05DFA0A2701F056FA431BA34270
:10192000064606D37C1C281901F060FA2746354686
:10193000F2E70A2F04D9BDE8F840012001F09CBA73
:10194000F8BD00BF98230020F8B506460D4601F00B
:101950003BFA0F4A134653F8107F9F4206D12A469E
:1019600001463046BDE8F840FFF7C2BFD169BB6809
:10197000441A2C1928BF2C46A34202D92946FFF746
:101980009BFF224631460348BDE8F840FFF77EBF83
:1019900098230020A823002010B4C0E903230023CB
:1019A0005DF8044B4361FFF7CFBF000010B5194C41
:1019B000236998420DD0D0E90032816813605A60E3
:1019C0009A680A449A60002303604FF0FF33A361D2
:1019D00010BD2346026843F8102F536000220260B6
:1019E00022699A4203D1BDE8104001F0F9B9936829
:1019F00081680B44936001F0E7F92269E16992681C
:101A0000441AA242E4D91144BDE81040091AFFF774
:101A100053BF00BF982300202DE9F047DFF8BC80BA
:101A200008F110072C4ED8F8105001F0CDF9D8F875
:101A30001C40AA68031B9A423ED81444D5E90032E0
:101A40004FF00009C8F81C4013605A60C5F80090B8
:101A5000D8F81030B34201D101F0C2F989F31188EE
:101A6000D5E9033128469847302383F311886B6901
:101A7000002BD8D001F0A8F96A69A0EB04094A4507
:101A800082460DD2022001F0F7F90022D8F810307A
:101A9000B34208D151462846BDE8F047FFF728BFBA
:101AA000121A2244F2E712EB090938BF4A462946C6
:101AB0003846FFF7EBFEB5E7D8F81030B34208D050
:101AC0001444211AC8F81C00A960BDE8F047FFF7CC
:101AD000F3BEBDE8F08700BFA823002098230020B4
:101AE00000207047FEE70000704700004FF0FF3015
:101AF0007047000002290CD0032904D001290748AF
:101B000018BF00207047032A05D8054800EBC20023
:101B10007047044870470020704700BFC435000874
:101B2000202200207835000870B59AB00546084696
:101B300001A9144600F0C2F801A8FFF7BFF8431C42
:101B40005B00C5E900340022237003236370C6B232
:101B500001AB02341046D1B28E4204F1020401D826
:101B60001AB070BD13F8011B04F8021C04F8010C34
:101B70000132F0E708B5302383F311880348FFF7FB
:101B800059FA002383F3118808BD00BF08260020FE
:101B900090F8443003F01F02012A07D190F8452045
:101BA0000B2A03D10023C0E90E3315E003F06003D4
:101BB000202B08D1B0F848302BB990F84520212AC5
:101BC00003D81F2A04D8FFF717BA222AEBD0FAE766
:101BD000034A82630722C26303640120704700BF87
:101BE0001822002007B5052917D8DFE801F01916DB
:101BF00003191920302383F31188104A0190012121
:101C0000FFF7BAFA01980E4A0221FFF7B5FA0D481C
:101C1000FFF7DCF9002383F3118803B05DF804FBC0
:101C2000302383F311880748FFF7A6F9F2E7302342
:101C300083F311880348FFF7BDF9EBE71835000877
:101C40003C3500080826002038B50C4D0C4C0D49D9
:101C50002A4604F10800FFF767FF05F1CA0204F104
:101C600010000949FFF760FF05F5CA7204F118007A
:101C70000649BDE83840FFF757BF00BFD02A002013
:101C800020220020F8340008023500080D35000835
:101C900070B5044608460D46FFF710F8C6B2204658
:101CA000013403780BB9184670BD32462946FEF759
:101CB000F1FF0028F3D10120F6E700002DE9F047FD
:101CC00005460C46FEF7FAFF2A49C6B22846FFF73A
:101CD000DFFF08B10936F6B227492846FFF7D8FFDB
:101CE00008B11036F6B2632E0BD8DFF88880DFF823
:101CF0008890224FDFF890A02E7846B92670BDE874
:101D0000F08729462046BDE8F04701F09BBB252E11
:101D10002CD1072241462846FEF7BCFF60B9184B7C
:101D2000224603F1100153F8040B42F8040B8B42D6
:101D3000F9D107351034DFE7082249462846FEF777
:101D4000A9FF98B90F4BA21C197809090232C95D85
:101D500002F8041C13F8011B01F00F015345C95D83
:101D600002F8031CF0D118340835C5E704F8016BFC
:101D70000135C1E7E43500080D350008FD350008E0
:101D8000EC350008107AFF1F1C7AFF1FBFF34F8F3E
:101D9000024AD368DB03FCD4704700BF003C02401A
:101DA00008B5094B1B7873B9FFF7F0FF074B1A69A9
:101DB000002ABFBF064A5A6002F188325A601A6888
:101DC00022F480621A6008BD2E2D0020003C0240E3
:101DD0002301674508B50B4B1B7893B9FFF7D6FF76
:101DE000094B1A6942F000421A611A6842F48052A3
:101DF0001A601A6822F480521A601A6842F48062EB
:101E00001A6008BD2E2D0020003C02400B28F0B5C2
:101E100016D80C4C0C4923787BB90C4D0E460C237C
:101E20004FF0006255F8047B46F8042B013B13F099
:101E3000FF033A44F6D10123237051F82000F0BD8E
:101E40000020FCE7602D0020302D00201036000817
:101E5000014B53F820007047103600080C207047E3
:101E60000B2810B5044601D9002010BDFFF7CEFFA6
:101E7000064B53F824301844C21A0BB90120F4E77A
:101E800012680132F0D1043BF6E700BF10360008BB
:101E90000B2810B5044621D8FFF778FFFFF780FF25
:101EA0000F4AF323D360C300DBB243F4007343F063
:101EB00002031361136943F480331361FFF766FF74
:101EC000FFF7A4FF074B53F8241000F0D9F8FFF7F1
:101ED00081FF2046BDE81040FFF7C2BF002010BDC3
:101EE000003C024010360008F8B512F00103144619
:101EF00042D18218B2F1016F57D82D4B1B6813F0F5
:101F0000010352D02B4DFFF74BFFF323EB60FFF79C
:101F10003DFF40F20127032C15D824F00104661878
:101F2000244C401A40F20117B142236900EB01052D
:101F300024D123F001032361FFF74CFF0120F8BDFA
:101F4000043C0430E7E78307E7D12B6923F44073AF
:101F50002B612B693B432B6151F8046B0660BFF387
:101F60004F8FFFF713FF03689E42E9D02B6923F0E0
:101F700001032B61FFF72EFF0020E0E723F44073FD
:101F8000236123693B4323610B882B80BFF34F8F71
:101F9000FFF7FCFE2D8831F8023BADB2AB42C3D057
:101FA000236923F001032361E4E71846C7E700BF74
:101FB00000380240003C0240084908B50B7828B1BF
:101FC0001BB9FFF7EDFE01230B7008BD002BFCD001
:101FD000BDE808400870FFF7FDBE00BF2E2D0020B1
:101FE00010B50244064BD2B2904200D110BD441C41
:101FF00000B253F8200041F8040BE0B2F4E700BF50
:10200000502800400F4B30B51C6F240407D41C6FC0
:1020100044F400741C671C6F44F400441C670A4CB1
:10202000236843F4807323600244084BD2B2904289
:1020300000D130BD441C00B251F8045B43F820507D
:10204000E0B2F4E700380240007000405028004041
:1020500007B5012201A90020FFF7C2FF019803B0D4
:102060005DF804FB13B50446FFF7F2FFA04205D06C
:10207000012201A900200194FFF7C4FF02B010BDA6
:1020800070470000034B1A681AB9034AD2F8742843
:102090001A607047642D00200030024008B5FFF739
:1020A000F1FF024B1868C0F3407008BD642D00209A
:1020B00070470000FEE700000A4B0B480B4A9042B5
:1020C0000BD30B4BDA1C121AC11E22F003028B42F7
:1020D00038BF00220021FEF7F9BD53F8041B40F879
:1020E000041BECE7B8370008602E0020602E0020AB
:1020F000602E002070B5D0E915439E6800224FF095
:10210000FF3504EB42135101D3F800090028BEBF8C
:10211000D3F8000940F08040C3F80009D3F8000B61
:102120000028BEBFD3F8000B40F08040C3F8000B7E
:10213000013263189642C3F80859C3F8085BE0D22D
:102140004FF00113C4F81C3870BD0000890141F044
:102150002001016103699B06FCD41220FFF718BB24
:1021600010B5054C2046FEF7E7FF4FF0A04363652E
:10217000024BA36510BD00BF682D00206436000827
:1021800070B50378012B054650D12A4B446D984217
:102190001BD1294B5A6B42F080025A635A6D42F0B0
:1021A00080025A655A6D5A6942F080025A615A6932
:1021B00022F080025A610E2143205B6900F022FC6C
:1021C0001E4BE3601E4BC4F800380023C4F8003EE9
:1021D000C02323606E6D4FF40413A3633369002B97
:1021E000FCDA012333610C20FFF7D2FA3369DB07F5
:1021F000FCD41220FFF7CCFA3369002BFCDA00265E
:10220000A6602846FFF776FF6B68C4F81068DB68A5
:10221000C4F81468C4F81C684BB90A4BA3614FF0AA
:10222000FF336361A36843F00103A36070BD064BF5
:10223000F4E700BF682D0020003802404014004041
:1022400003002002003C30C0083C30C0F8B5446DAB
:10225000054600212046FFF779FFA96D00234FF0C6
:1022600001128F68C4F834384FF00066C4F81C2897
:102270004FF0FF3004EB431201339F42C2F8006974
:10228000C2F8006BC2F80809C2F8080BF2D20B685A
:102290006A6DEB65636210231361166916F0100610
:1022A000FBD11220FFF774FAD4F8003823F4FE6350
:1022B000C4F80038A36943F4402343F01003A3613A
:1022C0000923C4F81038C4F814380A4BEB604FF0F7
:1022D000C043C4F8103B084BC4F8003BC4F8106975
:1022E000C4F80039EB6D03F1100243F48013EA6582
:1022F000A362F8BD4036000840800010426D90F89F
:102300004E10D2F8003823F4FE6343EA0113C2F8FA
:10231000003870472DE9F84300EB8103456DDA681A
:10232000166806F00306731E022B05EB41130C46DC
:1023300080460FFA81F94FEA41104FF00001C3F8CF
:10234000101B4FF0010104F1100398BFB60401FA0D
:1023500003F391698EBF334E06F1805606F50046B1
:1023600000293AD0578A04F15801490137436F5088
:10237000D5F81C180B43C5F81C382B180021C3F8DE
:10238000101953690127611EA7409BB3138A928BD2
:102390009B08012A88BF5343D8F85C20981842EA6A
:1023A000034301F1400205EB8202C8F85C002146BC
:1023B00053602846FFF7CAFE08EB8900C3681B8AF2
:1023C00043EA8453483464011E432E51D5F81C3827
:1023D0001F43C5F81C78BDE8F88305EB4917D7F80B
:1023E000001B21F40041C7F8001BD5F81C1821EA96
:1023F0000303C0E704F13F0305EB83030A4A5A6075
:1024000028462146FFF7A2FE05EB4910D0F8003917
:1024100023F40043C0F80039D5F81C3823EA070735
:10242000D7E700BF0080001000040002826D126830
:10243000C265FFF75FBE00005831436D49015B582C
:1024400013F4004004D013F4001F0CBF022001203D
:10245000704700004831436D49015B5813F4004058
:1024600004D013F4001F0CBF0220012070470000AD
:1024700000EB8101CB68196A0B6813604B685360ED
:102480007047000000EB810330B5DD68AA6913686E
:10249000D36019B9402B84BF402313606B8A146842
:1024A000426D1C44013CB4FBF3F46343033323F05B
:1024B000030302EB411043EAC44343F0C043C0F8B6
:1024C000103B2B6803F00303012B09B20ED1D2F8A5
:1024D000083802EB411013F4807FD0F8003B14BFA2
:1024E00043F0805343F00053C0F8003B02EB41122D
:1024F000D2F8003B43F00443C2F8003B30BD00007B
:102500002DE9F041244D6E6D06EB40130446D3F8DF
:10251000087BC3F8087B38070AD5D6F814381907A2
:1025200006D505EB84032146DB6828465B6898479F
:10253000FA071FD5D6F81438DB071BD505EB840343
:10254000D968CCB98B69488A5A68B2FBF0F600FBAF
:1025500016228AB91868DA6890420DD2121AC3E9B5
:102560000024302383F311880B482146FFF78AFFAC
:1025700084F31188BDE8F081012303FA04F26B892A
:1025800023EA02036B81CB68002BF3D0214602487B
:10259000BDE8F041184700BF682D002000EB810323
:1025A00070B5DD68436D6C692668E6604A0156BB0C
:1025B0001A444FF40020C2F810092A6802F00302FE
:1025C000012A0AB20ED1D3F8080803EB421410F422
:1025D000807FD4F8000914BF40F0805040F00050D4
:1025E000C4F8000903EB4212D2F8000940F004409D
:1025F000C2F80009D3F83408012202FA01F10143BC
:10260000C3F8341870BD19B9402E84BF4020206033
:1026100020682E8A8419013CB4FBF6F440EAC440D9
:1026200040F000501A44C6E72DE9F8433B4D6E6D6B
:1026300006EB40130446D3F80889C3F8088918F05C
:10264000010F4FEA40171AD0D6F81038DB0716D51D
:1026500005EB8003D9684B691868DA68904230D27C
:10266000121A4FF000091A60C3F80490302383F364
:10267000118821462846FFF791FF89F3118818F049
:10268000800F1CD0D6F834380126A640334216D02D
:1026900005EB84036D6DD3F80CC0DCF81420013415
:1026A000E4B2D2F800E005EB04342F4451687145E0
:1026B00015D3D5F8343823EA0606C5F83468BDE8E2
:1026C000F883012303FA04F22B8923EA02032B8106
:1026D0008B68002BD3D0214628469847CFE7BCF81B
:1026E0001000AEEB0103834228BF0346D7F8180958
:1026F00080B2B3EB800FE2D89068A0F1040959F8DA
:10270000048FC4F80080A0EB09089844B8F1040FC6
:10271000F5D818440B4490605360C7E7682D00203B
:102720002DE9F74FA24C656D6E69AB691E4016F43A
:1027300080586E6107D02046FEF766FD03B0BDE805
:10274000F04F00F047BC002E12DAD5F8003E984852
:102750009B071EBFD5F8003E23F00303C5F8003EDB
:10276000D5F8043823F00103C5F80438FEF776FDE8
:10277000370505D58E48FFF7BDFC8D48FEF75CFD9B
:10278000B0040CD5D5F8083813F0060FEB6823F425
:1027900070530CBF43F4105343F4A053EB60310764
:1027A0001BD56368DB681BB9AB6923F00803AB6119
:1027B0002378052B0CD1D5F8003E7D489A071EBF23
:1027C000D5F8003E23F00303C5F8003EFEF746FDB2
:1027D0006368DB680BB176489847F30274D4B7029C
:1027E00027D5D4F85490DFF8C8B100274FF0010A7C
:1027F00009EB4712D2F8003B03F44023B3F5802FD6
:1028000011D1D2F8003B002B0DDA62890AFA07F3E6
:1028100022EA0303638104EB8703DB68DB6813B1FF
:10282000394658469847A36D01379B68FFB29F42CF
:10283000DED9F00617D5676D3A6AC2F30A1002F0C6
:102840000F0302F4F012B2F5802F00F08580B2F58C
:10285000402F08D104EB83030022DB681B6A07F5D5
:10286000805790426AD13003D5F8184813D5E10358
:1028700002D50020FFF744FEA20302D50120FFF796
:102880003FFE630302D50220FFF73AFE270302D57D
:102890000320FFF735FE75037FF550AFE00702D543
:1028A0000020FFF7C1FEA10702D50120FFF7BCFE03
:1028B000620702D50220FFF7B7FE23077FF53EAF80
:1028C0000320FFF7B1FE39E7636DDFF8E4A0019361
:1028D00000274FF00109A36D9B685FFA87FB9B45BA
:1028E0003FF67DAF019B03EB4B13D3F8001901F4C6
:1028F0004021B1F5802F1FD1D3F8001900291BDA30
:10290000D3F8001941F09041C3F80019D3F8001929
:102910000029FBDB5946606DFFF718FC218909FA95
:102920000BF321EA0303238104EB8B03DB689B6831
:1029300013B15946504698470137CCE7910708BF75
:10294000D7F80080072A98BF03F8018B02F1010233
:1029500098BF4FEA182884E7023304EB830207F597
:1029600080575268D2F818C0DCF80820DCE9001C57
:10297000A1EB0C0C002188420AD104EB83046368AC
:102980009B699A6802449A605A6802445A606AE7EE
:1029900011F0030F08BFD7F800808C4588BF02F8FC
:1029A000018B01F1010188BF4FEA1828E3E700BF5E
:1029B000682D0020436D03EB4111D1F8003B43F437
:1029C0000013C1F8003B7047436D03EB4111D1F890
:1029D000003943F40013C1F800397047436D03EB2D
:1029E0004111D1F8003B23F40013C1F8003B7047BC
:1029F000436D03EB4111D1F8003923F40013C1F802
:102A00000039704700F1604303F561430901C9B221
:102A100083F80013012200F01F039A4043099B0032
:102A200003F1604303F56143C3F880211A607047E6
:102A300030B5039C0172043304FB0325C0E906533F
:102A4000049B03630021059BC160C0E90000C0E94D
:102A50000422C0E90842C0E90A11436330BD000006
:102A6000416A0022C0E90411C0E90A22C2606FF085
:102A70000101FEF7FDBE0000D0E90432934201D10E
:102A8000C2680AB9181D70470020704703691960B1
:102A9000C2680132C260C269134482690361934211
:102AA00024BF436A03610021FEF7D6BE38B5044651
:102AB0000D46E3683BB16269131D1268A3621344BB
:102AC000E362002007E0237A33B929462046FEF767
:102AD000B3FE0028EDDA38BD6FF00100FBE700001F
:102AE000C368C269013BC36043691344826943619F
:102AF000934224BF436A436100238362036B03B1A3
:102B00001847704770B53023044683F31188866AEE
:102B10003EB9FFF7CBFF054618B186F3118828466A
:102B200070BDA36AE26A13F8015BA362934202D309
:102B30002046FFF7D5FF002383F31188EFE700005D
:102B40002DE9F84F04460E46174698464FF03009D7
:102B500089F311880025AA46D4F828B0BBF1000FEC
:102B600009D141462046FFF7A1FF20B18BF3118820
:102B70002846BDE8F88FD4E90A12A7EB050B521AD4
:102B8000934528BF9346BBF1400F1BD9334601F153
:102B9000400251F8040B43F8040B9142F9D1A36AA7
:102BA00040334036A3624035D4E90A239A4202D327
:102BB0002046FFF795FF8AF31188BD42D8D289F3EA
:102BC0001188C9E730465A46FEF75AF8A36A5B44B3
:102BD0005E44A3625D44E7E710B5029C01720433D2
:102BE00003FB0421C0E906130023C0E90A33039B59
:102BF0000363049BC460C0E90000C0E90422C0E98B
:102C00000842436310BD0000026AC260426AC0E924
:102C100004220022C0E90A226FF00101FEF728BE5B
:102C2000D0E904239A4201D1C26822B9184650F86B
:102C3000043B0B60704700231846FAE7C368C2697B
:102C40000133C3604369134482694361934224BFE3
:102C5000436A43610021FEF7FFBD000038B504461A
:102C60000D46E3683BB123691A1DA262E269134471
:102C7000E362002007E0237A33B929462046FEF7B5
:102C8000DBFD0028EDDA38BD6FF00100FBE7000046
:102C900003691960C268013AC260C269134482695B
:102CA0000361934224BF436A036100238362036B81
:102CB00003B118477047000070B530230D46044635
:102CC000114683F31188866A2EB9FFF7C7FF10B14A
:102CD00086F3118870BDA36A1D70A36AE26A01338E
:102CE0009342A36204D3E16920460439FFF7D0FF81
:102CF000002080F31188EDE72DE9F84F04460D46DA
:102D0000904699464FF0300A8AF311880026B34660
:102D1000A76A4FB949462046FFF7A0FF20B187F3C5
:102D200011883046BDE8F88FD4E90A073A1AA8EBB3
:102D30000607974228BF1746402F1BD905F14003CD
:102D400055F8042B40F8042B9D42F9D1A36A403377
:102D5000A3624036D4E90A239A4204D3E1692046AB
:102D60000439FFF795FF8BF311884645D9D28AF3D2
:102D70001188CDE729463A46FDF782FFA36A3B4416
:102D80003D44A3623E44E5E7D0E904239A4217D1CB
:102D9000C3689BB1836A8BB1043B9B1A0ED013604E
:102DA000C368013BC360C3691A44836902619A42E4
:102DB00024BF436A036100238362012318467047DE
:102DC0000023FBE700F030B94FF08043586A7047AA
:102DD0004FF08043002258631A610222DA60704784
:102DE0004FF080430022DA60704700004FF08043CC
:102DF00058637047FEE7000070B51B4B0163002568
:102E0000044686B0586085620E4600F0BFF804F1B3
:102E10001003C4E904334FF0FF33C4E90635C4E9B5
:102E20000044A560E562FFF7CFFF2B460246C4E9E8
:102E3000082304F134010D4A256580232046FEF75E
:102E4000B1FC0123E0600A4A0375009272680192A6
:102E5000B268CDE90223074B6846CDE90435FEF799
:102E6000C9FC06B070BD00BF002600207036000807
:102E700075360008F52D0008024AD36A1843D0625F
:102E8000704700BF982300204B6843608B688360C5
:102E9000CB68C3600B6943614B6903628B69436212
:102EA0000B6803607047000008B5264B26481A6976
:102EB00040F2FF110A431A611A6922F4FF7222F0EC
:102EC00001021A611A691A6B0A431A631A6D0A43DE
:102ED0001A651E4A1B6D1146FFF7D6FF02F11C0151
:102EE00000F58060FFF7D0FF02F1380100F5806047
:102EF000FFF7CAFF02F1540100F58060FFF7C4FF3D
:102F000002F1700100F58060FFF7BEFF02F18C0155
:102F100000F58060FFF7B8FF02F1A80100F58060BE
:102F2000FFF7B2FF02F1C40100F58060FFF7ACFFCC
:102F300002F1E00100F58060FFF7A6FFBDE8084060
:102F400000F0EEB800380240000002407C36000875
:102F500008B500F059FAFEF703FCFFF793F8BDE857
:102F60000840FEF771BE000070470000EFF30983D0
:102F700005494A6B22F001024A63683383F30988EA
:102F8000002383F31188704700EF00E0302080F3C6
:102F9000118862B60C4B0D4AD96821F4E06109042E
:102FA000090C0A43DA60D3F8FC20094942F0807228
:102FB000C3F8FC200A6842F001020A602022DA7796
:102FC00083F82200704700BF00ED00E00003FA051F
:102FD000001000E010B5302383F311880E4B5B68BE
:102FE00013F4006314D0F1EE103AEFF30984683C57
:102FF0004FF08073E361094BDB6B236684F3098830
:10300000FEF78EFB10B1064BA36110BD054BFBE72D
:1030100083F31188F9E700BF00ED00E000EF00E066
:103020002F030008320300080F4B1A6C42F0010214
:103030001A641A6E42F001021A660C4A1B6E9368FB
:1030400043F0010393604FF0804353229A624FF0A4
:10305000FF32DA6200229A615A63DA605A60012212
:103060005A611A60704700BF00380240002004E037
:103070004FF0804208B51169D3680B40D9B2C943FB
:103080009B07116107D5302383F31188FEF77EFB80
:10309000002383F3118808BD1F4B1A696FEAC252DF
:1030A0006FEAD2521A611A69C2F308021A614FF02C
:1030B000FF301A695A69586100215A6959615A6981
:1030C0001A6A62F080521A621A6A02F080521A6218
:1030D0001A6A5A6A58625A6A59625A6A1A6C42F0F3
:1030E00080521A641A6E42F080521A661A6E0B4AA7
:1030F000106840F480701060186F00F44070B0F5F4
:10310000007F1EBF4FF4803018671967536823F49F
:103110000073536000F054B9003802400070004062
:10312000334B4FF080521A64324A4FF440411160E1
:103130001A6842F001021A601A689107FCD59A6871
:1031400022F003029A602A4B9A6812F00C02FBD11B
:10315000196801F0F90119609A601A6842F4803226
:103160001A601A689203FCD55A6F42F001025A673E
:103170001F4B5A6F9007FCD51F4A5A601A6842F0DD
:1031800080721A601B4A53685904FCD5184B1A68A0
:103190009201FCD5194A9A60194B1A68194B9A4248
:1031A000194B21D1194A1168194A91421CD140F298
:1031B00005121A60144A136803F00F03052BFAD1A5
:1031C0000B4B9A6842F002029A609A6802F00C0275
:1031D000082AFAD15A6C42F480425A645A6E42F478
:1031E00080425A665B6E704740F20572E1E700BFAD
:1031F00000380240007000400854400700948838AE
:10320000002004E011640020003C024000ED00E0DA
:1032100041C20F41074A08B5536903F001035361E6
:1032200023B1054A13680BB150689847BDE80840C0
:10323000FFF7D0BE003C0140E02D0020074A08B552
:10324000536903F00203536123B1054A93680BB13C
:10325000D0689847BDE80840FFF7BCBE003C01407D
:10326000E02D0020074A08B5536903F004035361B9
:1032700023B1054A13690BB150699847BDE808406E
:10328000FFF7A8BE003C0140E02D0020074A08B52A
:10329000536903F00803536123B1054A93690BB1E5
:1032A000D0699847BDE80840FFF794BE003C014054
:1032B000E02D0020074A08B5536903F0100353615D
:1032C00023B1054A136A0BB1506A9847BDE808401C
:1032D000FFF780BE003C0140E02D0020164B10B5EA
:1032E0005C6904F478725A61A30604D5134A936AA0
:1032F0000BB1D06A9847600604D5104A136B0BB126
:10330000506B9847210604D50C4A936B0BB1D06BD8
:103310009847E20504D5094A136C0BB1506C9847E5
:10332000A30504D5054A936C0BB1D06C9847BDE852
:103330001040FFF74FBE00BF003C0140E02D0020D1
:10334000194B10B55C6904F47C425A61620504D5DE
:10335000164A136D0BB1506D9847230504D5134AD7
:10336000936D0BB1D06D9847E00404D50F4A136EEE
:103370000BB1506E9847A10404D50C4A936E0BB163
:10338000D06E9847620404D5084A136F0BB1506F92
:103390009847230404D5054A936F0BB1D06F984723
:1033A000BDE81040FFF716BE003C0140E02D0020B4
:1033B00008B5FFF75DFEBDE80840FFF70BBE000053
:1033C000062108B50846FFF71DFB06210720FFF779
:1033D00019FB06210820FFF715FB06210920FFF73E
:1033E00011FB06210A20FFF70DFB06211720FFF72E
:1033F00009FB06212820FFF705FBBDE8084007214F
:103400001C20FFF7FFBA000008B5FFF745FE00F0EB
:103410000BF8FDF78FFEFDF767FDFFF7A5FDBDE893
:103420000840FFF7CFBC00000023054A19460133CE
:10343000102BC2E9001102F10802F8D1704700BF59
:10344000E02D0020034611F8012B03F8012B002A80
:10345000F9D1704753544D3332463F3F3F005354E8
:103460004D3332463430780053544D333246343283
:10347000780053544D3332463434365858000000E7
:10348000012033000010410001105A0003105900C0
:10349000071031000000000054340008130400003D
:1034A0005E3400081904000068340008210400009C
:1034B0007234000800000000650E0008510E00087C
:1034C0008D0E0008790E0008850E0008710E0008A8
:1034D0005D0E0008490E0008990E0008000000006B
:1034E000010000000000000063300000E834000824
:1034F000F0230020002600204172647550696C6F33
:10350000740025424F415244252D424C002553451D
:103510005249414C2500000002000000000000005C
:1035200081100008ED10000840004000A02A002093
:10353000B02A00200200000000000000030000008C
:103540000000000031110008000000001000000021
:10355000C02A002000000000010000000000000060
:10356000682D002001010200E51B0008F51A000883
:10357000911B0008751B00084300000080350008FF
:1035800009024300020100C03209040000010202E6
:103590000100052400100105240100010424020299
:1035A0000524060001070582030800FF0904010045
:1035B000020A000000070501024000000705810221
:1035C0004000000012000000CC350008120110017C
:1035D00002000040091241570002010203010000ED
:1035E0000403090425424F41524425006F6D6E6962
:1035F000627573663470726F2D6F6E650030313294
:1036000033343536373839414243444546000000AB
:1036100000400000004000000040000000400000AA
:103620000000010000000200000002000000020093
:103630000000020000000200000002000000020082
:1036400000000000751200082D150008D9150008AB
:1036500040004000C82D0020C82D002001000000BF
:10366000D82D002080000000400100000300000071
:103670006D61696E0069646C650000000001804244
:1036800000000000AAAAAAAA00010040FFFF000053
:103690000000000000A00A0040050001000000003A
:1036A000AAAAAAAA40020001CFFF00000000000061
:1036B000000000000000000000000000AAAAAAAA62
:1036C00000000000FFFF00000000000000000000FC
:1036D0000000000000000000AAAAAAAA0000000042
:1036E000FFFF0000000000000000000000000000DC
:1036F00000000000AAAAAAAA00000000FFFF000024
:1037000000000000000000000000000000000000B9
:10371000AAAAAAAA00000000FFFF00000000000003
:10372000000000000000000000000000AAAAAAAAF1
:1037300000000000FFFF000000000000000000008B
:1037400000000000000000000A000000000000006F
:103750000300000000000000000000000000000066
:103760000000000000000000000000000000000059
:1037700000000000000000008300000000000000C6
:1037800000000F0000000000FF009600000000088D
:10379000009600000000080004000000E03500086A
:1037A0000000000000000000000000000000000019
:1037B0000000000000000000FFFFFFFFFFFFFFFF11
:1037C000FFFFFFFFFFFFFFFFFFFFFFFFFFFFFFFF09
:1037D000FFFFFFFFFFFFFFFFFFFFFFFFFFFFFFFFF9
:1037E000FFFFFFFFFFFFFFFFFFFFFFFFFFFFFFFFE9
:1037F000FFFFFFFFFFFFFFFFFFFFFFFFFFFFFFFFD9
:020000040801F1
:1000000000060020B5120108B94E0908154E09086E
:10001000814E0908154E09084D4E0908B71201080E
:10002000B7120108B7120108B7120108B1A50B08F1
:10003000B7120108B7120108B7120108B712010878
:10004000B7120108B7120108B7120108B712010868
:10005000B7120108B712010849B10B0871B10B08BA
:1000600099B10B08C1B10B08E9B10B08351A0B089F
:100070005D1A0B08891A0B08B51A0B08E11A0B0850
:10008000091B0B08351B0B08B9190B08B71201081F
:10009000B7120108B7120108B712010811B20B0814
:1000A00035B30B0839B30B084DB30B0851B30B082C
:1000B00055B30B0869B30B087DB30B08B7120108E1
:1000C000B7120108C1200B0869220B08B7120108FA
:1000D000B7120108E5B20B08B7120108F9B20B0814
:1000E00075B20B08B7120108B7120108A1B30B08CB
:1000F000A5B30B08B9B30B08BDB30B08611B0B0804
:10010000B7120108B712010891B30B08B712010822
:100110000DB30B08B7120108B7120108B712010896
:100120008D1B0B08B51B0B08E11B0B080D1C0B08E6
:10013000391C0B08B7120108B7120108B7120108E1
:10014000B7120108B7120108B7120108DDAC0B089D
:10015000611C0B088D1C0B08B91C0B0821B30B0884
:10016000B7120108B7120108B7120108B712010847
:10017000B7120108B7120108B7120108B712010837
:10018000B7120108B7120108B7120108B712010827
:10019000B7120108B7120108B7120108B712010817
:1001A000B7120108B7120108B7120108B712010807
:1001B000B7120108B7120108B7120108B7120108F7
:1001C000B7120108B7120108B7120108B7120108E7
:1001D000B7120108B7120108B7120108B7120108D7
:1001E000C55701083D8502089DEC030895AA05083E
:1001F00095B00508410F0608C5730608897B0608F7
:10020000C17E060805E40608210B070895E00708EB
:10021000813B0808D94808086D400908514509087C
:1002200019460A0891A10A08E9C70A08A1D20A08D2
:1002300069020B0849090B080000000000000000DB
:1002400081F0004102E000BF83F0004330B54FEA87
:1002500041044FEA430594EA050F08BF90EA020FF4
:100260001FBF54EA000C55EA020C7FEA645C7FEA87
:10027000655C00F0E2804FEA5454D4EB5555B8BFAA
:100280006D420CDD2C4480EA020281EA030382EA1B
:10029000000083EA010180EA020281EA0303362DAD
:1002A00088BF30BD11F0004F4FEA01314FF4801C80
:1002B0004CEA113102D0404261EB410113F0004F92
:1002C0004FEA03334CEA133302D0524263EB430349
:1002D00094EA050F00F0A780A4F10104D5F1200EE7
:1002E0000DDB02FA0EFC22FA05F2801841F1000142
:1002F00003FA0EF2801843FA05F359410EE0A5F116
:1003000020050EF1200E012A03FA0EFC28BF4CF046
:10031000020C43FA05F3C01851EBE37101F00045FC
:1003200007D54FF0000EDCF1000C7EEB00006EEB09
:100330000101B1F5801F1BD3B1F5001F0CD3490893
:100340005FEA30004FEA3C0C04F101044FEA4452EA
:1003500012F5800F80F09A80BCF1004F08BF5FEA71
:10036000500C50F1000041EB045141EA050130BD51
:100370005FEA4C0C404141EB0101013C28BFB1F563
:10038000801FE9D291F0000F04BF01460020B1FAAE
:1003900081F308BF2033A3F10B03B3F120020CDA81
:1003A0000C3208DD02F1140CC2F10C0201FA0CF05F
:1003B00021FA02F10CE002F11402D8BFC2F1200CC4
:1003C00001FA02F120FA0CFCDCBF41EA0C0190407A
:1003D000E41AA2BF01EB0451294330BD6FEA0404C3
:1003E0001F3C1CDA0C340EDC04F11404C4F12002AE
:1003F00020FA04F001FA02F340EA030021FA04F3C0
:1004000045EA030130BDC4F10C04C4F1200220FA16
:1004100002F001FA04F340EA0300294630BD21FA54
:1004200004F0294630BD94F0000F83F4801306BF1A
:1004300081F480110134013D4EE77FEA645C18BF0E
:100440007FEA655C29D094EA050F08BF90EA020FA5
:1004500005D054EA000C04BF1946104630BD91EA9D
:10046000030F1EBF0021002030BD5FEA545C05D1A0
:100470004000494128BF41F0004130BD14F58004DF
:100480003CBF01F5801130BD01F0004545F0FE4153
:1004900041F470014FF0000030BD7FEA645C1ABF88
:1004A000194610467FEA655C1CBF0B46024650EABF
:1004B000013406BF52EA033591EA030F41F40021EB
:1004C00030BD00BF90F0000F04BF0021704730B571
:1004D0004FF4806404F132044FF000054FF0000146
:1004E00050E700BF90F0000F04BF0021704730B507
:1004F0004FF4806404F1320410F0004548BF4042DC
:100500004FF000013EE700BF42004FEAE2014FEA30
:1005100031014FEA02701FBF12F07F4393F07F4F0B
:1005200081F06051704732F07F4208BF704793F00E
:100530007F4F04BF41F40021704730B54FF4607421
:1005400001F0004521F000411CE700BF50EA010224
:1005500008BF704730B54FF000050AE050EA0102CD
:1005600008BF704730B511F0004502D5404261EB3D
:1005700041014FF4806404F132045FEA915C3FF47E
:10058000D8AE4FF003025FEADC0C18BF03325FEA1B
:10059000DC0C18BF033202EBDC02C2F1200300FACC
:1005A00003FC20FA02F001FA03FE40EA0E0021FAF1
:1005B00002F11444BDE600BF70B54FF0FF0C4CF4DF
:1005C000E06C1CEA11541DBF1CEA135594EA0C0F91
:1005D00095EA0C0F00F0DEF82C4481EA030621EACC
:1005E0004C5123EA4C5350EA013518BF52EA033507
:1005F00041F4801143F4801338D0A0FB02CE4FF0B9
:100600000005E1FB02E506F00042E0FB03E54FF0E8
:100610000006E1FB03569CF0000F18BF4EF0010EE0
:10062000A4F1FF04B6F5007F64F5407404D25FEADC
:100630004E0E6D4146EB060642EAC62141EA55518F
:100640004FEAC52040EA5E504FEACE2EB4F1FD0CD1
:1006500088BFBCF5E06F1ED8BEF1004F08BF5FEA4F
:10066000500E50F1000041EB045170BD06F0004601
:1006700046EA010140EA020081EA0301B4EB5C04AE
:10068000C2BFD4EB0C0541EA045170BD41F48011A6
:100690004FF0000E013C00F3AB8014F1360FDEBFCB
:1006A000002001F0004170BDC4F10004203C35DAA7
:1006B0000C341BDC04F11404C4F1200500FA05F32A
:1006C00020FA04F001FA05F240EA020001F00042CB
:1006D00021F0004110EBD37021FA04F642EB060141
:1006E0005EEA430E08BF20EAD37070BDC4F10C046B
:1006F000C4F1200500FA04F320FA05F001FA04F22F
:1007000040EA020001F0004110EBD37041F100011A
:100710005EEA430E08BF20EAD37070BDC4F1200525
:1007200000FA05F24EEA020E20FA04F301FA05F28D
:1007300043EA020321FA04F001F0004121FA04F235
:1007400020EA020000EBD3705EEA430E08BF20EA05
:10075000D37070BD94F0000F0FD101F0004640003F
:1007600041EB010111F4801F08BF013CF7D041EAC1
:10077000060195F0000F18BF704703F000465200C5
:1007800043EB030313F4801F08BF013DF7D043EA96
:100790000603704794EA0C0F0CEA135518BF95EA4C
:1007A0000C0F0CD050EA410618BF52EA4306D1D1D3
:1007B00081EA030101F000414FF0000070BD50EAF2
:1007C000410606BF1046194652EA430619D094EA7C
:1007D0000C0F02D150EA013613D195EA0C0F05D166
:1007E00052EA03361CBF104619460AD181EA0301BA
:1007F00001F0004141F0FE4141F470014FF0000072
:1008000070BD41F0FE4141F4780170BD70B54FF00C
:10081000FF0C4CF4E06C1CEA11541DBF1CEA13558C
:1008200094EA0C0F95EA0C0F00F0A7F8A4EB05046E
:1008300081EA030E52EA03354FEA013100F0888065
:100840004FEA03334FF0805545EA131343EA12632E
:100850004FEA022245EA111545EA10654FEA0026E3
:100860000EF000419D4208BF964244F1FD0404F59C
:10087000407402D25B084FEA3202B61A65EB0305F8
:100880005B084FEA32024FF480104FF4002CB6EBB5
:10089000020E75EB030E22BFB61A754640EA0C0035
:1008A0005B084FEA3202B6EB020E75EB030E22BF75
:1008B000B61A754640EA5C005B084FEA3202B6EBB6
:1008C000020E75EB030E22BFB61A754640EA9C0075
:1008D0005B084FEA3202B6EB020E75EB030E22BF45
:1008E000B61A754640EADC0055EA060E18D04FEA03
:1008F000051545EA16754FEA06164FEAC30343EAA3
:1009000052734FEAC2025FEA1C1CC0D111F4801F6F
:100910000BD141EA00014FF000004FF0004CB6E768
:1009200011F4801F04BF01430020B4F1FD0C88BF07
:10093000BCF5E06F3FF6AFAEB5EB030C04BFB6EB12
:10094000020C5FEA500C50F1000041EB045170BD05
:100950000EF0004E4EEA113114EB5C04C2BFD4EB32
:100960000C0541EA045170BD41F480114FF0000EB6
:10097000013C90E645EA060E8DE60CEA135594EA32
:100980000C0F08BF95EA0C0F3FF43BAF94EA0C0F35
:100990000AD150EA01347FF434AF95EA0C0F7FF4AA
:1009A00025AF104619462CE795EA0C0F06D152EAFE
:1009B00003353FF4FDAE1046194622E750EA4106E2
:1009C00018BF52EA43067FF4C5AE50EA41047FF4F3
:1009D0000DAF52EA43057FF4EBAE12E74FF0FF3C58
:1009E00006E000BF4FF0010C02E000BF4FF0010C29
:1009F0004DF804CD4FEA410C7FEA6C5C4FEA430CA2
:100A000018BF7FEA6C5C1BD001B050EA410C0CBFF0
:100A100052EA430C91EA030F02BF90EA020F002052
:100A2000704710F1000F91EA030F58BF994208BFB9
:100A300090422CBFD8176FEAE37040F00100704776
:100A40004FEA410C7FEA6C5C02D150EA013C07D1CD
:100A50004FEA430C7FEA6C5CD6D152EA033CD3D018
:100A60005DF8040B704700BF8446104662468C4612
:100A70001946634600E000BF01B5FFF7B7FF002845
:100A800048BF10F1000F01BD4DF808EDFFF7F4FF6E
:100A90000CBF012000205DF808FB00BF4DF808EDF9
:100AA000FFF7EAFF34BF012000205DF808FB00BF1C
:100AB0004DF808EDFFF7E0FF94BF012000205DF83E
:100AC00008FB00BF4DF808EDFFF7CEFF94BF0120F3
:100AD00000205DF808FB00BF4DF808EDFFF7C4FFEC
:100AE00034BF012000205DF808FB00BF4FEA410C35
:100AF0007FEA6C5C02D150EA013C0AD14FEA430C18
:100B00007FEA6C5C02D152EA033C02D14FF0000054
:100B100070474FF0010070474FEA410212F5001292
:100B200015D211D56FF47873B3EB625212D94FEA34
:100B3000C12343F0004343EA505311F0004F23FA1E
:100B400002F018BF404270474FF00000704750EA73
:100B5000013005D111F0004008BF6FF00040704730
:100B60004FF00000704700BF4A0011D212F500128A
:100B700011D20DD56FF47873B3EB62520ED44FEAF5
:100B8000C12343F0004343EA505323FA02F0704775
:100B90004FF00000704750EA013002D14FF0FF30B3
:100BA00070474FF0000070474FEA4102B2F1E04356
:100BB00024BFB3F5001CDCF1FE5C0DD901F0004C44
:100BC0004FEAC0024CEA5070B2F1004F40EB830094
:100BD00008BF20F00100704711F0804F21D113F1C0
:100BE0003872BCBF01F00040704741F480114FEAF9
:100BF0005252C2F11802C2F1200C10FA0CF320FA82
:100C000002F018BF40F001004FEAC1234FEAD3239E
:100C100003FA0CFC40EA0C0023FA02F34FEA430308
:100C2000CCE77FEA625307D150EA01331EBF4FF091
:100C3000FE4040F44000704701F0004040F0FE40AC
:100C400040F40000704700BF80F0004002E000BFA9
:100C500081F0004142001FBF5FEA410392EA030FA7
:100C60007FEA226C7FEA236C6AD04FEA1262D2EBF1
:100C70001363C1BFD218414048404140B8BF5B42F6
:100C8000192B88BF704710F0004F40F4000020F08F
:100C90007F4018BF404211F0004F41F4000121F0A5
:100CA0007F4118BF494292EA030F3FD0A2F10102EF
:100CB00041FA03FC10EB0C00C3F1200301FA03F12D
:100CC00000F0004302D5494260EB4000B0F5000F50
:100CD00013D3B0F1807F06D340084FEA310102F10F
:100CE0000102FE2A51D2B1F1004F40EBC25008BFC1
:100CF00020F0010040EA03007047490040EB00008B
:100D0000013A28BFB0F5000FEDD2B0FA80FCACF18B
:100D1000080CB2EB0C0200FA0CF0AABF00EBC250B8
:100D200052421843BCBFD0401843704792F0000FA6
:100D300081F4000106BF80F400000132013BB5E7F9
:100D40004FEA41037FEA226C18BF7FEA236C21D06F
:100D500092EA030F04D092F0000F08BF08467047D4
:100D600090EA010F1CBF0020704712F07F4F04D1A2
:100D7000400028BF40F00040704712F100723CBFB5
:100D800000F50000704700F0004343F0FE4040F4DF
:100D9000000070477FEA226216BF08467FEA23639D
:100DA0000146420206BF5FEA412390EA010F40F488
:100DB000800070474FF0000304E000BF10F00043D4
:100DC00048BF40425FEA000C08BF704743F09643BB
:100DD00001464FF000001CE050EA010208BF7047D6
:100DE0004FF000030AE000BF50EA010208BF70475D
:100DF00011F0004302D5404261EB41015FEA010C72
:100E000002BF84460146002043F0B64308BFA3F169
:100E10008053A3F50003BCFA8CF2083AA3EBC2534B
:100E200010DB01FA02FC634400FA02FCC2F120026A
:100E3000BCF1004F20FA02F243EB020008BF20F0A1
:100E40000100704702F1200201FA02FCC2F1200207
:100E500050EA4C0021FA02F243EB020008BF20EAFC
:100E6000DC7070477BB972B90029BEBF00204FF01B
:100E7000004106E008BF00281CBF6FF000414FF0A2
:100E8000FF3000F015BAADF1080C6DE904CE002971
:100E900009DB002B1ADB00F0A3F8DDF804E0DDE944
:100EA000022304B07047404261EB4101002B1BDB81
:100EB00000F096F8DDF804E0DDE9022304B04042DA
:100EC00061EB4101524263EB43037047524263EBD3
:100ED000430300F085F8DDF804E0DDE9022304B007
:100EE000404261EB41017047524263EB430300F023
:100EF00077F8DDF804E0DDE9022304B0524263EB49
:100F00004303704753B94AB9002908BF00281CBFE2
:100F10004FF0FF314FF0FF3000F0CAB9ADF1080CCF
:100F20006DE904CE00F05CF8DDF804E0DDE90223B1
:100F300004B0704730B1012390FAA0F0B0FA80F00D
:100F40001844704708460029FBD02123F4E700BF6E
:100F5000430803F05533C01A830803F0333300F01D
:100F60003330184400EB101000F00F3000EB00207D
:100F700000EB0040000E704707EE900AF5EEC07AD5
:100F8000F1EE10FA01D400F00BB8F1EE677A08B573
:100F900017EE900A00F004F8404261EB410108BDF1
:100FA000D0B5FFF7B1FA0C4B002206460F46FFF70B
:100FB00003FBFFF7D9FD0446FFF784FA074B002235
:100FC000FFF7FAFA02460B4630463946FFF73CF97E
:100FD000FFF7CAFD2146D0BD0000F03D0000F04102
:100FE0002DE9F047089D04468E46002B4DD18A42DC
:100FF000944669D9B2FA82F252B101FA02F3C2F10F
:10100000200120FA01F10CFA02FC41EA030E94409F
:101010004FEA1C48210CBEFBF8F61FFA8CF708FBC0
:1010200016E341EA034306FB07F199420AD91CEB98
:10103000030306F1FF3080F01F81994240F21C81CA
:10104000023E63445B1AA4B2B3FBF8F008FB103312
:1010500044EA034400FB07F7A7420AD91CEB040447
:1010600000F1FF3380F00A81A74240F20781644417
:10107000023840EA0640E41B00261DB1D44000239C
:10108000C5E900433146BDE8F0878B4209D9002D00
:1010900000F0EF800026C5E9000130463146BDE88A
:1010A000F087B3FA83F6002E4AD18B4202D38242F4
:1010B00000F2F980841A61EB030301209E46002DA3
:1010C000E0D0C5E9004EDDE702B9FFDEB2FA82F2F8
:1010D000002A40F09280A1EB0C014FEA1C471FFA56
:1010E0008CFE0126200CB1FBF7F307FB131140EA3D
:1010F00001410EFB03F0884208D91CEB010103F10A
:10110000FF3802D2884200F2CB804346091AA4B2CB
:10111000B1FBF7F007FB101144EA01440EFB00FE9F
:10112000A64508D91CEB040400F1FF3102D2A64504
:1011300000F2BB800846A4EB0E0440EA03409CE7A3
:10114000C6F12007B34022FA07FC4CEA030C20FA50
:1011500007F401FA06F31C43F9404FEA1C4900FA70
:1011600006F3B1FBF9F8200C1FFA8CFE09FB1811ED
:1011700040EA014108FB0EF0884202FA06F20BD960
:101180001CEB010108F1FF3A80F08880884240F2B0
:101190008580A8F102086144091AA4B2B1FBF9F0F4
:1011A00009FB101144EA014100FB0EFE8E4508D9EF
:1011B0001CEB010100F1FF346CD28E456AD9023874
:1011C000614440EA0840A0FB0294A1EB0E01A14259
:1011D000C846A64656D353D05DB1B3EB080261EBC7
:1011E0000E0101FA07F722FA06F3F1401F43C5E9A1
:1011F000007100263146BDE8F087C2F12003D840D7
:101200000CFA02FC21FA03F3914001434FEA1C4718
:101210001FFA8CFEB3FBF7F007FB10360B0C43EA0A
:10122000064300FB0EF69E4204FA02F408D91CEBBA
:10123000030300F1FF382FD29E422DD902386344B8
:101240009B1B89B2B3FBF7F607FB163341EA034158
:1012500006FB0EF38B4208D91CEB010106F1FF38A7
:1012600016D28B4214D9023E6144C91A46EA00469E
:1012700038E72E46284605E70646E3E61846F8E630
:101280004B45A9D2B9EB020864EB0C0E0138A3E779
:101290004646EAE7204694E74046D1E7D0467BE75A
:1012A000023B614432E7304609E76444023842E7D2
:1012B000704700BF02E000F000F8FEE772B6374862
:1012C00080F30888364880F3098836483649086034
:1012D00040F20000CCF200004EF63471CEF2000174
:1012E0000860BFF34F8FBFF36F8F40F20000C0F272
:1012F000F0004EF68851CEF200010860BFF34F8F28
:10130000BFF36F8F4FF00000E1EE100A4EF63C7114
:10131000CEF200010860062080F31488BFF36F8FBF
:10132000A9F0A4F9A4F078FB4FF055301F491B4AEF
:1013300091423CBF41F8040BFAE71D49184A91421B
:101340003CBF41F8040BFAE71A491B4A1B4B9A426F
:101350003EBF51F8040B42F8040BF8E7002018498F
:10136000184A91423CBF41F8040BFAE7A9F082F910
:10137000A4F0A6FB144C154DAC4203DA54F8041B40
:101380008847F9E701F0F4F8114C124DAC4203DA4A
:1013900054F8041B8847F9E7A9F06AB90006002051
:1013A000002200200000010808ED00E000000020FD
:1013B00000060020D8350E0800220020842C0020D2
:1013C000882C0020684F0120E00101083802010844
:1013D00038020108380201082DE9F04F2DED108A7E
:1013E000C1F80CD0C3689D46BDEC108ABDE8F08FF3
:1013F000002383F311882846A0470020A4F008F9B1
:10140000FEE7A3F065FF00DFFEE7000001F0FF014B
:10141000102A2BDB10F0070F08D010F8013B013A1F
:101420008B422DD010F0070F42B3F6D1F0B441EA51
:10143000012141EA014122F007047FF00007002367
:10144000F0E80256083C85EA010586EA010685FABD
:1014500047F5A3FA87F586FA47F6A5FA87F68EB917
:10146000EED1F0BC01F0FF0102F0070232B110F83A
:10147000013B013A83EA010313B1F8D10020704720
:1014800001387047002D06BF35460338073815F080
:10149000010F07D1013015F4807F02BF013015F430
:1014A000C03F0130F0BC0138704700BF10F8012B7D
:1014B00011F8013B012A28BF9A42F7D0D01A704791
:1014C000034613F8012B002AFBD1181A0138704784
:1014D00038B50022002304460D46FFF7DFFA28B98D
:1014E00020462946BDE8384000F00AB8204605F1FC
:1014F000004100F005F8404261EB410138BD00BFFA
:10150000D0B50C4B002206460F46FFF755F8FFF703
:101510002BFB0446FEF7D6FF074B0022FFF74CF8E3
:1015200002460B4630463946FEF78EFEFFF71CFB9F
:101530002146D0BD0000F03D0000F04103680022CC
:101540001B68184710B503685B680446984708B1E4
:1015500094F84D0010BD000038B504467BF08AFDBC
:101560000E4B1D680146E86A02681268904751F008
:1015700089FCEB6A93F89C1050F070FC94F83730BB
:101580005BB183F0CFFCEB6AD3F8A030C01AB0F5A2
:10159000FA6F24BF002384F8373038BD942C002024
:1015A00070B50E4605465DF04DF95DF00FF910B9C6
:1015B0000124204670BD0A4B93F94632012BF7D126
:1015C0005DF040F9437A002BF2D15DF03BF9847A6B
:1015D000002CEDD1034A314628467BF089FFE8E72D
:1015E000984C0020AC290C08034BD3F8B0320BB94F
:1015F0007BF0F6BC01207047984C00202DE9F043A9
:101600002DED028BC47F91B006460F468CB990F940
:101610000430002B00F0FE807F4B1D68A86A036831
:101620005B6B9847044650B97C4A394630467BF09C
:101630005FFF204611B0BDEC028BBDE8F083B368BC
:101640004BB933685B6B3946304611B0BDEC028B49
:10165000BDE8F0431847E86AFFF774FF0446002826
:10166000E7D1394630467CF037FEDFF8E4810546A5
:10167000394630467BF064FF98ED967AD8ED957A3E
:10168000B4EEE77A2840F1EE10FAC5B209D598F920
:101690005032032B05D0624A394630467BF028FF92
:1016A0002546D8ED7E7AB0EE088AF4EEC87AF1EEDF
:1016B00010FA0BD517EE900AFEF726FF594ACDE92E
:1016C0000001394630467BF013FF0025D8ED7F7AC4
:1016D000F4EEC87AF1EE10FA0BD517EE900AFEF789
:1016E00013FF514ACDE90001394630467BF000FF37
:1016F0000025D8ED807AB8EE087AF4EEC77AF1EEDC
:1017000010FA0BDD17EE900AFEF7FEFE474ACDE910
:101710000001394630467BF0EBFE0025B8F9E43194
:10172000042B07DC052200923946414A30467BF003
:10173000DFFE0025D8F8940A5DF0E0F880B198F952
:1017400046326BB1D8F8943AB8F94822B3F90E3062
:101750009A4205DA374A394630467BF0C9FE002501
:10176000DFF8F09039463046FFF71AFF99F8593CF8
:10177000002B48D100EA05042F484FF4806100F0A7
:10178000EDFE78B1D8F8943AB3F90C30A3F2E24206
:1017900092B2B2F5FA7F05D9284A394630467BF035
:1017A000A7FE0024264890F8F4325BB100F53B70A8
:1017B0002CF0F4FA054628B9224A394630467BF027
:1017C00097FE2C4600212E2204A80DF10C0803914F
:1017D000ACF0AEFED9F8440C4246322108F01CF9B8
:1017E000054600287FF425AFD9F8440C03689B68B0
:1017F0009847154ACDF800800346394630467BF0BD
:1018000077FE2C4615E7114A394630467BF070FECC
:101810000024B1E701240CE7942C0020BC290C081B
:10182000D3290C08F6290C08162A0C08382A0C08AB
:101830005A2A0C08792A0C08982C0020B42A0C0883
:10184000987C0020DC2A0C08D0D80C089F2A0C08B1
:10185000984C0020986C002070B505460E46FFF7A6
:101860009FFE3146044628467CF0E2FB2040C0B291
:1018700070BD0000F0B591B005460E467BF016FF36
:101880000446D8B1102128467BF010FCB0B10021ED
:101890002E2204A803AF0391ACF04AFE10F0C0F969
:1018A00032233A4601210FF0CBFC044630B9054BF8
:1018B00000973246102128467BF000FC204611B0EC
:1018C000F0BD00BFF02A0C0870B505460E46B1B950
:1018D00090F910408CB116480AF0FAFFDFED157A46
:1018E000B0EEC00AB4EEE70AF1EE10FA07D4124ADD
:1018F000012128467BF0FCFD3446204670BDAB68D4
:101900009BB10E4B1B68D86AFFF71CFE044630B132
:101910005BF0A6FA0A4A042154F0E4FBEDE73146F5
:101920002846BDE870407CF08DB90124E5E700BF92
:10193000982C002000000034FC2A0C08942C002075
:101940000E2B0C0838B504467CF086FD0546B0B178
:101950000C4805F033FB40B10B49A1F598400FF05E
:10196000ADFD10B1074800F0CDFD2046FFF7F4FDB6
:101970000123064984F8373020467CF07DFC284658
:1019800038BD00BF982C0020608A0020302B0C0846
:10199000F8B505460E461746C2B1232901D00129E4
:1019A00014D81E4807F0BEFB044668B10024204648
:1019B000F8BD95F91030022B08D05BF051FA184AA7
:1019C000062154F08FFBF2E7002EF2D03A46314662
:1019D00028467CF0F7FD04460028E7D0114ED6F8E3
:1019E000442C06F6D8339A4203D003F214702CF03C
:1019F0000BFED6F8440C03689B6B98470A4B83F8A0
:101A0000C0022846FFF7A8FD4FF0FF330749C6F88C
:101A1000743C28467CF030FCC9E700BF982C0020BD
:101A2000402B0C08986C0020987C0020582B0C0848
:101A3000F8B505460E467BF0E5FB104B93F91B729B
:101A40000446CFB90E48BD212CF074FD38B10D4BC2
:101A500032464FF4804128467BF030FB3C46084834
:101A6000BC212CF067FD38B1074B32464FF4804162
:101A700028467BF023FB00242046F8BD984C00202C
:101A8000847F00206C2B0C08982B0C0800207047DA
:101A9000014800F0E1BC00BF982C002003685B689F
:101AA000184700000DF040B864F07CBA5CF018BE36
:101AB00024F090BD50F054BB07F06ABC4EF012BC4D
:101AC0000AF006BA02F00ABE4CF0A8BF14F00CB936
:101AD00060F080BA5FF0FEBE0CF026B945F07EBF24
:101AE0000AF074BF13F05EBC66F010B85CF01ABB6D
:101AF0005AF03CBC06F07ABE04F0EEB909F072BDB3
:101B00000AF054B90BF044BF0CF0BCB90AF096BD12
:101B10000CF064B801F01EB900F5657016F01ABF3C
:101B200007F0A6B990F82031B02202FB030390F829
:101B3000482193F8693012B1012B28BF01231846C0
:101B400070470000034808602C21117008221A60B9
:101B5000704700BFDC2E0C0870B5044604F58E55A6
:101B600000F5BD4054300835FFF7F6FC002128464B
:101B70000FF0DCFF802120460CF0F2FB18B126F0BC
:101B8000ADFB24F041F904F50053D3ED7E7ADFED8F
:101B9000236A93ED807A67EEA67A04F58052FDEE13
:101BA000E77A02F21441D1ED006AF8EEE77A02F525
:101BB000826267EEA67A03F6A823FDEEE77A05F5C2
:101BC000457017EE901A43F8041CD2ED007AF0EE3F
:101BD000E77A67EE877A04F5A851C3ED007A29F019
:101BE000B7FB04F5A04694ED467AD6ED8F7AE7EE82
:101BF000007AC6ED8F7AB0EE670A27F0D7F84FF477
:101C0000001186ED8F0A20460CF0AAFB20B1284671
:101C1000BDE870400EF0B8BA70BD00BF0000C84209
:101C2000FFF79ABF10B500F580430446D3F8440C83
:101C300003689B6B984704F5A04393F87B3233B954
:101C400028B104F52D50BDE8104080F071BE10BDE4
:101C5000FFF7E8BF38B54FF4801104460CF080FB65
:101C6000054620B9012120460CF07AFB05460221E9
:101C700020460CF075FB48B115B9204602F0D6FCA1
:101C800004F58E5008300EF07DF901E0002DF7D1FB
:101C90004FF4805120460CF063FB30B104F5BC409A
:101CA0005030BDE8384060F0BBBA38BDFFF7D2BF56
:101CB00038B54FF4801104460CF052FB0121054663
:101CC00020460CF04DFB18B115B9204602F0AEFCD1
:101CD000102120460CF044FB60B1204602F016FDB6
:101CE0004FF4800120460CF03BFB18B926F0F6FAC1
:101CF00024F086F9202120460CF032FB28B1204642
:101D000002F07AFD204602F091FE4FF40051204689
:101D10000CF026FB10B1204602F072FE8021204616
:101D20000CF01EFB28B126F0D9FABDE8384024F0AB
:101D30008FB838BDFFF7BCBF00F5804300F5BA404F
:101D4000D3F8681C2C307EF035B80000FFF7F4BFE4
:101D500010B5044616F0CAFE90F915308BB190F814
:101D6000F43173B194F9AC335BB1064B1B68DB6A99
:101D700093F89C302BB904F56570BDE8104016F05F
:101D80009DBC10BD942C0020FFF7E2BF2DE9F84365
:101D9000424B1B68DB6A93F89C300446002B7AD0D8
:101DA00000F5805797F8D134002B74D007F0BAF9BA
:101DB000002870D004F5F65507F58059083599F8D4
:101DC000161028460DF082FC002864D004F59076A9
:101DD0003046FFF7A7FE02285DD994F840324FF055
:101DE000B00808FB034393ED697AF1EE007AB4EE94
:101DF000E77AF1EE10FA4ED499F8161028460DF055
:101E000015FF04F50053B3F9E42107EE902AB8EE6C
:101E1000E77AB4EEC07AF1EE10FA0CDD94F84022C5
:101E200008FB0242F8EE677A92ED697AF4EEC77A1F
:101E3000F1EE10FA2FDCD7F8C023D3F8A41A002A49
:101E4000B8BF52428A4226DCD7EDF17AD3ED7F6AE1
:101E50009FED136AF8EEE77A66EE866AF4EEE67AAC
:101E6000F1EE10FA17DC03F6A82292ED007A27EEC5
:101E7000067AF4EEC77AF1EE10FA0CD494F8401218
:101E8000B02202FB01612846B3F9E6219C31BDE88E
:101E9000F8430DF031BABDE8F88300BF942C002060
:101EA0000000C842FFF772BF2DE9F04190F84032C0
:101EB0002D4D00EB03132F68D3F87C8100F590764D
:101EC00004463046FFF72EFE474514D0022814D9A9
:101ED00004F58047C5F8008097F86C3C012B15D8B5
:101EE00017D104F5A045D5F8D03DE3B9D5F8D43DD8
:101EF000CBB905230BE0022810D804F5804393F8F2
:101F00006C2C5AB1052283F86C2C07E0013B87F852
:101F10006C3C04F5B050043010F0FCFF2046BDE8E6
:101F2000F04109F005BD114B1B68D86A03685B6876
:101F3000984780460028ECD194F84012B02303FB68
:101F400001617431204605F0A9F8D5F8B43D0FCBF6
:101F500005F6B85605F6D85586E80F0085E80F0057
:101F600087F86C8CD5E700BF882C0020942C0020CB
:101F7000FFF79ABF10B500F5A04300F5805493F821
:101F80007B221AB1002384F8D1340AE0D3F8C83296
:101F9000042B07D100F5B940203080F067FF84F8AA
:101FA000D10410BD0123EEE710B500F5804400F523
:101FB0009743D4F8441C5833994200F5A04308D005
:101FC00000F598421C3291421CBF4FF0FF32C3F81B
:101FD0003422074AC3F82422064AC3F82822FFF70E
:101FE000C9FFD4F8440C0368BDE810401B691847CA
:101FF0000000C8420000C8C2FFF7D6BFF7B500F521
:10200000A0460446D6F8C8328B420D463FD00B1F7F
:1020100000F5B947594207F1200759413846019167
:1020200080F014FE0199384680F010FE042D02D194
:1020300018486CF0F1FBD6F8C832012B18D1032DEB
:1020400016D104F5BD4054307BF01EF840B1204657
:1020500007F068F820B104F528503C306CF0D6FB4E
:102060002046C6F8C85203B0BDE8F04002F02EBCCE
:10207000072DF5D104F54950D6F8442264230521F3
:1020800092FBF3F31030044A54F02CF8E8E703B065
:10209000F0BD00BFD45600203C2C0C0838B500F52C
:1020A00080450446D5F8440C03689B6B984700288C
:1020B00040D004F5A04393F8C022DABBD5F8441C05
:1020C00004F597425832914236D193F874222AB9D6
:1020D00001212046BDE83840FFF790BFB3F82A231E
:1020E000152A27D193F8A41C11F0010120D1D3F8AF
:1020F000C822072A1CD093F91A3D0BB90421E8E73E
:1021000020460AF0E5FBDFED0F7AB4EEE70AF1EEC8
:1021100010FAF3DB04F5B940203080F0E7FD002829
:10212000ECD004F54950084A0621103053F0DAFF8C
:102130000721CEE70321CCE704F598431C339942ED
:10214000F8D138BD0000B442602C0C0838B5214CE1
:10215000D4F8442C04F6D8339A422DED028BB0EE1D
:10216000408A03D00020BDEC028B38BD04F58055B9
:10217000D5F8C832042B23D194F86D3C33B11649FD
:10218000A1F6DC202CF0B8FC0028ECD19FED137AEE
:10219000F0EEC87AF4EEC77AF1EE10FA07D49FEDAC
:1021A000100A28EE008ABDEEC88A85ED918A0D4896
:1021B00080F09CFD0028D5D0002385F87732D2E747
:1021C000B5F82A13A4F5804006F072F90028D3D19F
:1021D000C8E700BF986C0020608A0020000000342F
:1021E0000000C8423889002010B52DED028B00F5A3
:1021F000A0430446D3F8C822042A0BD104F032F9D4
:102200002046B0EE408A04F0FFF938EE400ABDECFB
:10221000028B10BD03F6046393ED000AF7E700009C
:102220002DE9F0412DED028B00F51C758AB00446B6
:10223000284612F06FF804F58E50002307A90830E5
:102240000793089309930FF0FDFA00287FD09DEDC6
:10225000090ADFED567A04F5A04595ED957A20EE52
:10226000270ADFED537AA7EE270A04F5A74064306A
:1022700004F5804685ED950A65F05CFE2046FFF783
:102280000DFFD6F8440C03689B6B984795F87B329A
:10229000002B57D1002855D095F8C032002B51D1D2
:1022A000D5F8C832042B69D09FED428A204604F04D
:1022B000CDF9C5F88C0FD6F8442C04F5974370334C
:1022C0009A4204F500581AD195F8483EBBB9B8F9BE
:1022D000743A002B04DC384AD2F8342AD2060ED5E0
:1022E000D5F8B41DD5F8BC2D49680A33521A6421BB
:1022F0004B438242ACBF9B181B18C5F88C3FD6F8E5
:10230000702CD5F88C1FD5F8C83205912046049260
:1023100003930CF087FAB6F97E6C07462046FFF768
:1023200063FFCDE90076F0EE400ADDE90332D8ED37
:10233000A01A95EDB91A0599B0EE480A04F52D508A
:102340007FF09AFF0AB0BDEC028BBDE8F08104F586
:102350009070FFF7E7FB02280AD994F84032B022C8
:1023600002FB034393F8D82112B193ED710A70E791
:10237000284611F069FEB1EE400A6AE704F5BB4752
:1023800004F5BB48483708F1580804F5BB414246FC
:102390003831384615F0A4FF002885D0414638462C
:1023A00016F032F8B0EE408A80E700BFCDCC4C3E4C
:1023B000CDCC4C3F00000000984C0020FFF730BF10
:1023C00000F5804200F59843D2F8442C14339A4229
:1023D0001FBF00F5A040D0F85C320B60012008BFA1
:1023E0000020704710B500F5804200F59843D2F800
:1023F000442C14339A420C4612D000F54050D0F8C9
:10240000780403681B69984707EE900A9FED057AE8
:10241000F8EEE77A012067EE877AC4ED007A10BD06
:102420000020FCE70AD7233C10B500F5804200F5F8
:102430009843D2F8442C14339A420C460AD000F543
:102440004050D0F8780403685B699847012084ED18
:10245000000A10BD0020FCE730B505460FC985B065
:102460006C4684E80F0040F279322146284604F099
:10247000ADFC0C4B03F54062D3F8443C93420ED1C3
:102480009DF8001011F0040102D1204615F024FD42
:102490000548214604F052FD012005B030BD002062
:1024A000FBE700BF986C0020982C002000F58040CE
:1024B000D0F8440C03689B6C1847000000F580407E
:1024C000D0F8440C0368DB6C1847000010B500F529
:1024D000805300F50050D3F8D0431460D3F8CC33C8
:1024E0000B60D0F8343A9B0509D4D0EDA06AD2ED48
:1024F000007A9FED037AE6EEC77AC2ED007A10BD4E
:1025000035FA8E3C38B50D4D04462946A5F5984060
:102510000FF0E6F804F5804305F13C0183F86D0CFB
:1025200004F58E5008300EF075FF04F5BC40D0ED78
:10253000017AF1EE677AC0ED017A38BD608A002039
:1025400010B5044600F590701EF04AFA2046BDE82A
:102550001040FFF7D7BF0000FFF7F2BF00F50050B3
:10256000D0F8343A194214BF01200020704700000F
:1025700038B5054B1C6823680A461D68034B0146A5
:102580002046A847002038BD942C0020982C00201D
:1025900070B52DED028B0446036804F500559B6D64
:1025A0009847D5F8343A1B0618D5B5F9E431B5F992
:1025B000E611CA1A0B4402EBD27203EBD37352102A
:1025C0005B1000EE902A00EE103A04F58E50F8EE03
:1025D000E00AB8EEC00A08300EF0DAFC5A4BB5F843
:1025E00016221A7004F5BD455EF094FA54355DF07C
:1025F000E3FE00212846FFF701F8544E0123B07195
:102600002846F3717AF036FD28B928467BF048FE5B
:10261000B0FA80F040093071042120460BF0A0FE92
:1026200020B104F5A84004304DF00EFF28467AF0A2
:1026300021FDE8B994F8403204F5A04504EB0313FA
:1026400041F28832D3F87C61D5F84C3EF31A9342BC
:102650000ED904F59070FFF765FA022808D9C5F87D
:102660004C6E204605F54A6504F0A8FC00232B605B
:10267000B4F9A4301BB9B4F8A230A4F8A430B4F86B
:10268000A430DFED338A07EE903AF8EEE77AB7EE42
:10269000008A88EE270AD4ED2B7AF0EEE77AF4EE82
:1026A000E87AF1EE10FA09D5B4F9A23007EE903AC3
:1026B000F8EEE77A88EE277A84ED2B7AD4ED2B0AB0
:1026C00026F076FA20BB4EF0CBFD40F27D124FF49F
:1026D00080114EF07DFD4CF057FA4BF0BFFE04F533
:1026E00037503C30B0EE408A73F016FE04F53D5092
:1026F000B0EE480A183073F00FFEB0EE480ABDEC99
:10270000028B04F542500C30BDE8704073F004BEFB
:10271000D4ED2B7A94ED460AF0EEE77AF4EEE87AFF
:10272000F1EE10FA09D5B4F9A23007EE903AF8EEBE
:10273000E77A88EE277A84ED2B7AD4ED2B0A26F0FF
:1027400037FA0028BFD0C6E7A0230020D58C002090
:1027500000000034FFF71CBF70B500F5A04604462A
:1027600096F9183D002B28DD06F0DCFC28BB04F5AB
:10277000BD45543528467BF093FDF0B128467AF0EC
:1027800079FCD0B182F0CEFBD6F86432C01A96F94B
:10279000183D4FF47A72534398420ED301221C2104
:1027A0002846FFF7F5F840B104F54950034ABDE863
:1027B00070400621103053F095BC70BD802C0C0881
:1027C00030B52DED028B044683B000F58E5001A983
:1027D00008300FF009F8002871D004F5A04595EDF8
:1027E000937ADDED017AB4EEE77AF1EE10FA08D5CE
:1027F00004F5BD4054307AF047FC10B1019BC5F898
:102800004C3204F50054D4ED8E6AB4F9E431052B52
:10281000B8BF052307EE903AB4F9E63107EE103A57
:10282000B8EEC77AF8EEE77A37EE077A1820C6EEE8
:10283000870AB6EE007AF4EE470AF1EE10FAC8BF46
:10284000F0EE470A9FED2D7A67EE877A9FED2C7A9E
:1028500086EEA71AF0EE007AB4EE671AF1EE10FADF
:1028600048BFB0EE671ADDED017AF4EEC77AF1EEFB
:1028700010FACCBF86EEA70AB0EE410A26F0AAFAFB
:10288000B0EE408A1F480DF0BBFF90B91E484021B2
:10289000FFF764FE68B11D4BD3F8C832012B08D195
:1028A000F7EE007AB4EEE78AF1EE10FA58BFB0EE18
:1028B000678AB0EE480A03B0BDEC028B30BD04F568
:1028C000BD4054307AF0E0FBB7EE008A0028D9D042
:1028D00046205DF0C1FBB4EEC80ADFED0D7AF1EEE3
:1028E00010FAD8BFB0EE480A87EE800AA9F074FD4E
:1028F0002F209FED081ADFED080ABFE73333333F7F
:1029000017B7D138603E0020982C0020987C00201A
:10291000000034428FC2D53F9A99193FF8B504465A
:102920005BF090FF0368DB689847054610B9002507
:102930002846F8BD204606F089FA04F58046074689
:10294000D6F8440C03689B6B984780B10E4BD3F8C4
:10295000440C03685B6B984748B104F5005494F944
:102960008D32002BE3D0032BE1D03D46E0E796F813
:10297000583C002BDCD004F5005494F95052023D31
:1029800018BF0125D4E700BF986C002073B500F58F
:10299000804202F68C4393ED000AD2F8442C00F5F5
:1029A000964374339A422BD100F50053D3F88C3AF6
:1029B000B3F90840003C18BF012400F5A04300F51E
:1029C000375500F58050D3F8DC62D0F8C02393F877
:1029D000D8320435B61A5BB10A488DED010A4FF4BE
:1029E0000061FFF7BBFD9DED010A80F00100C3B25D
:1029F00022463146284602B0BDE870407CF0FEBA5F
:102A00000024DAE7982C002010B5044605F046FEB5
:102A100098B104F5A042D2F8DC3203F58C41503174
:102A2000C2F8DC1204F58051D1F8C0130029BEBFF2
:102A3000A3F58C43503BC2F8DC322046FFF7A6FFDB
:102A4000BDE8104004205DF0F3BA00002DE9F0412C
:102A50002DED048B00F5005696EDA08ADFED378A48
:102A600028EE288A00F58048BDEEC88A00F5A04708
:102A700008F68C4393ED009AD7F8E03218EE102A4E
:102A80001A4408EE102A054646205DF0E5FAB8EE35
:102A9000C88AD6ED8A7AD8F8440CA0EE278A05F5C4
:102AA000964374339842FDEEC87A17EE904A42D1AD
:102AB000D6F8903AB3F90860003E18BF01260368C3
:102AC0005B699847C0B9D8F8440C03689B6B98477A
:102AD00090B9D7F8843F022B0ED1284609F04CFD5F
:102AE00050B107F6F843D3ED007A67EEA87AFDEE11
:102AF000E77A17EE903A1CB205F53C5805F580557B
:102B000008F11C08D5F8C433E41A97F8D8323BB161
:102B10000B484FF40061FFF721FD80F00100C3B2C4
:102B2000B0EE490ABDEC048B324621464046BDE872
:102B3000F0417BF09FBF0026C1E700BF0000C84204
:102B4000982C002010B504460BF0AAFF68B100B223
:102B500000EB4000C0EB001300EE103AB8EEC00AE4
:102B6000BDE8104013205DF063BA2046FFF76EFF0A
:102B7000F6E7000010B50E48FFF7D0FEB0B10D4CDF
:102B800004205DF069FAD4F88C0A5CF0CBF80420DC
:102B90005DF04EFA13205DF05FFAD4F8900A5CF015
:102BA000C1F8BDE8104013205DF042BA10BD00BF6F
:102BB000982C0020984C0020F8B52DED028B04468F
:102BC000FFF7ACFE002800F0818004F5804704F593
:102BD0009742D7F8443C0432934277D004F59742A9
:102BE0002C32934272D004F59742503293426DD00A
:102BF00004F597423432934268D004F597423C3250
:102C0000934263D004F596427C3293425ED004F541
:102C10000055F6EE008AD5F88C0A5BF043FFB4EE5F
:102C2000E80AF1EE10FA3EDDB0EE087AFFEE007A27
:102C3000E0EE077AB0EE670AD5F8A42A07EE902AEC
:102C400004F5A046B8EEE77AD6EDB77AF8EEE77A63
:102C50005142E7EE007AFDEEE77A17EE900AC6EDF4
:102C6000B77A26F057F9C6F8DC02D7F8442C04F5F9
:102C7000974378339A4222D0D5F8900A5BF012FF3E
:102C8000B4EEE80AF1EE10FAB0EE408A21DCFEEE76
:102C9000007AB4EEE70AF1EE10FA22D5B0EE087A27
:102CA000F7EE007A19E0FEEE007AB4EEE70AF1EEF4
:102CB00010FAC1D5B0EE087AF7EE007AB8E72348EB
:102CC0004FF48051FFF74AFC0028D5D0BDEC028BB1
:102CD000F8BDB0EE087AFFEE007AE8EE077AB0EEC3
:102CE000678A204605F0DAFC08B1B1EE488AD5EDD6
:102CF0007F6AD6EDB87A9FED166A05F6A82595EDA0
:102D0000007AB5EEC08AF1EE10FACCBF28EE268A22
:102D100027EE488AF8EEE77A66EE866AE8EE067AEB
:102D200027EE067AFDEEE77AFDEEE66ABDEEC77A9B
:102D300016EE902A17EE101A17EE900AC6EDB87A22
:102D400026F0E8F8C6F8E002C0E700BF982C0020A3
:102D50000000C84270B5044604F5804582F0E2F8F0
:102D6000D5F8543CC31AB3F5FA6F064603D9D5F823
:102D7000440C06F06BFE2E4BC5F8546CD3F8440C93
:102D80000268136898470021204609F0A1FDDFED95
:102D9000297AB0EEC00AB4EEE70AF1EE10FA45D592
:102DA00004F5BC43D3ED017AB1EE047AF0EEE77A94
:102DB000F4EEC77AF1EE10FA38D504F51C7011F074
:102DC00043F9F6EE007AB0EEC00AB4EEE70AF1EE8F
:102DD00010FA2BD504F5AE5595ED037AF0EE087A8E
:102DE000B4EEE77AF1EE10FA05F10C051ED504F504
:102DF000375004307CF072F904F53C501C307BF005
:102E0000E9FE04F5415034307CF016FE95ED007A71
:102E1000F7EE007AB4EEE77AF1EE10FA06D504F593
:102E200047502830BDE870407CF05CBB70BD00BFEF
:102E3000986C00200000003400F5005393F9DB315A
:102E4000012BC3BF00F52D5090ED290ADFED047A68
:102E50009FED040AC8BF20EE270A46205DF0E8B8BF
:102E60000000C842000000002DE9F8432DED028B60
:102E700000F5804909F68C43D3ED008A054609F038
:102E800099F90746D9F8440C03681B6A984705F579
:102E90004156343698B14B4CD4F8A032002B0EDD9D
:102EA00082F040F8D4F8A032C01A40F6B733984206
:102EB00005D8B4F9944230467CF0CAFD74E005F5BB
:102EC000A04805F5005498F8793F43B1B4F96C3245
:102ED000002B04DD05F5405393F98A3003BBD9F884
:102EE000443C05F596457435AB4267D00021B0EE01
:102EF000680A30467CF044FB054604205DF0ACF8DF
:102F00002BB207EE903A94ED887AF8EEE77AE0EE8D
:102F1000077AFDEEE77A17EE904A3C4424B2CAE7FE
:102F20000121284609F01EFB9FED277AB4F96C3287
:102F3000C0EE077A08EE103AB8EEC88A9FED230A71
:102F400028EE278AD8EDB77AF8EEE77A67EE807A2E
:102F50009FED1F0A27EE800AA9F062F8B4F9E43168
:102F6000DFED1C7A98EDBA7A20EE270A07EE903A48
:102F7000F8EEE77A0021B4EEE77AF1EE10FA58BFE6
:102F8000F0EE477A80EE277A3046DFED137AB0EE26
:102F9000480AA7EE270AF0EE680A7CF04DFCBDEE69
:102FA000C00A10EE103A1CB2BDEC028B20460B4951
:102FB000BDE8F84341F2941225F0BCBF391E18BF9A
:102FC000012194E7987C002000A08C450AD7233C7F
:102FD00035FA8E3C0AE81C41E02E65426CEEFFFF9C
:102FE00038B500F540530546D3F878040368DB682C
:102FF0009847014605F5475028307CF055FA04B251
:103000002846FFF78BFC70B107EE904A05F5005596
:10301000B8EEE70AD5F8980A5BF084FEBDEEC00A68
:1030200010EE103A1CB220460349BDE8384041F288
:10303000941225F07FBF00BF6CEEFFFF38B590F80B
:103040004032B02202FB030393ED697AF7EE007A77
:10305000B4EEE77AF1EE10FA044600F5A0451CD56F
:10306000002109F035FCDFED407AB0EEC00AB4EE85
:10307000E70AF1EE10FA10D5D5F8C832012B0CD0C2
:10308000072B0AD0002385F838320023C5F83C32DC
:103090002046BDE8384009F08DB881F043FFD5F8EF
:1030A0004032C5F84002C31AB3F57A7F84BF0023CB
:1030B00085F83832204609F07DF8D5F8C832012B62
:1030C00007EE100A2DD0072B2BD0B8EEC77ADFED14
:1030D000276AC7EE267A04F50052B2F9302200EED4
:1030E000102AB8EEC00A27EE800ADFED1F7AB0EE94
:1030F000C07AB4EEE77AF1EE10FA14D4002385F822
:10310000383295F8383204F547502830D3B97CF07E
:10311000B3F8BDE83840164900B241F2941225F0E8
:1031200009BF9FED140A95F83822002AE9D101223F
:10313000934285F83822E4D0072B1CBF0023C5F842
:103140003C32DEE795ED8F7ADFED0B7A67EEC77ADA
:103150009FED0A7A67EE877AFDEEE77A17EE901A0E
:103160007CF0A2F9D5E700BF0000003400A08C4538
:103170006CEEFFFF00000000E02E65420000C84238
:1031800070B52DED028B00F5B946203682B00546AC
:1031900030467FF0DBFC0446D8B905F50052D2F882
:1031A0008C3AB3F9083073B905F5BC43D3ED017A15
:1031B00092ED8B7AF0EEE77AF4EEC77AF1EE10FA40
:1031C0004CBF0124002430467FF0D4FC002808BF07
:1031D000002430467FF0BAFC28BB05F5A043D3F8A5
:1031E0003432013319D0F4B99FED1A8A2846FFF71B
:1031F0003BFE07EE900AB8EEE70A8DED010AD4B95E
:1032000015205CF015FF9DED010A1A2002B0BDECFF
:10321000028BBDE870405CF00BBF002CE4D0284668
:10322000FFF70CFF02E02846FFF7DAFE07EE900AF0
:10323000B8EEE78ADAE71A205DF09CF99DED010A05
:1032400008B9B0EE480A15205CF0F2FEB0EE480A6C
:10325000DBE700BF0000000010B500F50053D3ED20
:103260007F6ADFED137A9FED136A03F6A82393EDCF
:10327000007A00F52D5366EEA76A27EE277AD3ED84
:103280002A7A67EE867AFDEEE66ABDEEC77AFDEE33
:10329000E77A044616EE902A17EE101A17EE900AF7
:1032A00025F038FE04F5A044C4F8E00210BD00BFCC
:1032B0000000C842A00CB34510B504460BF054F80A
:1032C000031E26DB04F5005191F9DB219A4220DD33
:1032D00004F5A040D0F8C842022C1AD0D1ED8D7A66
:1032E000DFED0C6AD31A66EEE76A07EE102A07EEE6
:1032F000903AB8EEC77AF8EEE77A87EE876AD0EDB3
:10330000B87AF8EEE77AE6EE867AFDEEE77AC0ED77
:10331000B87A10BD0000C84270B52DED028B00F5E3
:10332000A045D5EDB77A9FED400A9FED407AF8EEC3
:10333000E77A044667EE807A9FED3D0AF0EEE76A91
:10334000F4EE476AF1EE10FAC8BFF0EE477A27EEC6
:10335000800AA8F0A5FC25F05FFCB7EE008AC8EE55
:10336000007A04F50056C5EDB97A96F90C3243B3EC
:10337000204605F093F920BBB6F9E431D5EDBA6AE1
:10338000012BB8BF012307EE903AF8EEE77A86EEFC
:10339000A77AB4EEC87AF1EE10FA15D840F6C41246
:1033A0002449D5F8DC0225F0B5FDC5F8DC02D6F8D5
:1033B000A42A40F6C4139A42D4BFC6F8A42AC6F879
:1033C000A43ABDEC028B70BDD5EDB97AB4EEE77AC4
:1033D000F1EE10FAF5D588EE070A20EE000AA8F003
:1033E00049FEDFED157AD5F8DC0220EE270ADFED85
:1033F000137A20EE270A40F6C413FDEEC07A17EECA
:10340000904A9C42B8BF1C462246614225F082FD8C
:10341000C5F8DC02D6F8A43AA342D4BFC6F8A43A51
:10342000C6F8A44ACDE700BF0AD7233C0000AA4251
:1034300035FA8E3C3CF6FFFFE02E65420000C842A4
:1034400010B500F540530446D3F8780403681B68B0
:10345000984704F50053D3F8A42A514225F05AFDA9
:1034600004F5A043C3F8DC022046BDE81040FFF796
:1034700053BF0000704700000120704708207047CC
:103480000120704770470000014B93F81802704705
:10349000984C0020034B93F9280A003818BF0120EC
:1034A000704700BF984C0020014B93F91A027047F7
:1034B000984C002013B5064BD3F8440C4B690468B4
:1034C000009308310EC9646CA04702B010BD00BF64
:1034D000986C002070470000002070477047000083
:1034E00038B5254DD5F8440C03685B6898470F281C
:1034F00034D80F2839D8DFE800F008360808080863
:103500000808083836363636363610241B4B93F802
:10351000492212B193F848320BB944F01004184B09
:10352000D5F8442C9A42A3F1080303D09A4218BF5D
:1035300044F01004134991F98D12C1B19A4218D088
:10354000032902D1104B9A4201D144F040040F48A4
:1035500079F090FD68B144F080040AE0182814BFA7
:1035600001241824D2E71824D0E70124CEE79A4298
:10357000EDD144F0010038BD986C0020985C00202B
:10358000AC780020984C0020707800206C8B0020D4
:1035900008B5044805F0C6FD00280CBF0120022034
:1035A00008BD00BF982C0020F0B52DED028B8BB02C
:1035B00005460EF035FB4FF48071D0F8047290EDA3
:1035C000828AD0F80C6204461448FEF7C7FF30B96F
:1035D000134BDFED147A93EDA07AA7EE678A2D7C6A
:1035E00081F0A0FCD4F81823D4F81C33D4F81413B9
:1035F0000892099327221C23CDE9003203900791FA
:1036000003AA1E21284604978DED058A069653F0DD
:103610009DFD0BB0BDEC028BF0BD00BF982C0020CF
:10362000984C002035FA8E3C2DE9F0432DED068BA9
:103630003F4ED6F8442C06F614439A428BB071D014
:10364000A6F5805306F58059D3F87874D9EDB77A8A
:103650003B6890F810809B689FED369AB8EEE7AA19
:10366000D9EDB87A3846F8EEE79A984707EE900A0F
:10367000F8EEE77A384667EE897A2AEE09AAFDEE77
:10368000E77A69EE899A17EE903A1DB23B681B699A
:10369000984707EE900AF8EEE77AD9ED978A67EE39
:1036A000897AA6F58040FDEEE77A06F6784617EEB1
:1036B000903ADFED217AF4EEE78AF1EE10FA58BF86
:1036C000F0EE678A1CB202F023FE3B68D6ED00AA3A
:1036D000DFED1A7A5B6908EE100A38466AEEA7AA8F
:1036E0009847FCEEE88AB8EEC88A18EE903AB722FE
:1036F00028EE098AADF824301A23CDE900323E21A4
:1037000003AA40468DED03AACDED049A8DED058AFE
:10371000CDED06AA8DED070AADF82050ADF8224098
:1037200053F014FD0BB0BDEC068BBDE8F08300BF79
:10373000986C00200AD7233C00FF7F470000C84256
:1037400008B502480AF010FE00B208BD982C00200F
:1037500054F0BEBF37B50D46134840F2EF2203F0D8
:1037600035FB2C7814F004040AD0696803220F4852
:1037700014F0EEFA0C4803B0BDE8304002F0DABCB9
:1037800001AA2146284614F0B7FB0028F2D0DDED4F
:10379000017A9FED077A67EE877A2246FDEEE77A97
:1037A00017EE901AE3E700BF982C0020708A0020E3
:1037B0000000C84210B5054C012384F84B3255F087
:1037C000C7F9002384F84B3210BD00BF985C00207D
:1037D00058F06CBC2DE9F0412DED028B4FF0000844
:1037E00082B0CDE900281E4F9FED1E8A0C4615467B
:1037F000B0EE480AB1F90220D7F88C1A4FF47A7368
:10380000064658F03BFF0123CDE90053B4F90020F0
:10381000D7F8901AB0EE480A30464FF47A7358F051
:103820002DFFB4F90420D7F8941A9FED0F0A4346F0
:103830003046CDE9005858F021FFCDE90058B4F9E1
:103840000620D7F8981AB0EE480A4FF47A7330463B
:1038500058F014FF02B0BDEC028BBDE8F08100BF50
:10386000984C00200000FA4400007A4438B5C5782E
:103870000B46352D044628BF352535220021184634
:10388000AAF056FE2A4604F10C01BDE83840AAF021
:1038900005BE000010B5074B93F9042440F24D34E7
:1038A00040F24D13002A08BF1C4654F099FF2043F4
:1038B00010BD00BF987C002010B5044614F04CFEEB
:1038C000204610BD10B50C4C002384F8773255F01B
:1038D00039FEA4F58052A4F58563D2F8442C9A42AF
:1038E00008D194F8F0322BB904F53B70BDE81040D4
:1038F0002BF05CB810BD00BF987C002013B5114CB4
:10390000A17DA4F59C700BF0E1FE68B1A17DA4F54A
:103910009C700CF049F938B1A17DA4F59C7002B0FF
:10392000BDE810400CF082B90EF07AF901A90DF053
:103930005BFF18B19DED010A02B010BD9FED020AB8
:10394000FAE700BF984C00200000000008B51248BC
:10395000D0F8442C00F60C439A4216D0B0F95C3CE7
:10396000ABB900F5805393F8012282B990F8592C35
:103970006AB993F8B13263B9A0F5804005F0D2FB83
:1039800000280CBF0320042008BD0220FCE705200E
:10399000FAE70620F8E700BF986C002010B5224B2C
:1039A00003F61442D3F8443C934290B0044638D016
:1039B00000231E48029314F0B5F9014618B91B48BC
:1039C00002AA14F0FBF9247C81F0ACFA184BDDED6F
:1039D000027AD3F8E02DD3F8E43D05930023F8EE06
:1039E000E77A9FED147A0793089309930A930B9350
:1039F0000C930D930E934FF6F853ADF83C30002323
:103A0000CDE9030267EE877A96228DF83E303323A4
:103A1000CDE90032572103AA2046CDED067A53F0B6
:103A200095FB10B010BD00BF986C0020708A00207C
:103A3000987C00200AD7233C10B555F0CBF80446FB
:103A400088B90A48A0F58052A0F58563D2F8442CC5
:103A500080F877429A4206D190F8F0321BB900F50F
:103A60003B702AF0A3FF204610BD00BF987C0020C9
:103A70000120704708B5034BD3F8440C03685B681A
:103A8000984708BD986C002030B587B005460EF009
:103A9000C7F804462D7C81F039FAD4F88422D4F892
:103AA00088320492059300211023CD22CDE9003203
:103AB0000290039102AA42F60C31284653F046FBCD
:103AC00007B030BD30B52DED028B89B005460EF044
:103AD000A7F800F55A7393E8070002AC84E80700E2
:103AE000DDED020A9DED030A2D7CF1EE600AB1EED8
:103AF000400AA8F027FB2046B0EE408A28F00EF8D6
:103B0000DFED0B7A049B079328EE278A0C23012212
:103B1000CDE90032A82105AA28468DED058A8DED54
:103B2000060A53F013FB09B0BDEC028B30BD00BF99
:103B3000E02E6542282938B5054623D007D8242928
:103B40002BD0272911D01B2908D1012413E04329A8
:103B500037D008D84029F8D0422928D02846BDE8D7
:103B6000384058F0E7BE5329EEE7122152F0ECFC42
:103B7000044610B90024204638BD297C13484BF078
:103B8000A3FBF8E7162152F0DFFC04460028F1D031
:103B9000297C0E484BF072FCEDE70C2152F0D4FC6E
:103BA00004460028E6D02846FFF78CFFE3E7102103
:103BB00052F0CAFC04460028DCD02846FFF764FF18
:103BC000D9E7017C02487EF0BFFFBEE79C80002061
:103BD00038890020F0B52DED028B05468DB01646D4
:103BE000B0EE408A0C46002930D0007C53F044FAF5
:103BF0000746287C54F044F900F121039F4207D284
:103C0000287C0DB0BDEC028BBDE8F04052F08ABCC0
:103C100063690893636A2269CDF82530236AA06935
:103C2000E1680792CDF829306222212327680590A8
:103C3000CDE900320691287C0397192303AAC221FB
:103C40008DED048A8DF8246053F080FA0DB0BDEC40
:103C5000028BF0BD70B52D4CD4F8442C04F61443FF
:103C60009A42054651D0A4F50054B4F8BE32DE079E
:103C700008D504F56F6393ED000A012204F6EC61A8
:103C8000FFF7A8FFB4F8BE32980707D520490222F3
:103C900091ED130A28464831FFF79CFFB4F8BE3275
:103CA000590708D51A49032291ED700A284601F5F3
:103CB000DE71FFF78FFFB4F8BE321A0708D514493A
:103CC000052291ED870A284601F50671FFF782FF6C
:103CD000B4F8BE32DB0618D50E4ED6F8C832042B27
:103CE00013D10DF09DFF044606F54A607EF05CFF9F
:103CF00094EDC70ADFED087A014620EE270A284630
:103D00000622BDE87040FFF765BF70BD986C0020CB
:103D1000985C0020987C0020E02E654270B5044637
:103D20000E461CF083FE90F82011B02303FB010126
:103D30007431204603F0B2F9054698B13EB10DF05A
:103D40006FFF90F87C3243F0020380F87C3204F578
:103D5000804304F59744D3F8440C7034A04201D159
:103D600005F0C4FD284670BD73B5164601910446A2
:103D70000DF056FF01990DF0A1FB054698B13EB13B
:103D80000DF04EFF90F87C3243F0020380F87C3255
:103D900004F58043D3F8440C04F5974370339842FC
:103DA00001D105F0A3FD284602B070BD30B505462F
:103DB00085B00C46D1E9040125F098FA40B1684677
:103DC00013F0C0FF6A462146284658F0C7FB08B9E1
:103DD000022068E0354840F24F32694602F0F6FFB3
:103DE000D4ED037AF4EE677AF1EE10FA22D69FED65
:103DF000307AF0EEE77AF4EEC77AF1EE10FA54BFBB
:103E0000012200229DF800302A4962F341036846EE
:103E10008DF8003014F000F90028D9D12648694601
:103E200068F09AFD40B94FF02DF8052216214EF0AA
:103E3000E1FDCDE70022E5E7D4ED017AFDEEE77A7A
:103E400017EE903ADB0706D41C4B03F54062D3F81B
:103E5000443C934226D11A490222A1F598400AF027
:103E600093F89DF8001011F0040102D1684614F097
:103E700033F80E48694603F061F894ED020AB4EE97
:103E8000400AF1EE10FA0BD6B5EEC00AF1EE10FAC8
:103E900006DD9DF800100A48C1F3400106F074FDEC
:103EA000002000E0042005B030BD00BF982C0020A9
:103EB00000000034608A0020184D0020986C00201B
:103EC0009878002010B52DED028BD1ED017A91ED9F
:103ED000008AFCEEE77A8AB0CDED037A9DF80C10EB
:103EE00005AA044658F024FBC8B1DFED0E7A059B05
:103EF000009368EE277A0022FDEEE77A114617EE6E
:103F0000903A06A813F03EFF23682046D3F8CC3041
:103F100006A9984700200AB0BDEC028B10BD022014
:103F2000F9E700BF0000C84237B5124DD5F8440C80
:103F300003681B6A0C46984740B9D5F8442C05F62F
:103F4000D8339A4202D0042003B030BDD4ED007AB9
:103F5000D4ED020A94ED010A0748FCEEE77ACDEDB4
:103F6000017A9DF8041003F03BFE0028EBD00020FE
:103F7000EAE700BF986C0020982C002008B5D1ED2E
:103F8000007A9FED087A0848F0EEE77AF4EEC77AF7
:103F9000F1EE10FA54BF0121002104F079FB00205A
:103FA00008BD00BF00000034982C002010B5D1EDF2
:103FB000007AFCEEE77A17EE903A9CB2012C02D020
:103FC000022C06D084B91148214663F021FF00205D
:103FD00010BD0F4890F8F8335B0707D558F040FF45
:103FE0000C4A052152F07EF80420F1E790F9E43301
:103FF0001BB958F035FF084AF3E7A0F5A04007F0D9
:1040000099FF002814BF00200420E1E77C800020F5
:10401000987C002054320C086F320C0838B58B8B1A
:10402000C02B05460C4631D8B12B0BD8112B00F014
:104030009680142B00F0968021462846BDE8384033
:1040400059F052BDB23B0E2BF6D801A151F823F026
:10405000BF400108394001083940010839400108D2
:104060003940010839400108394001083940010848
:10407000B540010839400108D9400108154101083F
:1040800039400108C9400108AB400108D42B08D0D1
:10409000B3F5967F49D0D02BCED1BDE83840FFF79D
:1040A00085BFBDE83840FFF769BF2146BDE838400D
:1040B000FFF77CBE2146BDE83840FFF703BF21462D
:1040C000BDE83840FFF730BF94ED000A2848FEF7FE
:1040D0003DF8E8B100201CE0264C94F86D3CBBB1E3
:1040E0002549A1F6DC202AF05FFD88B104F5805354
:1040F000012283F8252304F6D8310222A4F580405A
:1041000009F042FF0028E5D11C4B002283F825234B
:10411000042038BD174C94F86D3C002BF8D016499C
:10412000A1F6DC202AF0C4FCDFE7D1ED007A9FED98
:10413000147AF0EEE77AF4EEC77AF1EE10FA14D5BD
:10414000D1ED017AF0EEE77AF4EEC77AF1EE10FAEB
:104150000BD50C490222064809F016FFBAE70A49B6
:104160000222F8E709490222F5E70220D1E700BF61
:10417000982C0020986C0020608A0020987C0020F9
:1041800000000034707800209078002088780020AB
:1041900070B53F4B03F54062D3F8443C93428EB078
:1041A0000C4673D1CD78272D28BF27252722002143
:1041B00004A8AAF0BDF92A4604F10C0104A8AAF04B
:1041C0006DF9059B9DF836400093069B0193E443EF
:1041D000079B0293E4B2089B03938DF8364080F06E
:1041E000A1FE14F0810F04F08705064601D1802D51
:1041F00011D1684626F010FCDFED267A264B20EE22
:10420000270ADFED267AC3F8986220EE270ABDEE72
:10421000C00A83EDA30A14F0820F01D1802D11D1C1
:10422000684626F013FCDFED1B7A1B4B20EE270AB5
:10423000DFED1A7AC3F89C6220EE270ABDEEC00AB1
:1042400083EDA40A14F0840F01D1802D11D16846AA
:1042500026F00CFCDFED0F7A0F4B20EE270ADFED86
:104260000F7AC3F8A06220EE270ABDEEC00A83EDE4
:10427000A50A63060AD5DDED0C7A9FED087A064B98
:1042800067EE877AC3F8A862C3EDA97A0EB070BD55
:10429000986C0020E02E6542987C00200000C84207
:1042A00030B5214C91B0084602A9FFF7DFFAD4F8E7
:1042B000442C04F540639A4233D19DF83C30072BDF
:1042C0002FD104F58054DDED056AD4F8DC3D9FED77
:1042D000177A07EE903AF8EEE77AE6EEC77AFDEE47
:1042E000E77A17EE903AC4F8DC3D58F0B9FDD4F8FF
:1042F000B42DD4F8DC3D52689FED0D7A9B1A07EE81
:10430000903AF8EEE77A054667EE877A17EE900A5C
:10431000FCF7FAF8074ACDE900010621284651F0DA
:10432000E1FE11B030BD00BF986C00200000C84213
:104330000AD7233C88320C0810B51D4B03F54062A8
:10434000D3F8443C9342044696B008460FD108A9DE
:10435000FFF78CFA9DF8541003AA204658F0E8F8AD
:1043600038B958F07DFD134A042151F0BBFE16B058
:1043700010BDBDF8503023F004039BB2002BF6D0E3
:10438000DDED0B7A9FED0C7A039B009367EE877A45
:104390000022FDEEE77A114617EE903A04A813F0DA
:1043A000F1FC236804A9D3F8CC3020469847DEE717
:1043B000986C00209C320C080000C84230B48D7A02
:1043C0004B7A43EA0523CD7A43EA0543562B04464C
:1043D0000A461BD008D8522B12D0542B13D020469B
:1043E000114630BC58F05CBD03F18073863B23F06E
:1043F0007F43012BF3D8017C064830BC4BF006B953
:1044000030BCFFF7C5BE30BCFFF74ABF30BCFFF77A
:1044100093BF00BF9C80002000207047C8207047D9
:1044200001207047002070470020704790F89C30B2
:104430008B4286BF283150F82100002070470000D1
:1044400090F89C308B4286BF283150F82100002024
:104450007047000003207047014B93F81602704725
:10446000984C002070B504464C4808F02BFA18B15F
:10447000E36A43F40003E362484808F023FA88B192
:1044800046205BF0E9FDDFED467AB4EEE70AF1EE97
:1044900010FA07D8236B43F400032363636B43F4E0
:1044A00000036363E36A43F4F843E3623D4BD3F8EC
:1044B000440C03685B6898470138172814D8DFE874
:1044C00000F03A420C4442424242133A3A3A3A3AF3
:1044D0003A13131313131313133A334A92F848324F
:1044E0008BB392F849228AB3304B93F89C3C012B52
:1044F0003DD0022B44D02E4B1D68DDB12D4E2846F9
:1045000096F8821A46F03AFFA0B1E36A43F480734A
:10451000E36296F9BC321BB1236B43F480732363CF
:1045200096F8821A284646F061FF18B1636B43F48F
:104530008073636370BDD4E90C2342F4E04243F41A
:10454000E04322636363012300E00023216B41F415
:1045500080622263626B42F480606063002BC3D090
:1045600041F4406142F4406221636263BCE7E36A64
:1045700043F48003E362236B43F480032363BAE7CD
:10458000E36A43F48003E362236B43F48003236311
:10459000636B43F480036363ADE700BF982C002096
:1045A000000000B4986C0020985C0020987C0020EB
:1045B000888D0020984C002013B54FF44470CDE94D
:1045C000002113F0C1FF044628B1DDE9002158F0B5
:1045D00087FE024B2360204602B010BD9C340C08BD
:1045E000002070470020704700207047002070476F
:1045F00000F509503830704700487047245A0C08BD
:1046000000F58040D0F8440C03685B681847000050
:1046100000F5804300F59740D3F8443C58301B1A0E
:1046200058425841704700009B20704730B500F554
:10463000A043D3EDB77ADFED286AB8EEE77AD3ED81
:10464000B87AF8EEE77A85B0044627EE267A67EE68
:10465000A67A00F58E50002301A9083003938DED52
:10466000017ACDED027A04F6A8650BF0B3FC04F5EF
:104670003B522C32692128464DF0D0FA04F54152C4
:1046800008326A2128464DF0C9FA04F5405393F9DF
:104690008A2032B9D3ED207AF5EEC07AF1EE10FA25
:1046A00006DD04F546523C326B2128464DF0B6FA41
:1046B00004F54754283420467AF018FF28B104F155
:1046C00030026D2128464DF0A9FA0DF0A9FA0CF040
:1046D000F1FF05B030BD00BF0AD7233C10B54FF441
:1046E0008011044609F03CFE10B12046FFF79EFF02
:1046F0004FF48001204609F033FE28B123F0EEFD8F
:10470000BDE8104021F07CBC10BD000030B500F5C4
:104710008E5591B000230835029302A90023044668
:104720000DF1070228468DF807300DF063F803A954
:1047300028460CF0B5F808B92D4B03933022002120
:1047400004A8A9F0F5FEA3238DF8103095238DF869
:10475000113080F0EFFB04F5A042CDF81300D2F841
:10476000DC32ADF81B3004F58053D2F8E022CDF8EE
:1047700017104620D3F8C013D3F8C433ADF81D107A
:10478000ADF81F20ADF821305BF066FC10EE103A5A
:104790001520CDF823305BF05FFC10EE103ACDF819
:1047A000273004F52D539FED137AD3ED297A67EE68
:1047B000877A284617EE903ACDF82B30029BCDF839
:1047C0002F309DF807308DF83330039B0D930DF09B
:1047D00017FA04F580433022D3F8803C8DED0E0AA1
:1047E00004A904F6A8600F934DF054FB11B030BD3E
:1047F0002292CA7F0000C84270B58EB035220446AE
:1048000000216846A9F094FEA3238DF8003095237B
:104810008DF8013001238DF8023080F08BFB04F518
:10482000A04504F54056D5F85C32CDF80300D6F823
:104830007804CDF80710CDF80B3003681B69984752
:10484000ADF80F00D6F8780403689B689847ADF878
:1048500011001D4801F05CFDADF81300D6F8780496
:1048600003685B69984710EE103AD6F87804CDF8E3
:10487000153003689B69984710EE103ACDF819304F
:1048800004F5804303F6784135220968CDF81D1000
:10489000D5F8E01DCDF82110D5F8E41DCDF8251090
:1048A000D5F8DC1DCDF82910D5F88C1FD3F8703C55
:1048B000CDF82D1004F6A8606946CDF831304DF0E2
:1048C000E9FA0EB070BD00BF982C002030B587B05B
:1048D0001622044600216846A9F02AFEA3238DF87B
:1048E000003095238DF8013002238DF8023080F0DE
:1048F00021FB04F5A045CDF803002046CDF80710B4
:1049000004F010FCD5F8CC320393144B8DF80B0057
:104910001B68D86A90F89C308DF810300368DB690A
:10492000984795F8B1328DF812308DF8110023F0C8
:10493000D5FC22F0C9FCD5F8C8328DF813008DF8EB
:104940001430162295F8B2328DF81530694604F607
:10495000A8604DF09FFA07B030BD00BF942C002036
:1049600010B58AB02722044600216846A9F0E0FD70
:10497000A3238DF8003095238DF8013009238DF89D
:10498000023080F0D7FACDF803000420CDF80710EC
:104990005BF062FB10EE103A1320CDF80B305BF0A9
:1049A0005BFB10EE103A4620CDF80F305BF054FB65
:1049B00010EE103A1520CDF813305BF04DFB10EEE1
:1049C000103A0320CDF817305BF056FB10EE103A8A
:1049D0001A20CDF81B305BF03FFB10EE103ACDF8FB
:1049E0001F3004F599430C3327221B68CDF8233080
:1049F000694604F6A8604DF04DFA0AB010BD0000FB
:104A000013B5044600F6A86001904CF075FD0198BE
:104A10004CF00CFE94F9D83F01980BB14CF0AEFE6F
:104A2000204602B0BDE81040FFF79ABF7047000073
:104A300010B500F580430446D3F8440C03685B6866
:104A4000984704F50053014693F8982104F6A860AE
:104A50004DF0E0FB04F58E5008300DF02BFB04F513
:104A60009070BDE810401BF063BA00009FED020A91
:104A7000002245F063B800BF0AD7233C184B70B53D
:104A8000044640F8043B59F05DFD164E164B63603A
:104A90005425601959F00CFF66513035B5F5557F36
:104AA000F7D104F555705BF0CBFE04F27C75FF2363
:104AB00084F88C3784F894370C49284645F04EFA30
:104AC0000B4B1A6812B10B4880F0FAF91D600123F4
:104AD0002046094984F8C13745F040FA204670BDA8
:104AE000C0370020BC840C08D0840C0894B60D0894
:104AF0005497002094710C08B8740C082DE9F0410B
:104B000000F508519AB00D22143104464BF0B2FD65
:104B10000022BC48BC4E272144F088FF042100201D
:104B20005BF068FE132101205BF064FE4621022049
:104B30005BF060FE152103205BF05CFE5BF0C6FBC2
:104B400045F012FCB14A138843F0040313804FF080
:104B500000080AAF002110223846A9F0E9FC012321
:104B60008DF830303388ADF8283005A973680B9381
:104B7000384644F063FEC8B19DF91430002B15DDB2
:104B800059F060FE9DF81410036801391B68C9B222
:104B9000984758B1051D284644F09AFD30B9B368CE
:104BA000ADF8183006A9284646F07CF808F106084A
:104BB000B8F12A0F06F10C06CCD1954800220DF170
:104BC0000B0144F06DFB06AD064620B344F080FDBA
:104BD00008BB904B0FCB85E80F0004A9284644F092
:104BE0002DFE002840F036814FF004088A4B0FCB91
:104BF00087E80F0005A9384644F020FE28B105A833
:104C000044F066FD08B148F0010803A930468DF86C
:104C10000C8045F0F5FF814B0FCB85E80F0003A911
:104C2000284644F00BFE002846D00998002204A92B
:104C300044F036FB064600283ED044F049FD0546C8
:104C4000002839D19DF80C30013BDBB2032B96BF15
:104C5000734A0346D35C8DF828303046394645F018
:104C6000CFFF7048002205A944F01AFB064668F001
:104C7000B5F878B168F0B0F890F8302090F82810C6
:104C800090F84830114490F840200A44D34214BFB1
:104C90000125002586B130469DF90C8044F018FDB1
:104CA00050B91DB1B8F1000518BF0125394630468D
:104CB0008DF8285045F0A4FF04F50A500022B7EE05
:104CC000000A0121303044F039FF04F50950002278
:104CD000B7EE000A02210C3044F030FF012304F546
:104CE000F6510093504A002308318E2044F0A2FE72
:104CF00094F9A4C6BCF1000F1AD14C4E0FCE3D461C
:104D00000FC50FCE0FC50FCE0FC596E80F0085E873
:104D10000F0062460421384644F088FE9FED440AA5
:104D2000444845F0BBFC4448B7EE000A45F0B6FCE9
:104D30000125424A0095002304F5025140F2051076
:104D400044F078FE022104F50A50FFF78FFE04F5C7
:104D5000075003212830FFF789FE04F5075003218F
:104D60003030FFF783FE04F5095003213C30FFF794
:104D70007DFE04F50A5002210430FFF777FE04F5AA
:104D8000075002213C30FFF771FE022104F5085064
:104D9000FFF76CFE04F5075002213830FFF766FE7E
:104DA00004F5B94020307EF065F8254A1368D9072C
:104DB00008D42449156004F5005328330B6004F629
:104DC000BC73CB601F49022204F50B50012544F04F
:104DD00083FE1D4A0095002304F6A861FD2044F0DF
:104DE00029FE1A4B1A68D20705D4194A1D6004F52A
:104DF00087540C3414601648012144F089FE1AB01F
:104E0000BDE8F081F4710C0864740C08648D002016
:104E1000B8710C085C270C086C270C087C270C0860
:104E2000F0710C08C3710C08B0980C088C270C08A2
:104E300000000000D0710C08DF710C08C8B10D082B
:104E40008C2C002000220020EC260D08902C002045
:104E50001822002004A844F03BFC00283FF4C4AE14
:104E60004FF00C08C2E600BF0020704700207047DA
:104E700000207047002070470020704770470000F6
:104E8000002070470020704784B001A880E80E0021
:104E900004B00020704700000020704770470000F9
:104EA0001020704700487047E0800C0800487047A9
:104EB000F0800C0800207047704700000120704708
:104EC0000120704700207047002343608360C36067
:104ED00003614361002303767047000010B5044668
:104EE000FFF7F2FF0023637610BD0000027E531C23
:104EF000DBB2042B037600EB820288BF002382ED35
:104F0000010A88BF0376704710B50446FFF7EEFF2D
:104F1000D4ED017A9FED107A94ED020A637E77EE6C
:104F2000877A042B77EE807A94ED030A94BF0133DD
:104F3000052377EE807A94ED040A637677EE807A23
:104F4000637E94ED050A77EE807A00EE103AB8EEB3
:104F5000C00A87EE800A10BD0000000003F024BEE6
:104F600003F036B803F088BA03F040B801F090BC03
:104F700001F016B801F0B4B901F0FAB9FDF7ECBBD5
:104F8000FDF78CB870B5234B036000F54053044621
:104F9000D3F80C04204AC3F8502208B113F0E0FA09
:104FA0001E4B236004F5805393F8642E42B9D3F866
:104FB000605E2DB1284620F09BF8284613F0CCFA0D
:104FC00004F58650103077F0B1FA04F6D8705CF032
:104FD000B5FE04F6AC3504F64C36B54204D0183DA7
:104FE00028461FF0DBFCF8E70D4BC4F8903504F5BC
:104FF000DE6050F0DDF804F2C46050F0D9F804F23D
:10500000246050F0D5F804F5BF6050F0D1F8204688
:1050100070BD00BF1C680C08E0410D08EC1F0D08B6
:105020001CE90C0838B54B4B044640F8043B61F0D2
:10503000D9F804F1100010F0DBFA04F1680049F02F
:105040007BFA04F590701AF079FB04F51C700EF0F1
:10505000D1FF04F5657013F085FA04F5B26021F014
:10506000FFF804F6283060F09BFE04F6F83046F0B6
:10507000ABF804F6A8604CF041FE04F6BC7066F094
:10508000E7FD04F6D8705CF041FE04F58050143062
:1050900012F00CF804F58650103077F033FA04F56E
:1050A00087500C3049F00AFE04F58A5062F078FA15
:1050B00004F580530025284A83F8645104F58B5089
:1050C00004F58B5304331430136041F0CBF804F52E
:1050D0008E50294608300BF0C1F804F5C15010304D
:1050E00071F020FB04F5E750143074F02DFA04F54C
:1050F000F0500C3076F060FB04F5F350103076F091
:1051000095FF04F5F65008300AF00CF904F500504C
:10511000283071F0E9FF04F5025067F035F904F525
:10512000055077F08BFD04F5005304F5065083F825
:1051300098510A4D303077F0A3FE2B6813B1084820
:105140007FF0BEFE2046074944F008FF2C60204651
:1051500038BD00BFEC1F0D08BC960020C08D00209C
:10516000F8800C08F41E0D082DE9F04F2DED028B90
:1051700004469FB0FFF756FFE44B236004F50B5045
:10518000FFF77CFC04F52A50043004F5005879F050
:1051900039FA04F509531E33C8F8AC3A04F52B501C
:1051A000062388F8B03A18305CF0C2F904F5B94328
:1051B0002033C8F8583B0E934FF4006304F52D5686
:1051C000C8F85C3B04F507595A2304F58E5788F854
:1051D000DC3B09F11809CE4BDFEDCE8AC8F8549BB1
:1051E0000837C8F8507BB7EE008AC6F8603104F57E
:1051F0003450C94BC6F86831C6F8CC3186ED578AB1
:10520000C6ED598A1C3050F0F3FA04F534502830BA
:1052100050F0EEFA4FF0000AC04BC8F8383D88F85D
:1052200050AD06F5FC70FFF74FFEBD4BBD49C8F809
:10523000383D88F851AD304644F090FEBA4BC8F87E
:10524000583D08F658530022C8F85C7DC8F8606DD8
:1052500004F535555A63DA6304F53650012388F8AE
:105260009C3D1835303012F06DFD88F8C0ADAF4967
:10527000284644F073FE04F537504946043079F06F
:1052800077FD04F53C5049461C3079F0D5F904F51A
:105290004150494604F5405834307AF033F92C2215
:1052A000514608F50670A9F043F904F54750A049A6
:1052B000283004F5495A44F051FE0AF1100A9D4B7A
:1052C000C8F850320AF114007EF05EFD04F54A5B26
:1052D00004F54B530BF1080B2C3358460F9355F044
:1052E0000DF90F9B0BF1140B5B45F6D10723C8F8A2
:1052F00010340023A8F814344FF4CB7013F02AF9BB
:10530000C8F80C0404F5505018307EF03DFD04F54B
:1053100051501C307EF038FD874B1A680AB9C3F82B
:1053200000A0864BC8F8503204F551504FF480511C
:10533000C8F878543C3010F05DFA04F553503C3016
:1053400042F00AFB04F554503C3045F04FFD04F5A3
:105350005550103069F066FA04F5964004F5804522
:105360006C3004F0A5FA764BC5F86C3B04F596401A
:10537000743004F09DFA734BC5F8743B04F5964005
:105380007C3004F095FA704BC5F87C3B04F59740EF
:10539000043004F08DFA6D4BC5F8843B05F6983364
:1053A000002204F59740DA609A605A6083ED008A23
:1053B0002C3004F07DFA664BC5F8AC3B04F5974001
:1053C000343004F075FA634BC5F8B43B04F59740EC
:1053D0003C3004F06DFA604BC5F8BC3B04F59740D7
:1053E000503004F065FA5D4BC5F8D03B04F59740AA
:1053F000583004F05DFA5A4BC5F8D83B04F5974095
:10540000703004F055FA574BC5F8F03B04F597405F
:10541000783004F04DFA544BC5F8F83B04F5984049
:1054200004F5984A04F044FA0AF10C0A4F4BC5F807
:10543000003C504604F03CFA4D4BC5F80C3C04F5DA
:105440009840143004F034FA4A4BC5F8143C04F583
:1054500098401C3005F0B6FFFE2385F8503C05232C
:1054600085F86C3C4FF0FF3B434BC5F844ACC5F8A6
:1054700048ACC5F874BC119305F68C453F4B85EDDF
:10548000008A04F5994022464FF4007100931030D1
:10549000394B109404F5A0450FF092FB0023C5E9A9
:1054A000A333C5E9A533C5E9A7330323C5F8C8323B
:1054B000334BC5F834B2C5E9C334324BC5ED948AD9
:1054C000C5E9C53404F5A6402F4BC5F81C3385ED5E
:1054D000B98AC5F80843303012F034FC04F5A64010
:1054E0004C3012F02FFC04F5A64004F5A54A6830B4
:1054F00012F028FC0AF16C0A244BC5F87C33A5F89D
:1055000080B30AF1980012F01DFC41E01C680C0801
:10551000000080BF0000B4420000B4C264810C08E7
:1055200074810C08E8F20D085CF00D0804F00D0819
:10553000A0EA0D08E0410D080891002078350C081C
:10554000208B0C08048F0C08EC900C0874890C0854
:10555000288C0C08AC8C0C08948B0C08A48A0C08C2
:10556000248A0C088C8E0C089C8D0C08288D0C0845
:105570009C810C08188E0C085D4F01084C320C08F9
:10558000614F0108654F0108694F01080000FFFFE6
:10559000704B7149C5F8E0B35046C3F800A044F021
:1055A000DDFC4FF6FF73A5F8283304F5A7406B4BDD
:1055B0006B49A5F844B36430186044F0CFFC04F59F
:1055C000A84004304AF04AFC664BD8F8782412947C
:1055D000CDE91334644BCDE91534644BCDE9173470
:1055E000634BCDE91934634BCDE91B34624B1D93FA
:1055F0001EA911E903000CAB83E80300DDE91A01E1
:105600000AAB83E80300DDE9180108AB83E8030077
:10561000DDE9160106AB83E80300DDE9140104AB04
:1056200083E80300DDE9120102AB83E8030004F51F
:10563000BA4833465146CDE900290E983A467DF0E6
:1056400021FA08F12C084D4BC5F82C3D08F13C001F
:1056500012F078FB4A49404644F080FC494B1E68F2
:1056600016B149487FF02CFCC3F8008007F51B7782
:10567000464BC5F82C3D04F5BB40C5F8B47D85F814
:10568000306D85F8356D85F8596D383012F05AFB5C
:1056900004F5BB40483012F055FB04F5BB405830D0
:1056A00012F050FB1C22314605F6E850A8F040FFEE
:1056B00004F5BD4704F5BC40543750305CF074FC31
:1056C000384677F097FC324B3249C5F8D43E38461D
:1056D00044F044FC304A3149116004F5BE430C33B8
:1056E0001427B0B207FB00120136127C002AF8D151
:1056F0002B4A10802B4A16680EB12B48B2E704F5EE
:10570000BE401030136077F05FFC284BC5F8103FA7
:10571000274BC5F8203F642385F8243F254BC5F867
:10572000583F04F5BE40244BC5F85C3F2349203068
:1057300044F014FC224BC5F8203F20460123C5F855
:10574000806F85F8886F85F874321FB0BDEC028BCE
:10575000BDE8F08FA48C002078F60C08C4960020D9
:1057600018580D086D4F0108714F0108754F010859
:10577000794F01087D4F0108814F01084C810C08C9
:1057800080EE0D08D89E00200C810C08F4840C08D3
:10579000F42B0C08CC2B0C08788D002068760C08B4
:1057A000748D0020308D002028810C08342C0C08CA
:1057B00084810C08FC940C0854950C083C490D0895
:1057C000D4960C0810B57EF0BFFE064C064B186050
:1057D0002046FFF7C9FC2046044A0549BDE81040B1
:1057E000A6F038B9982C0020942C002020EC002042
:1057F000854F01080069C0F3401070470F299DBF15
:10580000302303FB0100503000207047014B93F917
:105810005D027047984C0020014BD3F8980A7047FE
:10582000984C002008B503689B68984730B9044B32
:1058300093F85E0CB0FA80F0400908BD0020FCE748
:10584000986C002008B5044806F0D0FD10B9034B51
:1058500093F8580C08BD00BF982C0020986C0020CD
:10586000022A10B50C4605D1BDE810400948352282
:1058700008F066BC084BD3F8440C03685B68984793
:10588000A04205D158F0DEFFBDE8104058F064BFDB
:1058900010BD00BF982C0020986C0020012910B585
:1058A0000C4614D0022907D0D1B90E4BC3F8801F83
:1058B00057F0D6FA0C4A05E00A4BC3F8801F57F0A0
:1058C000CFFA0A4ABDE81040062150F00BBC57F051
:1058D000C7FA074A062150F005FC024BC3F8804F77
:1058E00010BD00BF987C0020B3820C0888820C0891
:1058F0009C820C08012902D0022900D011B9024B68
:10590000C3F8841F704700BF987C0020622910B440
:1059100000F3888047291ADC402900F0958008DCD4
:10592000162951DC032904DD4F4B01248C40234010
:1059300053B95DF8044B59F057BEA1F19604012309
:10594000A3404A4C2342F4D05DF8044B7047A1F1C8
:1059500048031A2BEDD801A454F823F04959010843
:1059600033590108335901083359010833590108E3
:1059700049590108335901083359010833590108BD
:1059800033590108335901083359010833590108C3
:10599000335901083F5A01083F5A01083F5A01088C
:1059A00049590108335901083F5A0108495901086A
:1059B0003359010833590108495901084959010867
:1059C0003359010849590108A1F12703112BB0D817
:1059D000112BAED801A454F823F000BF4959010897
:1059E000335901083359010833590108495901084D
:1059F0003359010833590108335901083359010853
:105A0000335901083359010833590108495901082C
:105A10004959010833590108335901084959010806
:105A200049590108B02904DC952986DC6B2980D10D
:105A30008AE7A1F1D003022B3FF67BAF84E75DF844
:105A4000044B002359F0A2BD094B012283F87C2F9F
:105A5000A3F54053D3F8940A00283FF475AF5DF8DE
:105A6000044B642158F034BF10004100A1008004B1
:105A7000987C002038B50B46622B0446114600F393
:105A80009580472B13DC382B7ADC262B4CDC102B33
:105A900000F0B580162B00F00481042B00F0C680C6
:105AA0000A4620461946BDE8384059F0DBBAA3F152
:105AB00048021A2AF4D801A050F822F0075C010825
:105AC000A15A0108A15A0108A15A0108A15A0108C6
:105AD000315C0108A15A0108A15A0108A15A010824
:105AE000A15A0108A15A0108A15A0108A15A0108A6
:105AF000A15A01083D5C01087D5C0108A15A01081A
:105B00009B5C0108A15A0108855C0108375C01080B
:105B1000A15A0108A15A0108ED5B0108AF5C010818
:105B2000A15A0108155C0108A3F12702112AB7D870
:105B300001A050F822F000BFED5B0108A15A010856
:105B4000A15A0108A15A0108F15B0108A15A0108F4
:105B5000A15A0108A15A0108A15A0108A15A010835
:105B6000A15A0108A15A0108275C01080F5C01082D
:105B7000A15A0108A15A0108215C01081B5C010817
:105B8000402B8DD1931E5942624C594184F87B1FA2
:105B900057F066F9604A94F87B1F604B002908BFF4
:105BA00013465F4A062150F09DFA1FE09B2B00F040
:105BB0008B8007DC6B2B00F09180962B7FF470AF0D
:105BC00007211DE0AD2B77D00BDC9D2B7FF468AF58
:105BD0000124002A7ED0022A5AD14E4B83F87A4FF4
:105BE00056E0A3F1D002022A3FF65AAF01244FE05B
:105BF0008A1E4C4B5142514183F8511CF6E70A2151
:105C0000FFF72EFEF2E70A4601212046F8E70A4692
:105C10000421FAE70A460321F7E70A460C21F4E7D4
:105C20000A460F21F1E70A460021EEE70B21E7E7DC
:105C30000A460D21E9E70A460521E6E7354CD1B1D0
:105C400002290DD1012384F8783FA4F58053D3F8BD
:105C5000440C03685B6A984710B1334800F0A4FD18
:105C600057F0FEF8314A94F8781F314B002908BFED
:105C70001346304A96E784F8781FE6E72046FFF798
:105C80000DFEB3E7012429B1022901D12A4B1C756D
:105C9000204638BD284B1975FAE72046FFF72AFE43
:105CA000A4E7022AA2D1204806F044F99EE758F062
:105CB000C9FD58F051FD99E7022A97D19FED1F0ABF
:105CC0001948FCF743FA91E7022A8FD1164806F0EB
:105CD0009BFA8BE70F4B83F87A2FD9E7022A14D16E
:105CE000104DD5F8440C0368DB6B9847044628B187
:105CF0000121A5F5804002F0CBFCC9E757F0B0F8D0
:105D00000F4A042150F0EEF970E70748002102F035
:105D1000BFFC6BE7987C0020C8820C08AF6A0C08B7
:105D2000D0820C08986C0020982C00200B560C0890
:105D30006C8F0C08E0820C08984C002000000000DA
:105D4000F3820C0810B5084CD4F8440C03689B6B24
:105D5000984738B9D4F8440C04F61444001B18BF13
:105D6000012010BD0220FCE7986C002008B502213C
:105D700003205AF089FC022108465AF085FC0121D3
:105D800004205AF081FC022115205AF07DFC1320DA
:105D900002215AF079FC124806F094FDA8B10021C6
:105DA00046205AF071FC002149205AF06DFC002178
:105DB0004A205AF069FC002101205AF065FC0021BC
:105DC000BDE8084008465AF05FBC012146205AF061
:105DD0005BFC012149205AF057FC0121E8E700BF94
:105DE000982C002002490348052208F0CDB800BFD6
:105DF00070780020982C002038B5304B01241C709E
:105E000090F90A302B2B0CD12D487DF031F82D481C
:105E100007F098FEBDE838402B4801220921FBF726
:105E2000B7BD284D9FED290AD5ED460A6421032010
:105E30005AF0F4F9D5ED460A9FED240A64210220B8
:105E40005AF0ECF99FED220A03205AF0F1F89FED89
:105E5000200A02205AF0ECF89FED1E0A04205AF0A6
:105E6000E7F89FED1C0A15205AF0E2F813209FED89
:105E7000190A5AF0DDF8284606F024FDA0B10021E9
:105E800046205AF02FFC002149205AF02BFC00211B
:105E90004A205AF027FC002101205AF023FC00215F
:105EA00008465AF01FFCB2E7214646205AF01AFC79
:105EB000214649205AF016FC2146E9E76891002066
:105EC00038890020982C00206C8B002000000000F6
:105ED0000000C84200A08C4500F58040D0F8440C7A
:105EE00003681B6C1847000000F5005393ED9F7A80
:105EF00000F5A040B5EEC07AF1EE10FA5DBFD0F823
:105F0000B43DDFED086AD3ED017AD0F8CC0D5FBF68
:105F1000F8EEE77AE7EE267AFDEEE77A17EE900ADA
:105F2000704700BF0000C84200F5005090F8BC0266
:105F300028B141F00101084214BF01200020704740
:105F400013B50346FFF7F0FF58B103F5005191F880
:105F5000B40AC00705D501F52D6191ED000A02B024
:105F600010BD03F5A04422B904F6046494ED000AC0
:105F7000F5E794F89C2C022AF6D103F5A8400122FB
:105F800001A904304AF0F0F80028EDD09DED010A97
:105F9000E5E7000000F5A04393F8F02DFFF7D0BF30
:105FA00010B54B68516800F5A0448B42D8BF0A4633
:105FB000D4F8E80DCCBF1A46194622F0ABFFC4F85E
:105FC000E80D10BD10B50446564866F039FB10F0D8
:105FD000080217BF544BDFED557A93ED237AD3EDCA
:105FE000257A1FBF77EE877A9FED517A012267EEFF
:105FF000877A10F0010317BF4B4B9FED4C7AD3ED1E
:10600000256A93ED227A1CBF37EE667ADFED486A87
:1060100004F5005118BF27EE267AD1EDA16AF5EEFE
:10602000C06A18BF0123F1EE10FA3CDD3E4A9FED35
:10603000406AD2EDA16A66EE866A0122F4EE676AD2
:10604000F1EE10FA58BFF0EE667A04F5A04090F831
:10605000F01D69B393B1D0F8F43D06EE903AF8EE36
:10606000E66AF4EEC76AF1EE10FA58BFF0EE476A3E
:10607000FDEEE66A16EE903AC0F8F43DBAB1D0F8FB
:10608000F43D07EE103AB8EEC77AB4EEE77AF1EED7
:1060900010FAD8BFB0EE677ABDEEC77A17EE103AA5
:1060A000C0F8F43D03E0002ACFD1002BCDD110BDC4
:1060B000D3B1D0F8B43DD3ED016AD0F8E83DF8EEA5
:1060C000E66A76EE876A07EE103AB8EEC77AF4EE23
:1060D000C76AF1EE10FAD8BFB0EE667ABDEEC77AA5
:1060E00017EE103AC0F8E83D002AE0D0D0F8B43DF1
:1060F00093ED017AD0F8E83DB8EEC77A77EE277ACB
:1061000007EE103AB8EEC77AF4EEC77AF1EE10FA5D
:1061100058BFB0EE677ABDEEC77A17EE103AC0F8F6
:10612000E83DC4E7184D0020984C00200000000016
:106130000000C84200F5A0400023C0F8EC3D7047C5
:1061400073B51646054600236A463046009311F0A3
:10615000E7FE48B1DDED007A9FED287A67EE877A99
:10616000FDEEE77A17EE900A05F5A044C4F8EC0DB1
:1061700033785B071CD594F8F03DCBB105F5A8400A
:10618000012201A9043049F0EFFF88B1D4F8F43DB1
:10619000DDED016A9FED197A07EE903AF8EEE77AA5
:1061A000E6EEC77AFDEEE77A17EE903AC4F8EC3DDA
:1061B000D4F8C832042B1FD005F50055B5F9B62226
:1061C000002A16DDD4F8EC3D9FED0D7A83EAE371E9
:1061D000A1EBE37107EE901AF8EEE77A67EE877AA3
:1061E00007EE102AB8EEC77AF4EEC77AF1EE10FA8D
:1061F00002D50023C4F8EC3D02B070BD0000C842D7
:106200000AD7233C37B50B785A0704460D461DD5EF
:1062100000F5A840012201A9043049F0A5FFA8B16A
:10622000D5ED017A2B78DFED1C6AF8EEE77ADB0713
:1062300067EEA67A1BD59DED017AB4EEE77AF1EE12
:1062400010FACCBF0120002003B030BD2B78D5ED73
:10625000017A13F0010FF8EEE77A04F5A04411D1AA
:1062600004F6CC5393ED007AB8EEC77AE5E704F56F
:10627000A044D4F8B43D93ED017AB8EEC77AE7EEC6
:10628000667AD8E7D4F8B43D93ED017AB8EEC77AD0
:1062900077EE877AE4E700BF0AD7233C00F5005386
:1062A00000F58042B3F96632D2F8442C00EE103A81
:1062B00000F5974358339A42B8EEC00A0ED100F564
:1062C000A040D0F8C832042B02D090F875322BB120
:1062D00000F54A60D0ED007A30EE270A70470000E2
:1062E000014608B501F5A041FFF7D8FF01F6CC53F0
:1062F000D3ED007A9FED057AF8EEE77AE0EE477A83
:10630000FDEEE77A17EE900A08BD00BF0000C84214
:1063100037B500F5A045044695F8F03DFBB100F512
:10632000A840012201A9043049F01EFFB8B105F6CA
:10633000F452D2ED007A9FED0D7A05F6F853D3EDC5
:10634000006AF8EEE77AE6EE877ADDED016AE6EEBE
:10635000C77AFDEEE77A17EE900A03B030BD20460B
:10636000FFF7BEFFD5F8E83D181AF6E70000C8426F
:10637000014608B5FFF792FF01F5BC40D0ED017A68
:1063800037EEC00ADFED047A20EE270AFDEEC07A70
:1063900017EE900A08BD00BF0000C8422DE9F04189
:1063A00000F5BB4800F5BB4508F1480858350446E0
:1063B0002946404612F028F804F5BB4604F5A047EC
:1063C00038362A463146404687ED970A11F052FF8B
:1063D000DFED220A87ED980AB7EE001A762022F048
:1063E000F9FC04F52D5383ED710A2046FBF756FEA8
:1063F00004F58043D3F8440C03685B6898470B2886
:106400000BD006D80A280FD00023C7F8EC3DBDE812
:10641000F0810E38C0B20128F6D829462046FFF791
:10642000F1FE0028F0D011E029462046FFF7EAFEF1
:1064300030B90B484FF48041FCF790F80028E3D1C5
:106440002046FFF795FFB0F5FA6FE6DD2A463146A4
:106450002046BDE8F041FFF773BE00BF000000001A
:10646000982C002010B52DED028B00F5A043DFED38
:10647000208AD3F8DC2D93F8D83D07EE902AB8EEA9
:10648000E78ADA0728EE288A82B0044609D400F5A4
:10649000805202F58762D2ED007AF8EEE77AA7EE35
:1064A000E88A5B070FD504F5A840012201A9043052
:1064B00049F05AFE38B19DED010A30EE480A02B0AB
:1064C000BDEC028B10BD204604F58054FFF708FF99
:1064D00004F5876393ED000A07EE900AB8EEC00A50
:1064E000F8EEE77A28EEC00AA7EEA80AE5E700BFB3
:1064F0000AD7233C38B52DED028B00F5804200F51C
:106500009743D2F8442C34339A4204464DD100F5D7
:106510008053D3F8C85300F50053B3F9B432002BBD
:1065200066DD04F5AE5292ED037AF7EE007AB4EE32
:10653000E77AF1EE10FA5BD404F52D52D2ED0A7A27
:10654000F6EE006A67EEA67A87EE871AB5EEC01AF5
:10655000F1EE10FA4CD907EE905A9FED288AB8EE6A
:10656000E70A07EE903A04F5A84004F5A044F8EED7
:10657000E70A20EE080A043049F002FFD4F8EC3DA7
:106580009FED1F1ADFED1F0A002BBCBF07EE903AEC
:10659000F8EEE77A4FF42970B8BFA7EE880ABDEC91
:1065A000028BBDE8384022F015BC05F05DFBF8B960
:1065B00004F54053D3F8780403681B69984704F541
:1065C0000053DFED100AB3F9B43201EE103A04F5CE
:1065D000A04393ED970AB8EEC11A054640F27F201A
:1065E00022F0F8FBBDEEC00A10EE103A1BB296E79F
:1065F000BDEC028B9FED030A38BD00BF0AD7233CD8
:1066000000007A440000000010B504467EF08AFCC9
:1066100004F50053D3F8C82A801A41F28832904218
:106620000FD802212046FFF77FFC50B104F5A044AB
:10663000D4F8C822042A04D103F6BC2393ED000A3F
:1066400010BD9FED010AFBE70000000030B52DED05
:10665000028B00F5A045DFED298A95F8F03D83B067
:1066600004467BB3D5F8F43D9FED250A07EE903A3A
:10667000F8EEE77A00F5A84027EE800A012201A98A
:10668000043049F0A9FDE8B12046FFF733FFDDED06
:10669000017A05F6F85585ED000A37EE800A2046A6
:1066A0008DED010AFFF7B0FFDDED017A30EE270A2C
:1066B00020EE280ABDEEC00A10EE100A03B0BDECB1
:1066C000028B30BDD5F8B42DD5F8E83D52689B1A41
:1066D00008EE103A2046FFF7E1FDB8EEC88A2046E2
:1066E000A0EE288AFFF790FFBDEEC88AB8EEC88AF0
:1066F000A0EE288ABDEEC80ADEE700BF0000C8424F
:106700000AD7233C10B500F580430446D3F8440C67
:1067100003685B6A984718B104F5A04494F8780FB1
:1067200010BD000038B500F5A0440D46D4F8E83D92
:106730000B44C4F8E83D94F8F03D3BB1FFF7E2FFAD
:1067400020B9D4F8F41D2944C4F8F41D38BD000064
:1067500030B500F50050D0F8B022D3070FD4094B64
:1067600008201D785C688D4204D1224214BF0120AC
:10677000002030BD013803F10803F2D1F9E7012010
:10678000F7E700BF44850C0810B500F580430446C8
:10679000D3F8440C03685B68984701462046BDE87F
:1067A0001040FFF7D5BF000037B500F5A0440546FF
:1067B000D4F8CC3DC4F8E83D0023C4F8EC3DFFF725
:1067C000E3FFE0B105F5A840012201A9043049F03A
:1067D000CBFCA0B12846FFF795FF80B9DDED017A2B
:1067E0009FED097A67EE877A0123FDEEE77A84F858
:1067F000F03D17EE903AC4F8F43D03B030BD0023ED
:1068000084F8F03DF9E700BF0000C84238B50446FF
:106810000D46FFF7B9FF30B10321284611F05CFBAC
:1068200080F00103D8B204F5A04484F8F10D38BD1E
:1068300073B500F5A0444A68C4F8E82D0B780D46FE
:10684000D90741BFD4F8B43D5B689B18C4F8E83D54
:1068500094F8F13D064623B100F5BB415831FFF7EE
:10686000D5FF2B785B070FD506F5A840012201A9BB
:10687000043049F079FC38B1012384F8F03D6B68AD
:10688000C4F8F43D02B070BD002384F8F03DF9E790
:10689000F0B52DED028B044683B004F5A0450E46FD
:1068A0008DED010AFFF7C4FFDFED360A9DED010A09
:1068B00040F24310B7EE001A22F08CFAD5F8EC3D06
:1068C0005B4207EE903AF8EEE77A204667EE807A70
:1068D00004F50057FDEEE77AB0EE408A17EE901A05
:1068E000FFF720FFD7EDAE7AF5EEC07AF1EE10FAA1
:1068F00043DDD5F8EC3D002B3FDD2046FFF708FDDA
:1069000007EE900ADFED206AB8EEE77AD7EDAE7AAF
:1069100067EEA67AB4EEE77AF1EE10FA2DD531469D
:106920002046FFF785FF04F5BB413246483120463B
:10693000FFF706FCD5F8EC3D5B4207EE903AF8EE27
:10694000E77A204667EE887AFDEEE77A17EE901A2E
:10695000FFF7E8FEB5EEC08AF1EE10FA0DDDD5F8CE
:10696000EC3D07EE903AB8EEE77AC7EE087AFDEE16
:10697000E77A17EE903AC5F8EC3D03B0BDEC028B18
:10698000F0BD00BF000000000000C8C2F0B500F577
:10699000A04487B094F8D83D03F00503052B0746C3
:1069A0000BD04AF05DFC4FF4AE724FF480114AF008
:1069B0000FFC0025284607B0F0BD1E486A4603219B
:1069C00011F09AFA0028F4D01B4801AA032111F013
:1069D00093FA05460028ECD0184BDFED190A93ED29
:1069E000980A40F26D10B7EE001A22F0F3F904F69F
:1069F000D8530FCBB0EE401A02AEDFED111ADDED29
:106A0000010A9DED000AB7EE002A86E80F0022F089
:106A100013F9DFED0C7A20EE270A3046FDEEC07A3E
:106A2000032217EE901A11F093F931463846FFF71A
:106A3000FFFEBFE7508A0020708A0020987C00206B
:106A4000000000000000C842F7B50D4602210446D0
:106A5000FFF76AFA60B304F5A047D7F8C832042BF1
:106A600026D12046FFF790FE10B304F5A846043661
:106A700004F5BB4101236A464831304649F05EFACD
:106A8000B0B104F5BB41012301AA5831304649F0A9
:106A900055FA68B19DED017ADDED007A77EEC77A9F
:106AA00095ED007A37EE277A85ED007AC7EDA07A6A
:106AB00003B0F0BDF0B52DED048B00F5005489B0A6
:106AC00000F6F83694F8821A03910546304644F0F1
:106AD0004BFC03990746304644F058FC042F0399B9
:106AE000B0EE408A20D1002305A88DED050A06935B
:106AF000079324F0FFFC05F5A75005A9083022F004
:106B00001BFCDFED9B7A8DED050AB4EEE71AF1EE82
:106B100010FACDED060A8DED071A05DB05F5805359
:106B200093F84434DF070CD494F8B43A002262F3AB
:106B3000000384F8CC2A84F8B43A09B0BDEC048B85
:106B4000F0BD94F8B43A98075CBF43F0020384F8B0
:106B5000B43A04F52D6758BF04F6B82305F52B5158
:106B600058BF83ED008A103187ED001A2846FFF7E1
:106B70006BFF94F8CC3A092B00F2898004F6D423F9
:106B8000D3ED000A9FED7B9AB0EE480A22F010F890
:106B900000BB04F6B82394F8821AD3ED008A30467D
:106BA00044F012FC07EE900A9FED737AF8EEE77A54
:106BB00078EEC88A67EE877AF0EEE88A67EE897A1F
:106BC000F4EEE78AF1EE10FAC2BF94F8CC3A013342
:106BD00084F8CC3A04F6D42394F8821AD3ED008AD0
:106BE000304644F0F1FB07EE900AF8EEE77A9FEDAD
:106BF000637A67EE897A78EEC88A67EE877AF0EE74
:106C0000E88AF4EEE78AF1EE10FA02DD002384F858
:106C1000CC3A04F6D42383ED008A94F8B43ADA0728
:106C20008BD5284605F5A046FFF71CFC04F52D631F
:106C300093ED008A96F8F03D30EE488A002B4CD058
:106C400005F5A840012205A9043049F08DFA002875
:106C500049D17EF067F9D4F8C82A41F28831821A06
:106C60008A42034604F6BC2205F52B5144D982ED35
:106C7000008A284681ED008A0221FFF755F918B1F4
:106C800006F54A66F268B260C4F8C83A55E794F867
:106C9000B43A43F00103590784F8B43AB9D405F57E
:106CA000A042D2F8C822042AB3D102212846FFF715
:106CB0003BF90028ADD043F0040384F8B43A3868B7
:106CC000F9F722FC05F549561036CDE900012C4AAA
:106CD000062130464FF006FA9BE72846FFF754FDA1
:106CE0000028ADD1B5E704F52D6393ED000A9DEDC5
:106CF000058A38EE408AACE79FED200A92ED007AD3
:106D0000DFED207A28EE008AA7EE278A82ED008A3E
:106D1000C4F8C80AD1ED007A38EE678AF3EE0E7A2D
:106D2000B0EEC88AB4EEE78AF1EE10FA7FF705AF4D
:106D300094F8B43A5B070ED504F52D6405F5495671
:106D40002068F9F7E1FB1036CDE900010E4A062173
:106D500030464FF0C7F905F52A502422002134307F
:106D600009B0BDEC048BBDE8F040A7F0E1BB00BF6B
:106D7000000000340AD7233CCDCC4C3DCDCC4C3E5A
:106D800004850C08CDCC4C3F21850C0838B52DED81
:106D9000028B0D460446FFF765FB002320462B704F
:106DA000B0EE408AFFF730FC0221204638EE400A60
:106DB000FFF7BAF828B104F5005494F8B40A00F0CB
:106DC0000100BDEC028B287038BD000070B50B7857
:106DD00003F00503042B05460C46164615D105F5B0
:106DE000A0454AF03DFAB2B24FF480114AF0F0F9F2
:106DF000D5F8B42D636852689B1A13F5FA7FC8BFA3
:106E00006360237843F00103237070BDF8B500F58B
:106E1000805300F5A047D3F83864D7F88452B542C0
:106E2000044618D00D4A1268D26A92F89C2092B19A
:106E300000F5BB41751B25225831FFF7C7FF07EE50
:106E4000905AB8EEE70ADFED067A04F52D5020EEF1
:106E5000270A7BF09FFBC7F88462F8BD942C0020C2
:106E60000AD7233CF8B500F5A044054694F877C24C
:106E70000F4604F6B856BCF1000F53D004F6D853B1
:106E80000FCB86E80F00012384F8783297E80F00D3
:106E900004F6D85686E80F00D4F8E03D05F5BB4669
:106EA000583693B9D4F8E43D7BB9D4F8D03DD4F842
:106EB000DC2DC4F8E03DD4F8D43DC4F8E43D22B95B
:106EC000D4F8CC1D304610F043FF31462822284626
:106ED000FFF77CFF94F8D81D11F0040102D1304671
:106EE00010F0FAFF05F5BB4105F5BB4032463831DD
:106EF000483011F0F5F938B104F6B85604F6C85424
:106F000094E80F0086E80F00284604F049FB284665
:106F1000FFF744FA284604F06FFE2846BDE8F84023
:106F2000FEF7DABF04F6C8530FCB86E80F00012343
:106F300084F8773284F878C2A8E70000F8B500F545
:106F400000530446B3F90E32002B0E4633DB0B78A8
:106F500013F0020F14BF4FF0FF33012304F5A045D7
:106F600005F6B85785F8903D05F6C8530FCB87E86E
:106F70000F0096E80F0005F6D85787E80F0004F5D4
:106F8000BB41572258312046FFF720FF2046FFF72C
:106F90000BFC2046FFF702FA204604F02DFE0023EA
:106FA00085F87832C5F8943D85F87D322046BDE8F5
:106FB000F84004F0F5BA4FF0FF33CFE72DE9FF4179
:106FC000354B1B680546D86AFAF7BCFA002860D131
:106FD00005F5005393F9303A5A1C53D0002B11DDBC
:106FE00095F88122242107EE903A01FB025292ED9E
:106FF000A77AF8EEE77AB0EEC77AB4EEE77AF1EE68
:1070000010FA3FDC05F5805305F58E5693F84434AD
:1070100013F0010406F1080629D0C3F340079B07CB
:1070200033D495F8401295F868424FF0B00808FB49
:10703000015191F8893154BB022B18D9684610F0E0
:1070400081FE694630460AF04BFB044678B195F85C
:10705000403208FB03533A46D3F89811684610F0C3
:1070600077FE0AF0DDFD69460AF028FA044605F5C8
:107070001C700DF093F830460AF040F92846FBF7F3
:1070800041FA204604B0BDE8F0810024EFE73C4619
:10709000EDE70020F6E700BF942C002038B50C4B3C
:1070A0001B680546D86A0C46FAF74CFA10B1002462
:1070B000204638BD0AF0B4FD21460AF0FFF9044627
:1070C0000028F4D005F5A5406C3025F001F8EFE775
:1070D000942C0020F0B500F5A045002385F8773208
:1070E00085F8783205F6C853044600EE101A0FCB27
:1070F00087B005F6B85686E80F0002AE04F5BB422D
:10710000B8EEC00A30461749483243F077FF96E898
:107110000F0005F6D85787E80F0004F5BB4140F291
:107120005712583120460191FFF750FE0199204631
:10713000FFF76CFB01992046FFF77AFB04F500533B
:107140002046B3F90E32002BB4BF4FF0FF330123BA
:1071500085F8903DFFF722F9204607B0BDE8F040E2
:1071600004F04ABDD461002010B50349044643F041
:1071700045FF204610BD00BFD4610020F8B500F5E2
:10718000A04404F6C85305460E460FCB04F6B85784
:1071900087E80F00284606F10801FFF763FEB38871
:1071A000D4F8DC2D03EB830303EB83039B001BB2BA
:1071B000002BD8BF4FF4C873A4F87232D4F8B43D92
:1071C0005968521AC4F844229A680A32C4F8E02D69
:1071D000DB680A33C4F8E43D0023C4F8583284F86D
:1071E000743284F88832C4F848320023C4F83C3240
:1071F0004FF0FF33C4F8343295F88102242303FBA7
:107200000055D5F89C32C4F86C32F8BD70B50E4606
:1072100008310546FFF726FEB38805F5A04443B3C1
:10722000642213FB02F3C4F84432B4F97232002B27
:10723000D8BF4FF47A7305F52A50D8BFA4F872323C
:10724000242200213430A7F073F904F6046305F515
:10725000B94093ED000A314620307BF009FDD4F8A7
:10726000C832072B0CD128460421BDE87040FAF73C
:10727000C5BED4F84432002BD7DC40F6B833D2E791
:1072800070BD00000B7A00F5A04013F0020F14BF90
:107290004FF0FF33012380F8903D70477FB501F137
:1072A000080305460E460FCB6C4684E80F0005F533
:1072B000BB414831204610F0AFFE21462846FFF77B
:1072C000D1FD31462846FFF7DDFF04B070BD000058
:1072D0007FB501F1080304460E460FCB6D4685E8E5
:1072E0000F0004F5BB414831284610F095FE2946B1
:1072F0002046FFF7B7FD20463146FFF7C3FF33793D
:1073000007EE903A337E9B0748BF9FED0C7AF8EE6C
:10731000677A04F5A04448BF67EE877A9FED087A44
:1073200067EE877AFCEEE77A17EE903AC4F8883D6C
:107330000123C4F8A83D04B070BD00BF0000803B2D
:1073400000A00C477FB501F1080304460E460FCBA1
:107350006D4685E80F0004F5BB414831284610F022
:107360005BFE29462046FFF77DFD20463146FFF7AC
:1073700089FFB38804F5A0444FF47A725343C4F8EC
:10738000A03D0123C4F8A83D04B070BD2DE9F34130
:1073900000F5BB450446583500F5BB400E46383075
:1073A000294610F0F9FD04F5A047C0B94FF0FF33AE
:1073B000C7F8343206F10808404610F0F3FC032801
:1073C000024638D1F168284610F0C2FCB388C7F8ED
:1073D000A83D204602B0BDE8F041FEF7ABBE19F073
:1073E00025FBFAF79FFB012812D94FF0FF33C7F8AE
:1073F000343219F01BFB90F82031DFED140AB02273
:1074000002FB030090ED220A284611F073F8D1E741
:1074100004F58058D8F8C80321F0B0FCC7F834024E
:10742000D8EDF27A9FED0A0ADFED080AF8EEE77A66
:1074300027EE800AE8E701AA0021404610F0BEFCD2
:107440000028C3D001990022BDE700BF00007A44A4
:107450000AD7233C7FB501F1080304460E460FCB43
:107460006D4685E80F0004F5BB414831284610F011
:10747000D3FD29462046FFF7F5FC20463146FFF7AD
:1074800001FF04F5A0440023C4F8A83D04B070BD7A
:1074900037B504460D467DF045FDE060D5ED027A36
:1074A000F5EEC07AF1EE10FA15DD9FED127A67EE77
:1074B000877AFCEEE77AC4ED027A55F0D1FCA26837
:1074C0004FF47A73B2FBF3F30B4A062103B0BDE825
:1074D00030404EF007BE64F001FF0023009395F9A1
:1074E0000D2095F90E3095F90C1064F093FEA06014
:1074F000E3E700BF00007A4484850C082DE9F041E1
:107500002DED028B84B004460AF08AFB09F0DCFC06
:1075100004F5805304F5A04593F8C0360BB9002854
:1075200075D0D5F83432013371D1D5F85832002BEB
:1075300049D07DF0F7FCD5F85832C01AB0F5FA6F93
:1075400065D394F84022DFED5E7A9FED5E8A4FF0BE
:10755000B00808FB024292ED6A0A20EE270A21F0E9
:1075600025FCD5ED8F7A30EE670A21F01FFCDFEDA8
:10757000567A20EE080A04F5495720EE270A21F032
:10758000BDFBFDEEC07A103717EE906AC5ED8D7A1F
:10759000D5ED8F7A67EE887A17EE900AF8F7B4FF88
:1075A000CDE9020194F8403208FB0343D3F8A4016B
:1075B000F8F7AAFF454ACDE90001334606213846CF
:1075C0004EF090FD23E004F59070FAF7ABFA022834
:1075D0001DD994F84032B02202FB034393ED697A3F
:1075E000F1EE047AB4EEE77AF1EE10FA0FDD384BE3
:1075F0001B68D86A0368DB699847012803D07DF0CF
:1076000091FCC5F85802D5F85832002B91D104F5F9
:107610004053D5F83412D3F878044A1C036846D096
:107620001B6B98472B4807F0ABFA20B104F5A54037
:107630006C3026F0E9FF2046FEF79AFED5F844327A
:107640008342064636DA07EE906A9FED237AF8EE1B
:10765000E77A04F5495467EE877A103417EE900AFA
:10766000F8F752FF1D4ACDE90001204606214EF0F1
:1076700039FD01244FF0FF33C5F8343285F87442E8
:1076800005F6C8530FCB05F6B85605F6D85786E869
:107690000F0087E80F00124864F09CFF002385F874
:1076A0007732204604B0BDEC028BBDE8F0815B6B05
:1076B0009847B7E7074807F043FA0028C3D1F1E736
:1076C00035FA8E3CE02E65420000C84294850C08D5
:1076D000942C0020982C00200AD7233CB8850C0855
:1076E000184D00202DE9F04700F5A0462DED028B46
:1076F0004FF0FF33C6F8343206F6D8538C460746AF
:107700000FCBBCF804509CF8049088B004AC2D0A50
:1077100084E80F0020D007F5BB4808F1380821465F
:10772000404610F071FE21464046B0EE408A10F00F
:107730003BFDDFED567AB4EEE78AF1EE10FA0BDB93
:10774000EBB200EE903ADFED527AF8EE600A20EEEE
:10775000270A204610F0CEFE07F5405A96F8782208
:10776000DAF878049FED4B0A036807F5BB489B6A7B
:1077700008F1480822B307F5BB4122463831984743
:1077800007F50052B2F93E32002B1CDD07EE903AAD
:1077900096ED977AF8EEE77AB4EEE77AF1EE10FA22
:1077A00011DD07F5BB4122463831404610F098FD07
:1077B000F0B90025284608B0BDEC028BBDE8F08783
:1077C00022464146DBE7B9F1000F1CD1002D3CD128
:1077D000B2F93C32DAF87804D6ED940A00EE103AA9
:1077E0000368B8EEC00A1B6A9847B0EE408A0EE004
:1077F000002DDED106F6B85406F6C85696E80F00FE
:1078000084E80F00D6E707EE909AB8EE678A214623
:10781000404610F0F9FDB4EEC08AF1EE10FA17DB25
:10782000B6F8283303932146404610F0EDFDBCEE38
:10783000C00A07F54950039B174A8DED000A06213F
:1078400010304EF04FFC0125B4E79FED128ADEE7C1
:1078500007F5BB4122463831404610F041FD054650
:107860000028A6D0B6F8283303932146404610F0EE
:10787000CBFDBCEEC00A07F54950039B074A8DEDCE
:10788000000A062110304EF02DFC93E70000003472
:10789000E02E654200000000D4850C08F2850C083B
:1078A00070B500F5005500F5A046B5F94012002965
:1078B000ACBF01234FF0FF330029B8BF494286F81F
:1078C000903D89B2044604F0B3FAB5F93C3296ED26
:1078D000977A002BCABF07EE903ADFED0E7AF8EEEA
:1078E000E77AFCEEE77AF8EE677AB4EEE77AF1EE43
:1078F00010FA08D804F549501030074A06214EF016
:10790000F1FB012070BD204604F0AEF90028F1D152
:10791000F8E700BF0000000010860C082DE9F041D8
:1079200000F5BB4700F5BB453837583504462946B6
:10793000384610F031FB04F5A04604F5405830B34A
:10794000D6F834124B1C22D0D8F8780403681B6B8D
:107950009847D6F8A83D012B47D0D6F8A83D022B72
:1079600006D12046FEF7BCFCD6F8DC3D984243DD4C
:107970002046FEF7B5FCD6F8DC3DC01A0028B8BF9B
:107980004042B0F5FA7FCCBF0020012035E004F57D
:10799000BB402946483010F037FDDFED197AB4EED0
:1079A000E70AF1EE10FA16D53846294610F0FCFB2E
:1079B0009FED147ADFED140AF6EE007AE0EE077A16
:1079C00028469FED120AFDEEE77AF8EEE77A27EEF9
:1079D000800A10F08FFDD8F878049FED0D0A036837
:1079E0002A469B6A39469847B3E72046FEF778FC5B
:1079F000D6F8DC3D9842B0DB0120BDE8F08100BF45
:107A000000004843A00CB345000096430AD7233C2E
:107A100000000000F7B5374FD1ED026AD7F8CC3D32
:107A20009FED357A07EE903AF8EEE77A0546D7EE05
:107A3000876A0E46F5EEC06AF1EE10FA08DD55F0E1
:107A40000FFA2E4A06214EF04DFB012003B0F0BD87
:107A5000D1ED037A97ED956AF5EEC07AF1EE10FA62
:107A600013DDF4EEC67AF1EE10FA0ED555F0F8F902
:107A70000446D7F85402F8F747FD214ACDE9000142
:107A8000062120464EF02EFBDFE7DFED1E7A337C29
:107A9000B4EEE76AF1EE10FA54BFB0EE677AB0EEDA
:107AA000467A0BB90020D1E7B5EEC06AF1EE10FAC4
:107AB0000CDC86EE876A03EB830307EE903AF8EE60
:107AC000E77AF4EEC67AF1EE10FAEBD52C7C002CB6
:107AD000E8D17DF027FA6B69C01A337C4FF47A72D3
:107AE00053439842DED901232B747DF01BFA686161
:107AF0002046ABE7987C00200AD7233C28860C0858
:107B000039860C080AD723BC38B5054676F074FDD3
:107B100075F0BAFA044640B97DF004FAEB68C01A71
:107B2000AB68984284BFAC600124204638BD000099
:107B300038B504460D467DF0F5F904F5A0439FEDF8
:107B4000077AC3F8AC0DD5ED027A67EE877AFDEEC1
:107B5000E77A17EE902AC3F8A82D38BD00007A44C2
:107B600010B504467DF0DEF904F5A043D3F8AC2D42
:107B7000801AD3F8A82D90424FF0000084BFC3F8BC
:107B8000A80D012010BD000000F5A04393ED977AE9
:107B9000D3F8A82D22EAE27207EE902AF8EEE77AEF
:107BA0000020B4EEE77AF1EE10FA44BFC3F8A80D56
:107BB0000120704710B500F5005300F5A040B3F95F
:107BC0000E32002BB4BF4FF0FF33012380F8903DFD
:107BD00000F6D85400F6C8500FC884E80F0010BD56
:107BE00038B504462DED028BF0EE408AB0EE608A87
:107BF00009B301295ED0B5EEC08AF1EE10FA69DD55
:107C0000DFED357AB4EEE78AF1EE10FA62D8FCEED9
:107C1000C87A04F5495017EE903A304A06211030E0
:107C20004EF060FAFDEEC87A04F5005417EE903A73
:107C300084F8DB313CE0F8EE000A20F0B9FF40B1F7
:107C400004F580444FF0FF33C4F8743CBDEC028B64
:107C500038BD04F50053B3F9E42107EE902AF8EE9D
:107C6000E77AF4EEE87AF1EE10FAC4D8B3F9E63127
:107C700007EE903AF8EEE77AF4EEE87AF1EE10FAD1
:107C8000B9DBDFED157A68EEA77A04F58043FDEEE7
:107C9000E77A04F5495017EE902AFCEEE87AC3F82B
:107CA000742C062117EE903A0D4A10304EF01AFA55
:107CB0000120CBE7FCEEC07A00F5495017EE903A70
:107CC000084A0621103004F500544EF00BFAC4EDBA
:107CD0007C8AEDE70020B9E70000C8427F860C08E7
:107CE00058860C086C860C08D1F80D3000EE903ADE
:107CF000D1F80930097A00EE103AFFF771BF0000A1
:107D000070B58B88012B04460D4611D100F5907695
:107D10003046F9F707FF02280AD994F84012B02339
:107D200003FB016120467431BDE87040FFF7B6B92E
:107D300009F076FF05F10801BDE8704009F0BEBB0F
:107D4000F0B500F5A04600279F4B86F87D7289B0FC
:107D5000044608460D4683F8F17D23F0CBFF40B37F
:107D6000012386F8743204F54053D3F8780403688D
:107D7000DB6B984786F87B72C6F8947D03A80FF0FA
:107D8000E1FFB6F828134FF6FF73994208BF394652
:107D9000013104F5A54001AA89B26C3025F0B6FF87
:107DA00028B1BDF80600A0F115035842584186F8E5
:107DB00075026B885D2B00F0FF8032D81F2B29D80D
:107DC0000F2B01D800202AE0103B0F2BFAD801A27C
:107DD00052F823F0C77E0108DD7E0108E77E010826
:107DE000F17E0108057F0108D37E0108B57E0108F8
:107DF000C57D0108C57D0108C57D0108C57D010857
:107E0000C57D0108C57D0108C57D0108157F0108F4
:107E1000FB7E0108532BD5D1012086F87B0209B0E7
:107E2000F0BDBD2B18D8BB2B4BD8B22B7CD00CD8B7
:107E3000702B74D0722BC5D1D5ED027AFDEEE77AA6
:107E400017EE903AC6F8A83D3BE0B32BBAD12946CD
:107E50002046FFF755FF34E0C33B9AB2112AB1D850
:107E6000112BAFD801A252F823F000BF637F0108A5
:107E7000C57D0108637F0108C57D0108C57D010836
:107E8000C57D0108637F0108C57D0108C57D010826
:107E9000C57D01089B7F0108C57D0108C57D0108DE
:107EA000C57D0108C57D0108337F0108C57D010836
:107EB000537F0108002386F8B13229462046FFF798
:107EC0005DF90120ABE705F108012046FEF7CAFF86
:107ED000F7E729462046FFF799F9F2E729462046B9
:107EE000FFF7DCF9EDE729462046FFF7F1F9E8E76F
:107EF00029462046FFF726FAE3E729462046FFF702
:107F0000A9FADEE704F5974129227031204606F0F0
:107F10003BF8D6E729462046FFF738FAD1E729464D
:107F20002046FFF705FECCE729462046FFF7DCFE9A
:107F3000C7E7AB88012BC4D803F0010386F876327B
:107F400004F54950AB88214A062110304EF0CAF89A
:107F5000B7E7A988003918BF0121204600F098FB37
:107F6000AFE7EB6896F8C91E04F5BC44503473B90A
:107F70002B6963B96B6953B920465AF043F804285A
:107F80009FD196F8C91E20465AF046F899E705F1A8
:107F9000080220465AF07EF993E704F5BC4095EDBF
:107FA000041AD5ED020A95ED030A96F8C91E0022BF
:107FB00050305AF053F884E704F59740294658307A
:107FC000FFF766FA7DE700BF987C002090860C08DA
:107FD00000F5804200F59743D2F8442C58339A427A
:107FE00001D1FFF7ADBE01207047000010B500F5CC
:107FF000804200F59743D2F8442C58339A42044605
:108000000ED100F597410822703105F0BDFF04F54F
:108010004950044ABDE81040062110304EF062B8C5
:1080200010BD00BFA0860C08F0B506468FB009ADA4
:1080300006F5A04428460F460FF084FEB4F8283316
:108040004FF6FF72934208BF0023013306F5A540A7
:1080500007AA99B26C3025F059FEA0B117B10023E0
:10806000C4F88C3D95E80F0001AE86E80F00D4F807
:10807000E43D009304F6D85494E80E00034802F05F
:1080800037FD0FB0F0BD0120FBE700BF9078002066
:1080900070B5064606F5A045002103F0C9FED5F8E7
:1080A000944D7CB9304603F0DFFD10B90024204622
:1080B00070BDD5F88C3D012BF8DD7CF033FFC5F8A1
:1080C000940DF4E7D5F8A81D61B17CF02BFFD5F82D
:1080D000943DC01AD5F8A03D9842E7D90023C5F8D1
:1080E000A83D01213046FFF79FFF04460028DDD060
:1080F00006F54950044A062110304DF0F3FF0023E5
:1081000085F87D32D3E700BFC8860C0870B50A46F3
:108110008B88190A137E0546DB0748BF01EB8101F6
:1081200005F5A04448BF4900002603F081FE84F80D
:108130007D62284603F098FD10B90024204670BDEA
:10814000D4F8A81D51B1D4F88C3DD4F8882D9342B1
:10815000F3DD012BF1DDC4F8A86D01212846FFF7FE
:1081600063FF04460028E8D005F54950024A06217D
:1081700010304DF0B7FFE1E7E0860C0838B5054652
:1081800005F5A044898803F053FED4F8A83D83BBCD
:10819000D4F88C3D002BB8BF5B42012B02DC0024DD
:1081A000204638BD94F8912D94F8923D72B9002B79
:1081B000F5D005F54950D4F8CC2D6423062192FB67
:1081C000F3F310300C4A4DF08DFF01E0002BF0D19D
:1081D0000121C4F8A81D2846FFF726FF0446002801
:1081E000DDD005F54950054A062110304DF07AFFE3
:1081F000D6E70021EFE700BFF8860C0816870C08C9
:108200002DE9F0474B881F2B8AB004460A4631D827
:108210000F2B07D804F54950954A042110304DF032
:1082200061FF88E0A3F110010F29F3D801A050F8F5
:1082300021F000BF47830108098401081584010863
:10824000238401083D840108558301083B8301080C
:10825000158201081582010815820108158201089E
:108260001582010815820108158201084984010858
:108270002F840108702B00F0F5800CD8532B00F0F0
:10828000E9805D2BC6D100F5974058300AB0BDE8B3
:10829000F047FFF739BCB32B08D8B12B4BD8722B62
:1082A000B8D10AB0BDE8F047FFF76EBCD42B3BD87D
:1082B000BB2BAFD9A3F1BC02182AABD801A151F84E
:1082C00022F000BF378301083783010815820108B7
:1082D000158201081582010815820108158201081E
:1082E00037830108158201083783010815820108C8
:1082F00015820108158201083783010815820108DB
:1083000015820108158201083783010837830108A7
:108310003783010815820108158201083783010897
:108320001582010837830108DF2B04D040F6B832EC
:1083300093427FF46FAF01202FE020460AB0BDE8E2
:10834000F047FFF7DBB8114620460AB0BDE8F0471A
:10835000FFF7C8B904F5A04504F5B946D5F8C83209
:1083600004F5BB4704F5BB4804F5BB49072B06F1F0
:10837000200607F1380708F1580809F148090FD11C
:1083800004F5A54440340194D5F8443200934246A4
:108390004B46394630467AF02FFD0AB0BDE8F087EB
:1083A00000230DF1270133488DF82730FEF7EEFC4E
:1083B000D5EDA07AD5ED950A95ED981AD5F864A279
:1083C000CDED060A30EE670A04F5BD4054308DED60
:1083D000070A8DED051A74F04DFE0546204600F0A3
:1083E000A1FE9DF827309DED051ADDED060A9DEDF5
:1083F000070ACDE90203CDE900A54B4642463946BE
:1084000030467AF04FFCC8E72046918803F010FD13
:108410000020C2E7114620460AB0BDE8F047FFF74A
:1084200075BE20460AB0BDE8F047FFF731BE1146E1
:1084300020460AB0BDE8F047FFF7A0BE20460AB0CC
:10844000BDE8F047FFF72CBA20460AB0BDE8F04778
:10845000FFF764BA00F5974058300AB0BDE8F0471E
:10846000FFF7D8BA0AB0BDE8F047FFF779BB00BF05
:1084700030870C08982C002070B500F5804200F57C
:108480009743D2F8442C58339A4205460E4602D000
:108490000024204670BDFFF7B3FE04460028F7D045
:1084A00005F549503188103052F00AF8F1E7000024
:1084B00021F04003152B04D0A1F15E03584258412E
:1084C0007047012070470000102945D8DFE801F00F
:1084D000090D1115191D212529442D313540393932
:1084E0003C0000F598401430704700F596406C3021
:1084F000704700F596407430704700F596407C3028
:10850000704700F597400430704700F597402C30D5
:10851000704700F597403430704700F597403C3085
:10852000704700F597405030704700F5974058303D
:10853000704700F597407030704700F597407830ED
:10854000704700F59840704700F598400C30704730
:1085500000F598401C3070470020704700290DDB63
:10856000074890F8B02ACBB29A4207D3D0F8AC3A79
:108570000122595CA0F5005005F0E2BD704700BF34
:10858000984C00202DE9F34100F5005300F54955C2
:1085900093F8803A03F0010603F0020803F00407A1
:1085A0005B07044605F1100535D01F4A0621284611
:1085B0004DF098FD26B104F53750043076F02AFED0
:1085C000B8F1000F04D004F53C501C3076F09EFB4F
:1085D00027B104F54150343077F046FA04F5A04451
:1085E000012384F8793F114A114B1249B8F1000F69
:1085F00008BF1A46002F08BF1946CDE900210E4AD0
:108600000621002E18BF134628460C4A4DF06AFD7D
:1086100002B0BDE8F0810A4A0621284602B0BDE852
:10862000F0414DF05FBD00BF5D870C0852870C081C
:108630004C5E0D0859870C084C870C086E870C0897
:1086400080870C0810B5044600F53750043076F0EA
:108650000DFE04F53C501C3076F084FB04F54150CF
:10866000343077F03BFA04F5A04393F8792F5AB1F0
:10867000002283F8792F04F54950044ABDE81040E0
:10868000062110304DF02EBD10BD00BFA0870C0894
:1086900009B1FFF777BFFFF7D5BF000000F58043B2
:1086A0000A4AD3F8441C91420DD093F8513C43B987
:1086B00000F597425832914203D100F5A04090F85E
:1086C0007632184670470023FBE700BFAC780020E5
:1086D00010B504467CF026FC054BD3F8643CC01A68
:1086E000642804D82046BDE8104056F025B810BDD7
:1086F000986C002010B500F52954D4ED0C7AF5EEF5
:10870000C07AF1EE10FA8AB04FF0000304F13004A1
:1087100045D907930893099306AB019300F58E5052
:1087200007AB009303AA05AB04A9083008F04CFF7F
:1087300030B3DDED080A9DED070AA3F037FBDDED50
:10874000090AA3F033FBD4ED007A9DED047A77EEAD
:10875000A76AB4EEE70AF1EE10FAF4EEC76AACBF0E
:1087600001200020F1EE10FA0CD802309DED037AC2
:10877000F4EEC77AF1EE10FA0CD8003818BF0120D9
:108780000AB010BDF4EEC77AF1EE10FA9CBF0130CA
:10879000C0B2EBE7012894BF00200120F0E70020E1
:1087A000EEE7000010B5074B1A7A4AB901241C7293
:1087B0004AF068FB22461121BDE810404AF01AB980
:1087C00010BD00BF288C002010B5074B1A7A4AB1A3
:1087D00000241C724AF056FB22461121BDE81040CD
:1087E0004AF008B910BD00BF288C0020F0B505463E
:1087F00085B005F58E56684608360FF0A3FA69462F
:10880000304609F013F8A0B13248334C334F74F0BE
:1088100031FC40B105F52953D3ED0C7AF5EEC07A61
:10882000F1EE10FA07D8002328462380FB73FFF7E8
:10883000CBFF05B0F0BD2846FFF75CFFA0B363781F
:108840007BBB23780133DBB2082B237002D1304687
:1088500008F026FF2378092B02D1304608F018FFD4
:108860002378092B1DD94FF4857323804AF00AFB26
:10887000022210214AF0BEF87CF054FB6368C01A53
:1088800047F23053984209D905F54950144A02215C
:1088900010304DF027FC7CF045FB60602846FFF768
:1088A00081FF6378FB73C4E72678002EF9D0013E80
:1088B0006378F6B22670002BF3D0002EF1D16670EB
:1088C0004AF0E0FA324610214AF094F82846FFF7C1
:1088D0007BFFE6E76C8B0020288C0020D58C0020E5
:1088E000B4870C0800F5A040D0F8C832042B14BFA0
:1088F00090F8F4020120704773B500F580450192AD
:10890000A5F85C1C04467CF00DFBC5F8600CD5F89E
:10891000440C03685B68984785F85A0CD5F8440CFA
:1089200003685B6898470F28019A0BD80F2827D84F
:10893000DFE800F01C261C1C1C1C1C1C1C265026DE
:108940000A260A0A18281BD104F50056019296F946
:108950005032ABB1D5F8440C03685B68984785F892
:108960005A0C96F95032019A022B29E0204B93F8C9
:108970007A3F03B304F597412C31204605F004FB00
:10898000D5F8440C95F85A6C03685B68984704F571
:108990004954864204F1100422D0D5F8440C0368EF
:1089A0009B689847134A03460421204602B0BDE85D
:1089B00070404DF097BB04F5005393F95032022BF1
:1089C000D8D0042B0BBF04F5974104F59641343100
:1089D0006C31D2E72046FFF785FF0028D0D1B3E7FE
:1089E000054A0421204602B0BDE870404DF07ABB34
:1089F000987C0020C4870C08E6870C08F0B5044674
:108A000004F5804685B00F46154655F01BFED6F896
:108A1000440CA6F85C7C03685B68984718281ED84D
:108A2000DFE800F00D0D0D0D0D0D0D0D0D1D526843
:108A30000D0D57571D1D1D1D1D1D1D1D0D00314AFE
:108A4000D2F8C812012921D104F5005393F851320C
:108A5000023B012B1AD904F5405383F84C12D6F887
:108A6000440C294A294B052D18BF1346026803936D
:108A70009268904704F5495410340090039B244AAF
:108A8000042120464DF02EFB05B0F0BD92F87A3F50
:108A90003BB104F597412A462C31204605F074FA83
:108AA000DDE704F5005393F95132032B03D120463F
:108AB00003F01AFAD3E7022BEBD0042B15D104F5FF
:108AC00097412A465831E8E72046FFF70BFF002878
:108AD000C5D104F5005393F95132032BE7D0022B93
:108AE000D7D0042BEBD0012BB9D104F597412A46FE
:108AF0007031D2E704F5005393F95132042BAED113
:108B0000DDE700BF987C0020FC870C08336C0C0864
:108B100004880C0870B500F5495504461035124A12
:108B20000421284604F580464DF0DCFA0023A6F81F
:108B30005C3C04F5005393F89831032B12D196F85E
:108B40005A1C3022204605F0FBFAD6F8440C036884
:108B50009B689847054A034606212846BDE87040B1
:108B60004DF0C0BA70BD00BF18880C082F880C08E3
:108B700000F5405310B500220529044600F5495080
:108B800083F84C2200F110000CBF054A054A04216D
:108B900004F580444DF0A6FA0023A4F85C3C10BD17
:108BA00048880C0859880C0830B50B4687B0044635
:108BB000052A18D8DFE802F0172A0350175D00F5E0
:108BC000A043D3F8C832042B20D02C4D95F86D3C2F
:108BD000E3B12B49A1F6DC2025F06AFC28B1294B32
:108BE000012283F8F42207B030BD2549A1F6DC202C
:108BF00025F05EFF50B104F5974104225831A5F5E8
:108C0000804007B0BDE8304005F0BEB904F5A04390
:108C1000D3F8C832042BE6D004F5005393F91B3285
:108C2000022B0AD1154B93F86D3C33B11449A1F6D0
:108C3000DC2025F03DFC0028D1D104F59741042229
:108C40007031204605F0A0F904F507501B3007B03D
:108C5000BDE8304041F058BA0B4A112101A87BF021
:108C600023FA04F5BA4001AA01212C3076F0E8FF7E
:108C7000B9E707B0BDE8304003F036B9986C002082
:108C8000608A0020987C002074880C0870B52DED57
:108C9000048B04467CF03AF94F4BB4F8BE101A88A6
:108CA0004E4E8A4205464E4A06D019800023306057
:108CB0001370BDEC048B70BD33684A49C31A8B42F4
:108CC00076D90123137055F0BDFD55F075FC356064
:108CD00055F0B8FD55F070FC04F5405393F84B3255
:108CE00023B104F5BA402C3076F0FEFE55F08CFC32
:108CF0000428DED955F0A6FC0021204603F01EFC16
:108D000000212046F0EE409A03F022FC012120468B
:108D1000B0EE409A03F0DCFD00212046B0EE408A20
:108D200003F020FC04F5BD405430F0EE408A74F0AE
:108D3000ABF9DFED2D7A0028B0EE690A4FF00400A0
:108D400008BFB0EE678A57F073F9B0EE490A1320F6
:108D500057F06EF9B0EE680A152057F069F904F57E
:108D6000BA45B0EE680A1A2057F062F92C35462051
:108D7000B0EE480A57F05CF9284676F043FF08BB8E
:108D80000121084657F056FC9FED170A022057F0C4
:108D90004FF99FED150A032057F04AF9204603F0DA
:108DA000B5FFBDEC048B2046BDE8704004F0CABEA0
:108DB0001278002A3FF47DAF44F6206293427FF69A
:108DC00078AF80E72846FDF717F804F5A04393F93C
:108DD000363D2B2BD4D06CE7348C0020388C00200F
:108DE000368C0020400D03000000000000F580429A
:108DF00000F59743D2F8442C58339A4204D100F539
:108E0000A04090F8F402E8B10F4B93F8980103F5F5
:108E10004053A0F12702012A93F8883F0FD92C284C
:108E200009D00A2809D0A0F13102504250410A2B42
:108E300018BF002070470120F9E7012070470A3B66
:108E400058425841704700BF984C002008B500F5C3
:108E5000005393F8802042B193F8BC302BB1FFF758
:108E6000C5FF80F00100C0B208BD0120FCE7000092
:108E70002DE9F04700F50055DFF8A4A295F8BC9065
:108E8000044600F5BD408AB0543074F0F3F8DAF8C7
:108E9000C832042B06464CD000284AD0BAF82A1310
:108EA000AAF5A040FFF704FB014620B19AF8F012A2
:108EB0004B1E5942594104F50258404663F0F0FEFA
:108EC0009AF8883F0A2B074603D1A6BB00238AF8ED
:108ED000883F95F88030002B38D195F986308B4D3E
:108EE000012B03D0063BDBB2012B11D895F898314A
:108EF0000A2B0DD104F58046D6F8440C03681B6A92
:108F0000984728B1D6F8481C2B22204605F03CF89B
:108F10009AF8883F0A2B04BF37238AF8883F95F8D0
:108F200098310A2B02D1372385F898310AB0BDE871
:108F3000F0870121BFE740EA0903DBB2002BC8D16B
:108F4000734800F0EFF80028C0D0C2E7002EEDD043
:108F500004F5B940203079F01BFE0028E6D1204608
:108F6000FFF744FF0028E1D1002F00F0BD806949E0
:108F70003A46404663F06CFA95F98690B9F1010FD4
:108F800006D040F38580A9F10603DBB2012B7FD820
:108F90005FFA89F9B9F1010F4ED104F5804204F569
:108FA0009743D2F8442C58339A4209D104F5A04390
:108FB00093F8F43223B195F81B32013B012BB5D95C
:108FC00004F597410A227031204606AE04F0DCFF1A
:108FD00030460EF0B7FE95F999208ABBB9F1010F22
:108FE0002ED004F5A049B5F99A30D9F8B41DDFEDBB
:108FF0004A5AD1ED017A002BF8EEE77A51DD07EEFF
:10900000103AF8EEC76AE6EEA57A3046FDEEE77A4A
:1090100017EE901A0EF09CFE00234046CDE9043373
:1090200063F0DAFE04A964F037FC002856D0049BF4
:109030000893059B099316E00A2204F59841C3E7BB
:109040002046FCF751FF07EE900AE84604F5BB42C4
:10905000483221464046B8EEE70AFEF785F898E820
:109060000F0086E80F0095F98630012B10D03146AD
:109070002046FDF7CBFB31462046FDF75FFF95F913
:109080008630072B04D104F54054012384F84A327A
:1090900049F0F8FE3A4609210AB0BDE8F04749F028
:1090A000A9BCD5ED226A95ED255A95ED237A35EECA
:1090B000076A36EEC57AB4EEC67AF1EE10FA89BFC9
:1090C00037EE067A95ED9F7A27EE257AF6EE006A5E
:1090D00094BFE7EE257AE7EE267A96E7D9F8B43D15
:1090E0009A680892DB68A5E7B9F1000F3FF41EAF5C
:1090F00095F8BC30002B7FF419AF04F54950074AAE
:10910000052110304CF0EEFFC2E700BF984C002064
:10911000982C002080880C080000C84289880C0820
:10912000987C002010B5044600F5BD40543073F023
:10913000ABFF04F5A04494EDB37A48B1DFED067AB5
:10914000B4EEE77AF1EE10FAACBF0120002010BDBA
:10915000DFED027AF4E700BFCDCCCC3D6666663F1A
:1091600000F58043D3F8441C00F598431C33994222
:1091700004D100F5A04393F8C0229AB900F59743B3
:109180005833994210D100F5A04393F8C0224AB158
:10919000D3F8C822032A07D1B3F82A23A2F1160371
:1091A0005A425A41104670470022FBE72DE9F84F1A
:1091B00000F5804200F59743D2F8442C58339A4288
:1091C000054600F5A04704D100F5005898F9F431A0
:1091D00033B90023C7F8B43287F8B132BDE8F88F4D
:1091E0007BF0A0FED7F86842814634B1041B40F6FC
:1091F000C3139C4294BF002401242846FFF792FF2A
:10920000834620B1002487F8B04200263FE005F5F0
:10921000BD40543073F02EFF82460028F2D005F591
:10922000B9462036304679F0B3FC002840D097F894
:10923000B062C6BB44B305F5805141F27072D1F8FB
:10924000C033002BB8BF5B42934206DCD1F8C43375
:10925000002BB8BF5B42934228DD05F5A64105F51A
:10926000BB40303148300FF0CFF8DFED467AC7F819
:10927000B492B4EEE70AF1EE10FA4FF000034CBFDF
:1092800001260026C7F8B832012387F8B03205F569
:109290009070F8F747FC022833D9002C46D1002300
:1092A000C7F8B4329AE75C465E46EDE73446EBE732
:1092B000304679F055FC064638B1002CA5D04FF465
:1092C000FA73C7F8B83254469FE7D7F8C832012B73
:1092D00003D0032B0DD03446D9E7D8EDA57AF5EEAF
:1092E000C07AF1EE10FAF6DD97F8C032002BF2D119
:1092F000E5E72846FFF734FF0028ECD1002CDED14B
:10930000C5E705F5F65A05F5005B0AF1080A9BF872
:109310001610504606F050FB0028C0D09BF81610DF
:10932000504606F041FC0028B7D1B8E7D7F8B43270
:1093300013B9C7F8B49251E7D7F8B822A9EB0303E1
:109340009342FFF44BAF97F8B132002B7FF446AF56
:10935000012287F8B12298F8F431DB0705D505F52D
:10936000BD400C215430F8F713FB05F5495010307F
:109370002EB1054A0221BDE8F84F4CF0B3BE034AB6
:109380003146F8E700009642A0880C08B6880C0821
:109390002DE9F04F2DED028B054685B0002305F534
:1093A000005803937BF0BEFDD8ED7C7AF5EEC07AD1
:1093B000F1EE10FAC4BF9FEDBD7A67EE877A05F52E
:1093C000907BC8BFFCEEE77A07465846CCBF17EE45
:1093D000906A9626F8F7A6FB022840F2FC8095F8E2
:1093E00040329FEDB37AB02202FB0353D3ED697A8A
:1093F00067EE877AFCEEE77A17EE903A9E428CBFD2
:1094000000260126B8F9E431022BB8BF022307EE8B
:10941000903A05F58E50B8EEE78A03A9F6EE087A81
:10942000083028EE278A08F0DFF9044640B1DDED68
:10943000037AF4EEC87AF1EE10FAACBF01240024EE
:109440005846F8F76FFB05F5BD49012809F15409A5
:1094500005F5A04A16D8484673F00CFE90B18CB9B9
:109460009AEDB37ADFED937AB4EEE77AF1EE10FA83
:1094700008DDDDED037AF4EEC87AF1EE10FAACBF48
:1094800001240024484673F0F5FD0090002800F008
:10949000FA8095F8402205EB0212D2F8782172B1D9
:1094A00058460192F8F73EFB012800F29680019A97
:1094B00041F28731BA1A8A428CBF00220122DAF8BF
:1094C000641201B11AB9002C40F08980344605F5C8
:1094D000804105F59742D1F8441C583291421AD187
:1094E00098F91C22002A40F0828000228AF8B222D9
:1094F000DAF8C822042A00F0A880072A00F0B98010
:10950000032A08D12846FFF72BFE20B100248AF851
:10951000B142CAF868429AF8B22202B17CB907EEA9
:10952000904A9FED657ADAEDB36AF8EE677A67EEF6
:10953000877A9FED627AE6EE877ACAEDB37A28469B
:10954000FFF7F0FD0446A8B19AF8D002CAF8647299
:1095500008B9CAF8D47205F5804105F59742D1F8EB
:10956000441C5832914205D1DAF8682202B108B998
:10957000CAF868729AF8F8238AF8D04264F3C302F2
:109580008AF8F8236DF0B4FE21466DF08DFE4C4A4A
:1095900028465471FFF70AFE2846FBF797F934B1C5
:1095A00098F89A211AB97BF0BDFCC8F89C0188F89C
:1095B0009A412846FFF7B6FD002875D1484673F05A
:1095C00063FD80F00100C0B28AF8D80205B0BDEC9E
:1095D000028BBDE8F08F002614E700226FE71EF033
:1095E0007DFE1DF071FE00287FF470AF6FE75242E0
:1095F00007EE902A05F52E62F8EEE77A92ED007AF2
:10960000F4EEC77AF1EE10FA11DDDFED2E7A9AED65
:10961000B37ACAF8BC72B4EEE77A0122F1EE10FA1E
:109620008AF8B2227FF764AFCAEDB37A60E79AF89E
:10963000B222002A3FF45CAFDAF8BC2240F6B8311F
:10964000BA1A8A423FF651AF52E705F5B9402030C9
:1096500079F086FA00283FF45EAF9AED957ADFED57
:10966000197AB4EEE77AF1EE10FA7FF754AF009C66
:1096700051E79AED957AFEEE007AB4EEE77AF1EED4
:1096800010FAF4D447E7DAF8C822002C18BF3446A1
:10969000012A07D005F5B940203079F057FA0028A3
:1096A0003FF439AF002436E700208DE70000B442D4
:1096B0000000C8429A99993E9A99193E9A99593F41
:1096C000D58C0020CDCC4C3E002070470020704748
:1096D000012070470020704701207047034BD3F8EA
:1096E000C802431E58425841704700BF987C002072
:1096F00030B587B002A80EF025FB304879F026FA85
:1097000020B12F492F48FDF793F81FE02B4879F03F
:1097100027FAE8B12C4C04F12405234604F1100289
:10972000A4F11001A4F59470009579F03FFACDE909
:109730000045A4F6C85292ED970A244904F110039B
:10974000A4F11002A4F5947079F0F2F907B030BDDD
:109750001A4802A979F042FA08B102A9D2E71948D9
:1097600002F082FA0028CCD1194C94F8D83D5B075E
:109770001DD4D4F8EC3D002BC3D0114AA2F1200136
:10978000A2F110000EF0ACFD0028BAD1D4ED987A09
:109790000B490C48B7EE000A30EE670AFDF778F87F
:1097A0000C4A084802F12001FCF7FAFBCEE7A4F5C9
:1097B000A040FDF7EBF80028C8D1DAE7388900208F
:1097C000708A0020982C0020608A00204C570020CE
:1097D000987C0020508A002008B50A4890F88D3205
:1097E000013B012B03D8A0F50050F9F7E5F9064835
:1097F000F9F70AF90448F9F7A5F9BDE80840024865
:10980000F9F7BEBC984C0020982C0020124A9042D8
:1098100008B50ED002F1080188420AD002F1100109
:10982000884206D002F13801884202D05C32904270
:1098300006D10A4B93F94502B0FA80F0400908BD01
:1098400003681B6A984728B1054B93F84A0280F0D9
:109850000100F4E70120F2E70C780020984C00208A
:10986000985C0020104A904208B518D002F1080117
:10987000884214D002F11001884210D002F1380160
:1098800088420CD05C32904209D003681B6A98472A
:1098900038B1064B93F84A0280F0010008BD002061
:1098A000FCE70120FAE700BF0C780020985C00205C
:1098B000024A0260024A4260704700BF08890C08F1
:1098C000603E002008B50368DB6D98470648D0F875
:1098D000442C00F53D639A4205D0BDE80840A0F550
:1098E0008040FEF7AFBE08BD986C00202DE9F04126
:1098F000464CA4F585630025C11A4B42C4E9A7551F
:10990000A4F500584B41002284F82052A4F8765266
:1099100084F87A52C4F83C2284F8385284F8B15260
:1099200084F8B252C4F89852C4F8A852C4F84C2231
:1099300088F8EC344368D3F8FC31A4F8703204F6AC
:10994000C85306460FCB04F6B85787E80F0084F8D3
:10995000795284F88852C4F8945D7BF0E3FAA4F558
:109960008057C7F84C0C336830465B6998474FF016
:10997000FF3384F87C0284F87D5288F84C5284F8D6
:10998000F15D84F87B52C7F8743C336830469B6DB8
:1099900098470546002836D0336830469B6B984779
:1099A00084F8C002D8F878040368DB6B9847A7F600
:1099B000186075F097FDA4F5A04002F02BFDA4F50A
:1099C0003E5063F0D3F994F8F432CBB1A4F5A04043
:1099D000FFF7A8FBA0B904F6D46073F055FB78B983
:1099E000D7F8440C03685B6B984748B953F038FAD2
:1099F000074A06214CF076FB04F53B7024F004FE88
:109A00000448F8F74BFB2846BDE8F081987C00201D
:109A1000C8880C08982C002070B503681B6E0E4691
:109A200015469847044650B995F900303BB90548AA
:109A3000054B00683246C06A29461BF0F3FA2046FF
:109A400070BD00BF942C0020EC880C0810B50D4CA4
:109A5000204675F043FB04F5AC7075F0BBF804F5D7
:109A60002C7075F0E9FF084B03F5A042002182F845
:109A7000381203F500530021C2F83C12012283F88A
:109A8000102D10BD5C5A0020982C002008B52DED3B
:109A9000028B1520B0EE408A56F0CAFAB0EE480AA2
:109AA000BDEC028B1A20BDE8084056F0C1BA000098
:109AB00008B5084890F945320121A0F5005033B1AE
:109AC00002F006FFBDE80840462056F0B1BA02F0A9
:109AD00027FFF7E7984C00200420704700487047A4
:109AE0001EC10D08004870471EC10D08037A73B1EE
:109AF000D0ED037AFDEEE77A17EE903A084AC2F805
:109B0000DC32437A3BB10369C2F8E0327047436804
:109B1000D3F8F831F2E74368D3F8FC31F4E700BF3B
:109B2000987C002008B50023038100F114014068EF
:109B300007F070FE012008BD70B56E4E2DED048B50
:109B400006F5994304460121304693ED039ADFED73
:109B50006A9A02F0F3FC0121B0EE408A304602F02E
:109B6000F7FCC8EE297A06F500556068B5F9683249
:109B700004F1140108EE903AF8EEE88AB5F96A3279
:109B800068EEA78AC0EE297A08EE103AB8EEC88AC5
:109B900028EE278A07F03EFE95F96E3263B39FEDFB
:109BA000577AF0EEE87AF4EEC77AF1EE10FA23D5A0
:109BB000227A6368002A55D1012222720022E260D3
:109BC00094ED037ADFED4E7AD3F8F8314D4A4E48E2
:109BD00067EEC77A9FED4D7A67EE877AB0EE490A55
:109BE000FDEEE77A17EE901A0B44C2F8DC32002340
:109BF000012275F003FA08E0002343482372F0EED7
:109C0000490AB0EE680A75F0F5F9042056F010FA2A
:109C100095F96E3243B19FED397AF0EEC87AF4EEE1
:109C2000C77AF1EE10FA28D4002339486372F0EEB7
:109C3000490AB0EE480A74F037FE132056F0F8F9DE
:109C4000B5F96C32002B03DD324E96F98A3063BBD6
:109C500028482021F8F782FC002843D1254802F04B
:109C6000A9FA42E0D3EDC56A96ED467AD4ED037ABF
:109C7000E6EE877AC4ED037AA2E7637A2BB9012373
:109C800063726368D3F8FC3123611E4B2169C3F80A
:109C9000E0126368D3F8FC010023091A1A461C4835
:109CA000B0EE490A74F0E6FEC7E70121A6F5405080
:109CB00002F058FC80EE297AB5F96C32002106F1E9
:109CC000740007EE903AF8EEE77AF0EE490A27EED4
:109CD000870A75F0B1FDBDEC048B2046BDE87040ED
:109CE000FFF7D4BE0348F9F7BFF807EE900AB8EEC5
:109CF000E70AF0E7982C002000A08C450000003413
:109D0000E02E6542987C00205C5A00200000C8428A
:109D1000B45B0020985C00202DE9F04F2DED0C8BFA
:109D2000DFF8A0A39FEDDDDA9FEDDD9A97B00AF58D
:109D3000994300F1140504460121504693ED03BAFE
:109D400002F0FCFB01215046F0EE408A02F000FCDC
:109D500001215046B0EE408A02F004FCDFEDD17ADA
:109D600088EEA77A0AF5005601A8B6F968320AF516
:109D7000A04B0AEE903AF8EEEAAAB6F96A32DFEDA5
:109D8000CA8A6AEE87AA88EE277A0AEE103AB8EEF7
:109D9000CAAAB6F96C329FEDC58A2AEE07AA80EEF0
:109DA000277A09EE903AF8EEE99A6AEE8D7A69EE32
:109DB000879AF0EEEACAF4EEC8CACDED017AB0EEA9
:109DC000CACA6AEE0D7AF1EE10FAF0EEE9BAB4EE14
:109DD000C8CACDED027A58BF4FF0010969EE8D7AFD
:109DE00048BF4FF00009F1EE10FAF4EEC8BA9AED50
:109DF000460ACDED037A54BF4FF001084FF000083A
:109E0000F1EE10FA54BF0127002721F079FA01A9D9
:109E1000284620F095FD284620F084FE284620F0B4
:109E2000FBFD20EE090A284620EE280ABDEEC00AF6
:109E30008BEDB70A20F00AFE20EE090A4FF07E53A0
:109E400020EE280ADFED9A8A0A93BDEEC00ACDED16
:109E50000D8A8BEDB80A0DF1280B59466068CDEDDF
:109E60000C8ACDED0B8A07F0D5FC0021504602F09C
:109E70002FFDB0EEC00AB4EEC80AF1EE10FA16D506
:109E80005046FFF74FF990B9F4EEC8CAF1EE10FA58
:109E90000DD5B4EEC8CAF1EE10FA08D5F4EEC8BA82
:109EA000F1EE10FA44BF9BE80F0085E80F000AA806
:109EB00020F09CFE294612A88DED141A8DED120A91
:109EC000CDED130ACDED151A20F0A2FE0DF1100A0A
:109ED00051460EA88DED101ACDED048ACDED058A00
:109EE000CDED068A8DED0E0ACDED0F0ACDED111ADE
:109EF00020F060FCB6F96832DFED6E7A01EE103AC0
:109F0000B6F96A3209EE103AB6F96C3208EE903AB8
:109F1000B8EEC11AB8EEC99AF8EEE88A21EE271A0F
:109F200029EE279A68EEA78AF4EEC8CAF1EE10FA75
:109F300021EE0D1A29EE0D9A68EE8D8A07D594F858
:109F40002430DFED5B7A002B18BFB0EE671AB4EE59
:109F5000C8CAF1EE10FA07D594F82530DFED547A2F
:109F6000002B18BFB0EE679AF4EEC8BAF1EE10FA03
:109F700007D594F82630DFED4E7A002B18BFF0EEAF
:109F8000678A9AE807000DF11C0B8BE80700F1EED9
:109F9000410AC2209DED070A1EF01CFFC3208DED73
:109FA000070AB0EE491AF1EE490A9DED080A1EF0C3
:109FB00011FFB0EE681AF1EE680A8DED080AC420B0
:109FC0009DED090A1EF006FF514658468DED090A1F
:109FD00021F02CF912A928468DED120ACDED130AB5
:109FE0008DED141A20F0ACFC284620F09BFD06F6FF
:109FF000C853DDED076A93ED007A9FED290AC6EE9E
:10A00000877A06F572665846DDED086ACDED077A67
:10A01000D6ED007A86EEA77ADDED096A8DED087A35
:10A0200086EEA77A8DED097A21F06AF9B9F1000F71
:10A0300001D0CDED07AAB8F1000F01D08DED08AA2F
:10A040000FB1CDED099AF0EE4B0A9DED070A1A48C3
:10A0500074F0D0FF042055F0EBFFF0EE4B0A9DEDBD
:10A06000080A164874F020FC132055F0E1FF002187
:10A07000F0EE4B0A9DED090A114875F0DDFB204614
:10A08000FFF704FD84F8249084F8258084F8267076
:10A0900017B0BDEC0C8BBDE8F08F00BF35FA8E3CDD
:10A0A000E02E654200A08C450000C842000000344C
:10A0B00000000000CDCC4C3E5C5A0020B45B002078
:10A0C0000C5D0020982C002010B50446FFF7F0FC32
:10A0D0000B4B93F96E22022A0DD1B3F96C22002AA0
:10A0E00009DD03F5805393F98A3023B12046BDE89A
:10A0F0001040FFF711BE2046BDE81040FFF71CBD21
:10A10000984C00200A2070470048704795930C082F
:10A110000048704795930C08012070470120704754
:10A12000012070470120704701207047034BD3F88E
:10A13000C802031F58425841704700BF987C002056
:10A14000F8B5194D05F6C8530FCB05F6B85405F60A
:10A15000D85684E80F0086E80F00002705F53B700D
:10A1600085F87C7224F090FC104B1C68E66A33681A
:10A1700030465B689847A8B196F84D3093B1E36AD2
:10A180009B8F7BB152F06CFEE36A094A9B8F0621DC
:10A190004BF0A8FFE36A05F53B70998F24F060FA55
:10A1A000E36A9F870120F8BD987C0020942C002052
:10A1B000D8890C0810B50A4C94F8F032012B0BD159
:10A1C00004F53B7021F00AFDB4F82A33152B03D1B6
:10A1D00004F54A6078F09AFD0023C4F8683210BD97
:10A1E000987C002008B507F01BFD90F87C32DB0757
:10A1F00004D5BDE80840024824F0E2BA08BD00BF1B
:10A20000847F002010B5304C94F8F032012B0ED032
:10A21000A4F582610822A4F5A04003F0B5FE52F037
:10A220001FFEBDE81040294A06214BF05BBFB4F881
:10A230002A33162B05D0152B36D1D4F8C832072B6C
:10A240000AD1234804F022FA214804F057FBBDE864
:10A2500010401F4804F076BAA4F5A040F9F7F0F8D2
:10A26000A4F5A040F8F7F8FFA4F54053D4F8DC12A9
:10A2700093F9AC2264235A4304F54A6078F0A2FCB7
:10A28000C4F8DC0204F54A6078F0DEFD30B1BDE8C8
:10A2900010409FED100A462055F0CABEA4F5A0401C
:10A2A000BDE81040F8F7C8BD1E2B18BF4FF0FF33B4
:10A2B000074818BFC4F83432F9F7C2F80448F8F771
:10A2C000CBFF0348ECE700BF987C0020F0890C0826
:10A2D000982C00200000000010B5144BB3F82A336E
:10A2E000532B04461ED102F0E7FE9FED110A4620D3
:10A2F00055F09EFE9FED0E0A492055F099FE9FED08
:10A300000C0A4A2055F094FE462055F071FF492072
:10A3100055F06EFF4A2055F06BFF2046BDE8104017
:10A32000FFF794BBBDE81040FFF756BA987C0020B9
:10A33000000000000820704700487047888A0C0819
:10A3400000487047948A0C080120704708B50248FD
:10A35000FEF718F9012008BD982C0020014800F0F4
:10A3600057B900BF4478002010B50446FFF734FA0F
:10A370002046BDE81040FFF79BBB0000012070475E
:10A3800000487047088B0C0800487047108B0C0879
:10A39000012070470120704710B5054B03F6D854D3
:10A3A00003F6C8530FCB84E80F00012010BD00BF97
:10A3B000987C002008B50B4800F5A04200F500533A
:10A3C0000321D3F8A43A93FBF1F3C2F8DC32F8F797
:10A3D000A3FF0448F8F740FFBDE808400148F8F73C
:10A3E0002BBD00BF982C0020072070470048704705
:10A3F000F06D0C0800487047848B0C0801207047F2
:10A4000001207047012070477047000008B5002305
:10A41000037203610248FCF7C7F9012008BD00BFC1
:10A42000982C002010B5184CD4F88C3AB3F90830A9
:10A4300023B9D4F8983AB3F90830E3B10023037292
:10A440000361D4F88C0A54F0EDFA04F6A423D3ED9A
:10A45000007A0E48F8EEE77A27EE800ABDEEC00AD1
:10A4600080EDB70AA0F5A040F8F756FFBDE8104010
:10A47000074801F017BB037A002BE2D0A4F5005087
:10A48000F8F7DEFFF2E700BF984C0020987C002030
:10A49000982C002070B54E4DDFED4E7A95F8403285
:10A4A0009FED4D7A2DED048BB02606FB035393ED03
:10A4B0006A8A9FED4A9A28EE278A05F58053BDEEF9
:10A4C000C88A93EDF50AF8EEC87A044667EE897AF1
:10A4D00097EE870A1EF06AFC237AF0EE408A002B82
:10A4E00062D105F50053D3F88C3AB3F90830002B4C
:10A4F0005AD1284601F05EFE002855D195F8403229
:10A5000095F8681206FB035393F8892100294BD173
:10A51000012A49D993ED697AF0EE087AB4EEE77A28
:10A52000F1EE10FA40DBDFED2E7AB0EEE80AB4EE81
:10A53000E70AF1EE10FA37D5236993B37AF0F2FC0B
:10A540002369C01AB0F5FA7F32D8237A002B3CD0A9
:10A55000244DA5F1200696E80F0085E80F0094ED44
:10A56000038AA5F110013046B8EEC88A0DF04CFF01
:10A5700028EE098ADFED1C0A284670EE200AB0EEAC
:10A58000480A0DF0B7FF194B9FED190AD3F878046C
:10A59000BDEC048B03682A4631469B6ABDE87040D7
:10A5A00018477AF0BFFC20612369002BCDD0C5E7A6
:10A5B000104D84ED038A012323720023236105F1EA
:10A5C00010030FCB85E80F00BFE7BDEC048B70BD17
:10A5D000982C00200000C84235FA8E3C0AD7233C54
:10A5E000DB0FC93F708A002000007A44985C00208D
:10A5F00000000000508A0020052070470048704786
:10A60000F88B0C0800487047088C0C080120704734
:10A6100038B5474D2DED028BD5F88C0A9FED458A54
:10A6200054F000FAD5F8A43A07EE903AF8EEE77A3B
:10A6300005F5405427EE800AA5F50050BDEEC00A8E
:10A6400084EDB70AF8F768FED5F8900A54F0EAF9F5
:10A65000B5EEC00AF1EE10FADABF05F6A823D3ED85
:10A66000007AD5ED7F7A3448CBBF20EE270A20EE62
:10A67000270A20EE080A28EE400ABDEEC00A84ED43
:10A68000B80AF8F719FE95ED7F7AD4F8E00205F6DE
:10A69000A82327EE087AD3ED007A27EE888AFDEE0C
:10A6A000C77A17EE902AFDEEC87A17EE901A1EF0C0
:10A6B00031FCC4F8E0022048FDF7F0FF20B1D4F8E7
:10A6C000E0325B42C4F8E0321C4B93F8583C53B183
:10A6D00095F95032022B06D1002301214620C4E90E
:10A6E000B73355F0FFFF54F0ADF85F2155F052F944
:10A6F000D8B155F01FF9022817D194F87932A3B9CF
:10A7000094ED937AD5EDA77AB4EEE77AF1EE10FAEC
:10A710000BD5012384F87932BDEC028B084A094835
:10A72000BDE8384004214BF0DDBCBDEC028B38BDE8
:10A73000984C00200000C842982C0020986C002003
:10A74000108C0C08E85E002010B50446FFF744F8B2
:10A750002046BDE81040FFF7ABB900000620704767
:10A76000004870478C8C0C08004870479C8C0C0883
:10A770000120704701207047012070470120704779
:10A780007047000008B50248FCF70EF8012008BD2C
:10A79000982C002038B50E4C04F50055D5F88C0ADD
:10A7A00054F040F905F6A422D2ED007AF8EEE77AEB
:10A7B00004F5A04327EE800A2046BDEEC00A83EDD3
:10A7C000B70AF8F7A9FD2046BDE8384001F06AB99C
:10A7D000982C00200F20704700487047108D0C08FF
:10A7E00000487047188D0C08012070470120704701
:10A7F0000120704701207047012070477FB50B4D45
:10A8000005F54053002283F84A2205F5BB4348333F
:10A8100006460FCB6C4684E80F0000232846B36041
:10A820002146FCF78BFB012004B070BD982C002062
:10A8300010B53B4CD4F89832002B2CDD7AF072FB2B
:10A84000D4F89832C01A40F6B733984223D8A4F50A
:10A850004053D4F88C02D3F8A42A51421EF05AFB7C
:10A86000C4F8DC02A4F5A040F8F756FDD4F89C32F9
:10A87000002B14DC2B48F8F7EFFC2B4890F84A32F9
:10A8800093B30121A0F5405002F022F8BDE810403A
:10A89000462055F0CDBB2348F8F7D2FDE6E77AF025
:10A8A00041FBD4F89C32C01A40F6B7339842E1D845
:10A8B0001E4BDFED1F6A93ED7F7AD4F8900203F60A
:10A8C000A823D3ED007A27EE267A67EEA67ABDEEAE
:10A8D000C77AFDEEE77A17EE102A17EE901A1EF0EF
:10A8E00019FBC4F8E002C8E7A0F5805090F9DB310D
:10A8F000012B04DCBDE810400A48F8F79DBAD4F8F3
:10A90000A832002BF6D07AF00DFBD4F8A832C01A8A
:10A9100040F6B7339842EDD894EDA90AB6E700BFE8
:10A92000987C0020982C0020985C0020984C0020F7
:10A930000000C842D0ED027A0348FCEEE77A17EE39
:10A94000903A99B201F074BA982C002084B010B5F6
:10A9500003AC84E80E000B4821466F22FCF736FA60
:10A960009DF80C1011F0040102D120460DF0B4FA4C
:10A9700004482146FCF7E2FABDE81040012004B08B
:10A98000704700BF982C0020B0EEC00AFDEEC07AE0
:10A9900038B54FF6FF7205460C4617EE900A0021B7
:10A9A0001EF0B8FA07EE900A002CF8EEE77A054B95
:10A9B000C5ED027A14BF4FF0FF32012283F8902DCB
:10A9C00038BD00BF987C0020FEF792BE0C20704777
:10A9D000004870478C8D0C08004870470DC10D0869
:10A9E0000120704701207047012070470120704707
:10A9F0000120704708B50C48FDF7DCF80A480B4900
:10AA0000FBF704FF0848F7F789FF40B106484FF409
:10AA10008051F7F7A3FD10B10348FBF7C5FE0248CC
:10AA200000F0BEFD012008BD982C0020708A002097
:10AA300008B50D48F8F704FD0B48F7F76FFF50B164
:10AA400009484FF48051F7F789FD20B1BDE808406F
:10AA5000054801F027B80448F8F7FEFBBDE80840B8
:10AA60000148F8F7E9B900BF982C002008B50A485A
:10AA70004FF48051F7F772FD38B108480022D0F842
:10AA8000E81D00F6D8500DF063F9BDE80840024813
:10AA9000002101F0CDB900BF982C0020987C002047
:10AAA000881A10B51EF05EF9104BD3F88C2D0028D3
:10AAB000B8BF4042002AB8BF524248F6A041B2FB9C
:10AAC000F1F24FF47A7102FB011188420CDC93F829
:10AAD000D82DD20606D503F6D85403F6C8530FCBAB
:10AAE00084E80F00012000E0002010BD987C0020C9
:10AAF00084B070B52DED048B86B00FAD85E80E00E7
:10AB00004E4CDFED4F8A0646D4F8780404F5005425
:10AB100004F6A45393ED000A0368B0EEC00A5B6A22
:10AB20009847B4EEE80AF1EE10FAB0EE408A07DA80
:10AB3000012006B0BDEC048BBDE8704004B0704746
:10AB4000404928460DF06CFB02A8CDED030A8DEDBF
:10AB5000020A20F0C9FA04A88DED040AB0EE480AF2
:10AB6000CDED050A20F0BAF913A928468DED000AAB
:10AB7000CDED010A0DF054FB02A88DED020ACDEDDA
:10AB8000030A20F057FAB4EEE80AF1EE10FACFDB30
:10AB9000B4EEC08AF1EE10FA9FED2B9ADFED2B8A0E
:10ABA000DFED2B9A2BD802A8694620F087F904A87C
:10ABB0008DED040ACDED050A20F0F2F9684620EE8D
:10ABC000098A20F0EDF994F9903D07EE903AF8EEFD
:10ABD000E77A28EE288AA7EEA90A1EF0E7F820EE09
:10ABE000090ABDEEC88A20EE280A18EE101AFDEEFA
:10ABF000C07A304617EE902AFFF752FF99E738EEF9
:10AC0000400A38EE088A80EE080AA1F067FA02A826
:10AC1000B0EE408A20F0C4F994F9903DF0EE007A4D
:10AC2000B0EE697AA8EE677A07EE903AF8EEE77A26
:10AC3000A7EE270A1EF0BAF8C0E700BF985C002014
:10AC400000000034608A0020E02E65420000C84207
:10AC5000DB0FC93F10B504460848F7F75FFE20B97F
:10AC60002046BDE81040FEF743BD04484FF4805134
:10AC7000F7F774FC0028F3D010BD00BF982C00201B
:10AC80000020704700487047008E0C08004870474D
:10AC9000088E0C08002070470020704738B5154C0E
:10ACA00005460021204601F049FC042055F0C0F97A
:10ACB0000021204601F04CFC132055F0B9F9002189
:10ACC000204601F04FFC2846FEF7E0FE2046012119
:10ACD00001F0FEFD462055F0ABF96B6804F5A04489
:10ACE000D3F8F831C4F8DC326B68D3F8FC31C4F81F
:10ACF000E03238BD982C0020FEF7A8BE0B2070472C
:10AD000000487047C3860C08004870477C8E0C08CA
:10AD100001207047012070470120704700207047D4
:10AD200070B50B4E06F5A04505F6C8530FCB05F6DA
:10AD3000B85484E80F003046FBF7D6F80146304699
:10AD4000FCF7C8F9002385F8483E012070BD00BF1C
:10AD5000982C002038B53048F8F772FB2E48F8F7E9
:10AD60007BFA2D48F8F768F82B481021F7F7F6FB27
:10AD7000E0B12A4AD2F8CC3DD2F8DC2D9342D4BFC0
:10AD800000230123254C94F8482E72B973B304F6BE
:10AD9000C8530FCB04F6B85585E80F00A4F5A040C2
:10ADA000FBF7FCFA012384F8483E38BD1C4AB2F98F
:10ADB000741A0029F9DD02F540529FED1A7AD2F893
:10ADC000CC3DD2F8BC2D9B1A07EE903AF8EEE77A0C
:10ADD00067EE877A07EE101AB8EEC77AF4EEC77AF4
:10ADE000F1EE10FACCBF01230023CBE7A4F54053CA
:10ADF000642193F9AC22D4F8DC0212FB01F2D3F8FF
:10AE0000A41A8A42A8BF0A465142C3F8A42A1EF0D7
:10AE100081F8C4F8DC02C8E7982C0020987C002058
:10AE2000984C00200AD7233C38B52B4DB5F9403259
:10AE300083EAE371A1EBE37189B205F5405431B1C6
:10AE4000002BB4BF4FF0FF33012384F8903D23481B
:10AE500000F0EEFF94F87A32F3B995F91B32022B29
:10AE60001BD11F4D95F86D3C9BB11E49A1F6DC200E
:10AE700023F01EFE68B1012384F82533282205F64D
:10AE8000D831A5F5804003F07FF828B9002384F875
:10AE90002533012384F87A3238BD012B0CD10F48B9
:10AEA00000F0E2FE40B10D48FBF732FA0028B8BFCF
:10AEB0004042B0F57A7FD4DB95F91B32042BEBD1FD
:10AEC000074D95F86D3C002BE3D00649A1F6DC2038
:10AED00023F06AFECEE700BF984C0020982C00209B
:10AEE000986C0020608A002002207047004870475C
:10AEF000F08E0C080048704702C10D08024B00227A
:10AF0000C3E9B722704700BF987C002038B5094DCF
:10AF100004462846F7F778FD2846F7F713FE204643
:10AF2000F7F728FE2846F8F72BF92046BDE8384009
:10AF3000FEF7BEBD982C00200D20704700487047DA
:10AF4000688F0C0800487047708F0C08012070470C
:10AF500001207047012070470023C37480F824301B
:10AF6000012070470148002100F062BF982C0020AA
:10AF7000F0B5B54CD4F8D42DD4F8D03D2DED088BD8
:10AF80001343D4F8CC2D134389B005460FD1AF48F5
:10AF9000F8F756FAAD48F8F75FF99FEDAD0A46208D
:10AFA00009B0BDEC088BBDE8F04055F041B806F0A3
:10AFB00037FE90F87C32DB07E9D5B5F90830E97C3B
:10AFC00009EE103AB5F9103008EE903AB8EEC99A89
:10AFD000F8EEE88A002940F0D7809FED9EAA29EE7E
:10AFE0000ABA0122FDEECB7AA4F5A040C4ED917A15
:10AFF000FAF7A6FF686800F57F700790B0EE408A08
:10B000001FF0CEFFDFED947A20EE270A1DF04CFEF4
:10B010000798F0EE409A20F00DF8A4F5A040F0EE6D
:10B0200040AAFEF77FF8002879D104F6C85696E8C2
:10B030000F0005F1140787E80F0096E80F0004F6EB
:10B04000B85787E80F0004F6D85787E80F00D4F800
:10B05000DC3D824807EE903AF8EEE77AF0EE680AB7
:10B0600077EE8B7AB0EE690AFDEEE77A17EE903A4A
:10B07000C4F8DC3D0DF03EFA002384F8B13295F9B6
:10B080001230724803EB830303EB83039B0001211F
:10B09000A4F87232F6F7B2FF94F8C072002F73D1A1
:10B0A0006F4B9FED707AB3F9E43107EE903AF8EE0A
:10B0B000E77A67EE877AF4EEE7AAF1EE10FA63DD3D
:10B0C00051F0CEFE064619EE900AF5F71DFACDE9CD
:10B0D000040118EE900AF5F717FACDE9020119EE0E
:10B0E000100AF5F711FA604ACDE900010621304651
:10B0F0004AF0F8FF79F016FFC4F83072C4F81C0269
:10B1000079F010FF0123C4F82C0229EE8A0AEB74AF
:10B110001DF0F4FDBDEEC00A84ED8D0A34E079F037
:10B1200001FFD4F8D432C01A42F2107398427FF66D
:10B130007CAFF0EE087AF4EEE7AAF1EE10FA7FF7B2
:10B1400074AFBCEEC88A04F6D85718EE103A9BB21A
:10B1500008EE103AB8EEC88A04F6C856B4EEC89A9B
:10B16000F1EE10FA46D851F07BFE404A06214AF033
:10B17000B9FF96E80F0087E80F000123EB74032165
:10B18000A4F5A040F6F73AFF304803F0F9FC28B1E7
:10B190002E480321F6F732FF0023EB74D4F8C832AF
:10B1A000012B40F0B480D4F8CC3DAA699FED29AAC8
:10B1B0009B1A07EE903AD4F834320133F8EEE79A4E
:10B1C0005CD0DFED2B7AE9EE0A7AF4EEE79AF1EE45
:10B1D00010FA0ADA274905F114000DF015F9F4EE1A
:10B1E000C08AF1EE10FA00F2928018480321F6F7B7
:10B1F00005FF8CE051F034FE1F4A06214AF072FF31
:10B2000096E80F0005F1140C8CE80F0096E80F008B
:10B2100087E80F00D4F8DC3D07EE903A39EE488A13
:10B22000F8EEE77AF0EE680AE8EE0A7A3846B0EE11
:10B23000690AFDEEE77A17EE903AC4F8DC3D0DF0AE
:10B2400059F90121E9749BE7987C0020982C002093
:10B25000000000000000C842E02E6542708A002015
:10B26000984C00209A99993EB98F0C08788F0C0859
:10B27000000048C3608A0020948F0C08B5F90A309A
:10B2800007EE903AF8EEE77A05F1140667EE8A7A4F
:10B29000F4EEE79AF1EE10FA53DB434930460CF036
:10B2A00083FFDFED427AB6EE008AA0EE278A96E8A9
:10B2B0000F00BDEEC88A9FED3E0AB8EEC88A04F6BC
:10B2C000D85728EE008A87E80F00F0EE680A394860
:10B2D000B0EE480A0DF00EF9D4F8DC3D07EE903AD6
:10B2E000F8EEE77A28EE0A0AE9EE0A7AFDEEE77A46
:10B2F00017EE903AC4F8DC3D1DF000FDBDEEC00A2B
:10B3000084ED8D0AD4F8C832012B3FF45AAF2A4895
:10B3100003F016FC18B128480321F6F76FFED4F8A5
:10B32000C832012B17D1244803F0B0F9224803F0AA
:10B33000E5FA214809B0BDEC088BBDE8F04003F008
:10B3400001BA194930460DF05FF8F4EEC08AF1EE0B
:10B3500010FAA2D9D6E795F824302BB9174861F036
:10B3600039F9012385F824301348F8F769F81248B1
:10B37000F7F772FF1048F7F75FFD114890F84C326D
:10B380006BB1002380F84C3233220221A0F54050EB
:10B3900009B0BDEC088BBDE8F040FDF72FBB09B04C
:10B3A000BDEC088BF0BD00BF608A0020A00CB34547
:10B3B0000AD7233C708A0020982C0020184D0020CA
:10B3C000985C002010B50446FEF772FA2046054B43
:10B3D00040F8143B0CF0B6FC204603493EF0BEFD9D
:10B3E000204610BD6C900C0804900C080320704798
:10B3F00000487047D0900C0800487047DC900C085B
:10B40000F8B52A4D06460027A5F54050A5F8487224
:10B41000F7F782FF7368A5F58052D3F8F811D2F8D8
:10B42000A43A994205F500541FDBC4F8DC32736876
:10B4300092ED7F7AD3ED7F6A9FED1D6AF8EEE66AA2
:10B4400027EE067AF4EEC76AF1EE10FA16DBBDEECF
:10B45000C77A84EDB87A1748FDF720F920B1D4F8FF
:10B46000E0325B42C4F8E032F8BD5B429942DCDD79
:10B47000012385F84832C4F8DC72D8E702F6A82226
:10B48000D2ED007A67EE867AF4EEE76AF1EE10FA12
:10B4900089BF0123FDEEE77A85F84932002394BF86
:10B4A000C4EDB87AC4F8E032D5E700BF985C00205C
:10B4B0000000C842982C002070B500212DED028BB1
:10B4C00004463448344D01F039F832480021F0EE9A
:10B4D000408A01F03DF895F84832B0EE408AD3B189
:10B4E000B0EE680A042054F0A3FD95F8493293B3F6
:10B4F000B0EE480A132054F09BFD2648002101F0CD
:10B5000031F82046FEF7C2FABDEC028B2046BDE8BA
:10B510007040FEF7CDBA05F50056A5F54050F7F797
:10B5200073FAD6F8DC32002B0CDCD6F8DC32002BB8
:10B53000DBDA042054F090FDB4EEE80AF1EE10FAE4
:10B54000CED4D2E7042054F087FDB4EEE80AF1EE41
:10B5500010FAEADDC4E7114D0E48F7F7F3FAD5F813
:10B56000E032002B0CDCD5F8E032002BC5DA1320DA
:10B5700054F072FDB4EEC80AF1EE10FAB8D4BCE78C
:10B58000132054F069FDB4EEC80AF1EE10FAEADDBA
:10B59000AEE700BF982C0020985C0020987C00202B
:10B5A00000F5A0400023C0F88C3DC0F8883D80F82D
:10B5B000913D80F8923D704700F58043D3F8743C8C
:10B5C000002BCBBF07EE903A00F50050B8EEE70A2B
:10B5D000DFED037ADCBF90ED7A0A20EE270A704790
:10B5E0000000C8422DE9F0412DED028B00F58E5789
:10B5F00084B09FEDC88A0837054603A938468DED0B
:10B60000038A06F0F1F8B0B19FEDC37ADDED037A5D
:10B6100005F5A04367EE877AD3EDBA6A9FEDBF7A4E
:10B62000E6EE877AF4EE487AF1EE10FA48BFF0EED3
:10B63000487AC3EDBA7A2846F7F7C2F805F5804490
:10B64000B0EE408AF0EE000A9FEDB20A1DF09AFCBF
:10B6500004F68C43D3ED007A38EE678A05F5005680
:10B66000E0EE087AC3ED007A94F8583C002B40F0E5
:10B670009380D4F8442C05F5974334339A4205D08F
:10B6800005F597433C339A4240F0868008212846CE
:10B69000F6F764FF804630B1D6ED7A7A9FEDA07A56
:10B6A00067EE877A73E002212846F6F757FF0146D6
:10B6B000002855D0D6F8943A1B8B2846414608EE10
:10B6C000103A01F005F9D6F8940A4369B8EE488AB1
:10B6D000B0EE401A2BB3012B28D0DFED927AF0EEBA
:10B6E000671A96ED7A0A9FED8E7AF4EEC17AF1EE42
:10B6F00010FA20EE070A4FF0640124DBB6F8E421CB
:10B7000012FB01F2B0EE672A07EE902AF0EE400A33
:10B71000B8EEE70A1DF090FABDEEC00A10EE103A3E
:10B72000EBE0DFED807AF1EE481ADAE78DED010A01
:10B7300053F0EAF807EE900ADFED7A1A9DED011A50
:10B74000F8EEE77ACDE7B6F8E63113FB01F300EE49
:10B75000903AB0EE482AF8EEE00AF0EE671AD9E720
:10B76000B6F9E421B6F9E6319B1A07EE903A28467D
:10B77000B8EEE78A01F0ACF8B6F8E431642213FBC6
:10B7800002F307EE903AF8EEE77AE8EE007AFDEE83
:10B79000E77A17EE903AB0E005F5A043D3F8C83247
:10B7A000042B40F0A08005F5B940203077F018FA5E
:10B7B000C4F8700CD4F8440C03689B6B98470028BD
:10B7C0005ED094F8843C002B5AD0D4F8442C05F574
:10B7D00096436C339A4253D0D4F8703C9FED527A22
:10B7E00007EE903AD4F8803CF8EEE77A384627EE38
:10B7F000878A07EE903AF8EEE78A68EE878A06F0C5
:10B80000FFF9C8EE807A04F688439DED037A77EE5F
:10B81000877AB6EE007AB4EEE78AF1EE10FA4CBF02
:10B8200077EEC87ADFED3F7A77EE877A93ED007A8C
:10B83000FDEEE77AF8EEE77AB4EEE77AF1EE10FA89
:10B840000ADD37EE676ADFED396AB4EE666AF1EE5B
:10B8500010FA48BFF0EE477A04F68843C3ED007A49
:10B86000D4F8703CDFED2E6A07EE103AB8EEC77AD6
:10B87000A7EEA67ABDEEC77A17EE103AC4F8703C70
:10B88000D4F8440C03681B6B984740B1B4F97C2C86
:10B89000002AC2BFD4F8703C9B18C4F8703CB6F9BB
:10B8A000E621B6F9E411D4F8700C64235A435943E5
:10B8B0001DF030FBC4F8700CD6F8500B05F52D5573
:10B8C00095ED4A8A06F09CF9C8EE007A04F67844B1
:10B8D0009DED037A77EEC77AC4ED007A04B0BDEC33
:10B8E000028BBDE8F081D4F8442C05F598439A42C8
:10B8F00006D1D4F8743C002B02DDC4F8703C59E743
:10B9000005F5974358339A427FF4C6AE2846FFF7B1
:10B9100053FE01E7CDCCCC3DCDCC4C3ECDCC4C3F05
:10B920000000C842000000000AD7233C9A99993FC2
:10B9300030B500F58E5587B00835002304462846FB
:10B9400003930493059305F021F8002843D003A93D
:10B95000284605F077FF00283DD004F5A75393ED66
:10B96000027ADFED216A8DED017AB0EEC77AD3ED70
:10B97000057AB4EEE67AF1EE10FACDED027A06D54C
:10B98000F0EEE77AF4EEE67AF1EE10FA2AD401A8A6
:10B990001FF0A2FB03A901A81FF0E6FA04F500536B
:10B9A00093ED7C7AB5EEC07AF1EE10FAC4BFDFED0C
:10B9B0000F7A27EEC00A04F58044C6BFA7EE270A17
:10B9C0000123002384F8843CCABFFDEEC07A002323
:10B9D00017EE903A04E004F58044002384F8843C98
:10B9E000C4F8803C07B030BD000000340000C842FD
:10B9F0002DE9F0412DED028B00F5A04607EE901ADF
:10BA0000D6F8943D00F5BB45B8EE678A0446583534
:10BA100000F54057B3BB00F58043D3F8442C00F544
:10BA2000974358339A4203D000F598439A4229D15C
:10BA300096F8783233B304F5BB40294648300CF011
:10BA4000E3FCD7F878040368F0EE408A5B6AB0EE56
:10BA5000480A9847F0EE087A60EE277AF4EEE78A13
:10BA6000F1EE10FA0EDDBDEC028BD7F878049FEDF5
:10BA70000C0A036804F5BB412A469B6ABDE8F04105
:10BA800038311847B0EE480ABDEC028BD7F878047D
:10BA900096F9902D03682946DB6ABDE8F041184706
:10BAA0000000000070B504462DED028B04F5A045A2
:10BAB00079F02CFAD5F8003E474AC31A934206465D
:10BAC00072D907EE903AB8EE670ADFED447A9FED3F
:10BAD000441ADFED440A20EE270A40F295101DF0CB
:10BAE00079F9C5F8006E04F50056DFED3F7AD6F817
:10BAF000903AB3F9083008EE103A96F94232B8EEAF
:10BB0000C88AF0EE408A28EE278A0BB1B1EE488A47
:10BB10009FED367ADFED367AB4EEC78AF1EE10FA91
:10BB200052DA05F6FC53D3ED006AF4EEC76AF1EE83
:10BB300010FAB4EEE78AACBF01230023F1EE10FA4D
:10BB40003FD905F6FC5292ED007AB4EEE77AF1EEB9
:10BB500010FA36D82046FAF727FE96F9433200EE5F
:10BB6000103A06F6683306F53766D6ED000A93ED0F
:10BB7000001AB8EEC00A40F2A710F1EE600A20EEFB
:10BB8000080A1DF027F928EE800ADFED1A8A20EE58
:10BB9000280A2046FDEEC07A05F6FC5517EE901AED
:10BBA000FAF7C0FD85ED008A2046FAF70BFA204629
:10BBB000F7F742F9BDEC028B2046BDE87040F7F77D
:10BBC0004BBB002BC6D1C8E7B4EEE78AF1EE10FA02
:10BBD000C3D90023B5E700BF9F860100BD37863576
:10BBE0009A99193ECDCCCC3D5304693900000034FC
:10BBF000000000B40000C84270B5044600F5A5403E
:10BC00004FF0FF316C3022F0D7F8431C054604F5A5
:10BC1000A04603D1114BC6F8503270BD04F5BB41AC
:10BC200004F5BB40583138300CF0BEFA9FED0C7A69
:10BC3000F6EE007AE0EE077AFDEEE77A17EE900A6C
:10BC4000281A1DF08FF807EE900A9FED067AF8EE9D
:10BC5000E77A67EE877AC6ED947ADEE70000B442B1
:10BC6000A00CB3450AD7233C00F54050D0F8780427
:10BC700003689B6B18470000F7B500F54053054675
:10BC8000D3F8780403681B69984707462846FFF7EE
:10BC9000EBFF05F5A0440646D4F88C0D002862D1D0
:10BCA0003EB1D4F8CC3DC4F8983D3E4BC4F89C3D21
:10BCB0000120C4F8847D1DF055F8D4F88C3D94F92A
:10BCC000902D00FB0230C4F88C0D3EB3002301938D
:10BCD00094F8F03D002B4AD094F89C3C022B46D1BE
:10BCE00005F5A840012201A9043044F03DFA0028DE
:10BCF0003DD0D4F8F43DDFED2C6A07EE903AB8EE73
:10BD0000E77ADDED017AE7EE667AB1EE047AF0EEDD
:10BD1000E77AF4EEC77AF1EE10FA33D494F8913D55
:10BD2000002B3DD1D4F88C3DD4F89C2D002BB8BF0E
:10BD30005B42934234DBD4F8CC1DD4F8983DC4F870
:10BD4000981DCB1A03F2F31340F2E630834202F55A
:10BD5000D2328CBF0023012302F5F07284F8923DA9
:10BD6000C4F89C2D1CE0D4F8843DF81AA1E7D4F85F
:10BD7000E82DD4F8CC3D9B1A03F2F31340F2E632DF
:10BD80009342CBD8012384F8913D002384F8923D5F
:10BD9000D4F88C3D03F5D23303F5F073C4F89C3D21
:10BDA00003B0F0BDE0A501000AD7233C2DE9F04126
:10BDB00000F58048044698F86D3CA3B300F5A04513
:10BDC000D5F8E03D13B9D5F8E43D63B304F5BB46BF
:10BDD00004F5BB47204648365837FBF717F8394675
:10BDE00030460CF011FB04F5BB413A463831304681
:10BDF00085ED970A0CF03EFADFED0C0A85ED980A06
:10BE00007620B7EE001A1CF0E5FF04F52D5320460E
:10BE100083ED710AFFF730FFD8F8440C0368BDE8E2
:10BE2000F041DB6A1847BDE8F08100BF0000000068
:10BE3000012938B5044600F5A04512D800F5005395
:10BE400095F8D82DB3F90E3283EAE371A1EBE371D3
:10BE500089B2012998BF3C21920731D5FF2385F88B
:10BE6000903D07EE901AF8EE677A05F6A453C3EDFD
:10BE7000007A2046FFF7BCFDD5F8943D33BB204641
:10BE8000FFF7F2FE40B995ED987AF7EE007AB4EE3E
:10BE9000E77AF1EE10FA19DD79F044F804F5804301
:10BEA000C5F8940DD3F8440C03681B6A984768B131
:10BEB00004F549500021BDE8384010304EF000BB79
:10BEC000002BB4BF4FF0FF330123C8E738BD00009B
:10BED00010B500F5A744643420465BF0D7FF204638
:10BEE000BDE810405CF042B810B500F5A043044630
:10BEF00093F8F8339A0717D45B0700F549504FF0D1
:10BF000002014CBF094A0A4A10304AF0EBF804F526
:10BF1000A74064305BF08EFF04F528500121BDE896
:10BF200010403C3062F034BB10BD00BF50910C0893
:10BF30006A910C0870B500F5A046054696F9E443F1
:10BF40009CB196F8F833C3F380045B0729D4B6F9A3
:10BF5000EA33002B0BDC2846FFF7C6FF05F5285017
:10BF600001213C3062F014FB0124204670BD2146C3
:10BF7000FAF710F8B6F9EA3307EE903AF8EEE77AF6
:10BF8000B4EEE70AF1EE10FAE5D5D6F86432002BEC
:10BF9000E1D005F54950044A042110304AF0A2F8D6
:10BFA000E3E70024E1E700BF80910C0808B52DED20
:10BFB000028B08EE901A30B3F2B1B0F9083008EEF7
:10BFC000103AB8EEC88AF8EEE88A9FED100ADFED65
:10BFD000100A28EE800ADFED0F8A4FF4D470B7EE16
:10BFE000001A1CF0F7FEC8EE280A1CF04FFE20EEE7
:10BFF000280ABDEC028B08BD52F00AFD07EE900A3C
:10C00000B8EEE78ADFE79FED020AF2E70AD7233CA2
:10C010000000000000A08C4537B500F5005405462F
:10C0200094F96F32002B52D052F00CFC52F000FC0D
:10C03000C4F88C0A52F006FC52F0E6FBC4F8900AF1
:10C0400052F000FC52F0EAFBC4F8940A52F0FAFBFA
:10C0500052F0EEFB41F29411C4F8980AD4F88C0A1D
:10C0600052F03AFCD4F8900A41F2941152F034FCA8
:10C07000D4F8980A41F2941152F02EFC284600F0B0
:10C0800021FC48BBD4F8940A642152F021FC52F000
:10C09000D9FBD02153F07EFCC4F89C0A52F0D2FBAD
:10C0A000D22153F077FCC4F8A00A05F518501430DB
:10C0B0004921019054F0FCF901984A2154F0F8F913
:10C0C0000198462103B0BDE8304054F0F1B952F078
:10C0D000B9FB52F08FFBABE705F5A043D4F8940A07
:10C0E00093F87C3F642173B152F0F2FB6421462047
:10C0F00054F0D6F86421492054F0D2F864214A2043
:10C1000054F0CEF8C3E752F0E7FBEFE710B500F5C7
:10C1100000541E21D4F88C0A52F0E2FBD4F8900AA5
:10C120001E2152F0DDFBD4F8980A1E2152F0D8FBF4
:10C13000D4F8940A1E21BDE8104052F0D1BB000093
:10C1400007B500F0BFFB014658B90190462053F0F7
:10C15000C9FF0199492053F0C5FF01994A2053F0C6
:10C16000C1FF0021042054F08FFA0021132054F065
:10C170008BFA0021462054F087FA0021492054F020
:10C1800083FA00214A2054F07FFA0021152003B0E1
:10C190005DF804EB54F078BA10B5044654F0BAFCDC
:10C1A00054F00AF9204601F0CDFCBDE8104054F0EF
:10C1B000B9BB000038B500F50055044695F96F325B
:10C1C0000BB1002038BD0121F6F7C8F990B104F594
:10C1D0008043D3F8442C04F5984314339A4209D091
:10C1E00004F5964374339A4204D004F5974304331C
:10C1F0009A42E6D12046F6F791FB0028E1D0D5F827
:10C20000983AB3F90800DDE738B52DED028B00F55B
:10C21000804393F8583C002B40F0B9805D4A00F50C
:10C220009843D2F8442C143300F549549A4204F14F
:10C23000100408D0584A0321BDEC028B2046BDE80B
:10C24000384049F04FBF00F500559FED546AD5F8CE
:10C250008C2AB2F90830002BB8BF5B429BB207EEC4
:10C26000903A138B06EE903AF8EEE66AF8EEE77A2B
:10C2700066EE866AF4EEE67AF1EE10FA17DCD5F88F
:10C28000902AB2F90830002BB8BF5B429BB207EE90
:10C29000903A138B07EE103AB8EEC77AF8EEE77AC9
:10C2A00027EE067AF4EEC77AF1EE10FA01DD3C4A89
:10C2B000C1E700F5A6501C301FF030FCDFED397AE5
:10C2C00020EE270AF3EE0E7AB4EEE70AF1EE10FA4A
:10C2D00001DD354AAFE7042054F08EF9132054F005
:10C2E0008BF9152054F088F94D2054F085F94E2033
:10C2F00054F082F94F2054F07FF9502054F07CF92B
:10C30000152053F0A9FE9FED298AB0EEC00AB4EEC5
:10C31000C80AF1EE10FA0BD5102054F06DF9562032
:10C3200054F06AF9112054F067F9572054F064F979
:10C33000032053F0A1FEB0EEC00AB4EEC80AF1EE3D
:10C3400010FA0FD5022053F097FEB0EEC00AB4EEFB
:10C35000C80AF1EE10FA05D5182054F04DF919204D
:10C3600054F04AF9D5F88C0A811D0C303EF0B4FC2B
:10C37000D5F8900A811D0C303EF0AEFCD5F8980A35
:10C38000811D0C303EF0A8FC094A052154E7BDECA4
:10C39000028B38BD986C002094910C08CDCC4C3E9B
:10C3A000B4910C08E02E6542DC910C0800000034CA
:10C3B000F8910C0810B500F5005494F946329BB181
:10C3C000D4F8940A52F09AFAD4F8942AB4F948327C
:10C3D00030B1B2F906009842ACBF0020012010BD78
:10C3E000B2F906008342F7E70120F8E710B50446EA
:10C3F000FFF7E0FF60B104F5804478F093FDD4F8D6
:10C40000643CC01AB0F57A7F94BF0020012010BDB3
:10C410000120FCE770B50546FFF7E8FF05F500547D
:10C4200008B3D4F88C3A9A89DA80D4F8903A9A8989
:10C43000DA80D4F8983A9A89DA80D4F88C3A0026CF
:10C440001E81D4F8903A1E81D4F8983A1E8105F5E1
:10C450008043D3F8440CC3F87C6C03685B6898474E
:10C46000D4F8943A1E8105F5BD40543070F002FEB8
:10C4700080B3002652F0E6F9437A13B952F0E2F99C
:10C48000837A94F94622012A23D106B10BB32846B8
:10C49000FFF7ACFF05F5804494F85E3C38B30133F8
:10C4A000DBB20A2B84F85E3C0CD105F549501F4BDA
:10C4B0001F4A0421103049F015FE1E4A012384F85A
:10C4C000583C937294F85E3C0A2B02D90A2384F8F4
:10C4D0005E3C70BD2846FCF725FE0028C9D152F00D
:10C4E000B1F952F073F9061E18BF0126C2E7002BFE
:10C4F000EFD0013BDBB2032B88BF032384F85E3C03
:10C5000094F85E3C012B09D105F549500A4B084AC5
:10C51000BDE870400421103049F0E4BD002BD8D1B3
:10C52000044A84F8583C9372D3E700BF2FE60D0805
:10C5300008920C08D58C0020EB930C0800F50050F5
:10C540000A4690F9761AD0F88C0AFFF72FBD000042
:10C5500000F500500A4690F9771AD0F8900AFFF7D4
:10C5600025BD000000F500500A4690F9781AD0F871
:10C57000980AFFF71BBD000010B54FF48061044618
:10C58000F5F7ECFF04F5005328B1BDE81040D3F8EF
:10C59000940A52F039BBBDE81040D3F8940A52F027
:10C5A0003DBB0000F8B500F5005300F5A045D3F8F9
:10C5B000983AB3F9087017B9012385F8183F00F5C8
:10C5C000BD445434204670F055FD0646E0B9B7F539
:10C5D0007A6F2BDD78F0A6FCD5F8143F074683B1BF
:10C5E000C31A40F6B73293420DD901223146204694
:10C5F000F5F7A8F9C5F8146F85F8186FC5F80C722F
:10C6000001E0C5F8140FF8BD17F57A6F0EDA78F06F
:10C6100089FCD5F8143F6BB1C01A40F6B733984285
:10C62000F1D9012200212046F5F7B2F90023C5F81F
:10C63000143FE8E7C5F8140FE5E7000070B52DEDED
:10C64000028B044652F0FEF851F0B6FF30B9BDEC53
:10C65000028B2046BDE87040FFF7DCBE04F5804544
:10C6600095F8583C1BB978F05DFCC5F8680C20467D
:10C67000FFF7A0FE18B178F055FCC5F8640C204611
:10C68000FFF7C8FE2046FCF7E1FB04F50056002347
:10C69000C5F87C3C96F94A3263B3D6F8943AB3F9BC
:10C6A0000830322B26DD28B3323B1BB207EE903A1E
:10C6B00004F58E50B8EEE78ADFED207A083028EED8
:10C6C000278A04F09DF838B3B6F9E63196ED7A7A08
:10C6D00007EE903AF8EEE77A77EEC77A27EE888A87
:10C6E000DFED177A28EE278ABDEEC88A18EE103AD9
:10C6F000A5F87C3C2046FFF755FFD5F8440C0368AD
:10C700005B689847BDEC028B014604F5BE402030C3
:10C71000BDE8704054F0F2BD96F9D93196F9DB21AD
:10C720009B1A07EE903AF8EEE77A27EE888ABDEE7C
:10C73000C88A18EE103AA5F87E3CDBE70AD7A33C7E
:10C740000000C84270B500F500540546D4F84C32DC
:10C750000BB9002041E094F9D831002BF9DA00F54B
:10C760008043D3F8440C03685B6898470138172866
:10C7700032D801A353F820F075C80108B1C80108E8
:10C78000D9C70108A7C801089DC8010889C80108C0
:10C790007FC80108D9C70108D9C70108DDC701084A
:10C7A0006BC8010861C8010853C7010893C8010894
:10C7B00093C80108D9C70108D9C70108D9C701081A
:10C7C000D9C70108D9C70108D9C70108D9C70108C5
:10C7D000D9C70108BBC80108012070BD05F5A045F7
:10C7E000B5F82A63162EB4D0D4F84C1211F0020317
:10C7F00001F0010205D0A6F1150CDCF1000343EBBA
:10C800000C0311F0040043EA020303D0A6F11F0455
:10C810006042604143EA000211F0080007D01F2E79
:10C820001AD0A6F1110002288CBF0020012011F0BF
:10C83000100340EA020005D0102E0FD0A6F15202DC
:10C8400053425341034311F4006014BF95F8F412AE
:10C85000014643EA0100C0E70120E8E70123F1E7D0
:10C86000D4F84C02C0F34010B7E7D4F84C02C0F340
:10C870008010B2E7D4F84C02C0F3C010ADE7D4F892
:10C880004C02C0F30020A8E7D4F84C02C0F34020CB
:10C89000A3E7D4F84C02C0F380209EE7D4F84C0202
:10C8A000C0F3003099E7D4F84C02C0F3403094E76D
:10C8B000D4F84C02C0F380308FE7D4F84C02C0F3B8
:10C8C000C0308AE700F5005090F8D801C0097047E1
:10C8D00038B504460D4651F0B5FF0368DB6898474C
:10C8E000C8B104F50053D3F8940A6DB152F090F832
:10C8F00007EE900AB8EEE70A04F5A04494F87B3FEF
:10C900000BB1B1EE400A38BDB0F9083000EE103A74
:10C91000B8EEC00AF0E79FED010AF4E7000000005E
:10C9200038B52DED028B04460D4651F08BFF0368A0
:10C93000DB68984700283FD0214BD3F8943A5B69D5
:10C94000012B07D0BDEC028B29462046BDE83840BC
:10C95000FFF7BEBF4FF480612046F5F7FFFD0028CA
:10C96000F0D004F50053DFED177AD3F8940A93F969
:10C97000DB31028B08EE903A00EE102AF8EEE88ADE
:10C98000B8EEC08A68EEA78A52F04CF8B6EE001AEC
:10C99000A0EE011A04F5A044DFED0B0AB0EE680A20
:10C9A0001CF046FA94F87B3F28EE000A0BB1B1EE7A
:10C9B000400ABDEC028B38BD9FED030AF9E700BFCA
:10C9C000984C00200AD7233C0000000073B500F506
:10C9D000A045044695F89C3C022B00F6F83612D18F
:10C9E00000F5A840012201A9043043F0BDFB50B17D
:10C9F000019BC6F89C3230463EF05CFD2046FAF7BB
:10CA000059F802B070BDD5F8C832042B05D12046C4
:10CA1000F9F728FD8DED010AEAE705F604652B68B4
:10CA20000193E5E770B500F580460446D6F8440C5E
:10CA300003689B6B0D46984748B9D4ED460A9FEDB5
:10CA40001C0A64212846BDE8704053F0E7BBD6F8C5
:10CA5000440C04F5974104F500525831884292F88D
:10CA6000DA3192F9A4221FD104F5A04191F87402A1
:10CA700050B94AB1D3B204F5A041D1F8C812013976
:10CA8000012998BFD3B207E091F91C0D60B1D1F82C
:10CA9000C812042908D1C3B207EE903AD4ED460A71
:10CAA000B8EE670A6421CDE7002AF5D0E3E700BFBE
:10CAB000000000002DE9F04100F58048044604F52F
:10CAC0009843D8F8440C1433984203D100252846E3
:10CAD000BDE8F08103689B6B984750B104F5A04313
:10CAE00093F8F85315F0010503D0012283F8C02212
:10CAF000EDE704F5B940203076F0A6F9054608B117
:10CB00000125E4E704F5A04696F8C032002BDDD0FD
:10CB1000D8F8440C03689B6B984718B9002386F833
:10CB2000C032D4E794F8403294F86872B02202FB25
:10CB3000034393F88921AFBB012A0AD993ED697A9F
:10CB4000F1EE047AB4EEE77AF1EE10FAACBF012709
:10CB50000027D8F8442C04F5974358339A4202D161
:10CB600096F8743223B104F598431C339A423FD1AE
:10CB700004F50053204693F99882FCF7D3FA98B94C
:10CB8000204601F011FC0028BAD0002386F8C032FC
:10CB900094F88102242303FB0044D4F89C32C6F8A5
:10CBA0006C3294E72F46D4E778F0BCF9D6F8D4324B
:10CBB0004FF4FA62C01A642313FB082341F288324F
:10CBC000934238BF13469842DAD92046F9F7D0FB92
:10CBD000B0F5FA7FD4DD04F5805341F26E72D3F8DC
:10CBE000C43303F6B7339342CAD8002FC8D095E7B1
:10CBF00006F60463D3ED007AB2EE047AF0EEE77A3B
:10CC0000F4EEC77AF1EE10FA88DA002F3FF478AF2D
:10CC100004F58E50083003F0F3FD00283FF47EAF9A
:10CC200004F5005304F5F650997D083002F0FEFF3C
:10CC3000F1EE047AB4EEE70AF1EE10FAFFF660AF17
:10CC40006CE70000F8B52DED048B04460846164647
:10CC50001D46BDF9287053F0FFF904F50054304625
:10CC6000B0EE408A53F0F8F9B4F97422002AF0EEDD
:10CC7000408A37DAC2F1640307EE903A9FED207ADA
:10CC8000F8EEE77A67EE877A60EE278AD4ED9C7A31
:10CC90009FED1C1ADFED1C0A38EEC80ABC2020EEFE
:10CCA000270A1CF097F838EE288AB0EE409A94EDE7
:10CCB0009C0A9FED141ADFED140A28EE000ABD202D
:10CCC0001CF088F82846B0EE408AB0EE490A53F0CE
:10CCD000AFF9B0EE480ABDEC048B3846BDE8F84029
:10CCE00053F0A6B9D2D002F1640307EE903A9FED5B
:10CCF000047AF8EEE77A67EE877A28EE278AC5E7A6
:10CD00000AD7233C00A08C4500A08CC500B52DEDB2
:10CD1000048B042083B053F09FF90320B0EE408AC7
:10CD200053F0AAF9DFED189A9FED181ADFED180AF3
:10CD30008DED011AF0EE408AB0EE480AA8EEA90A7D
:10CD4000CF20CDED000A1CF045F8B0EE409AB0EED1
:10CD5000480A9DED011ADDED000AA8EEE90AD0208F
:10CD60001CF038F81820B0EE408AB0EE490A53F0B3
:10CD70005FF9B0EE480A192003B0BDEC048B5DF8F2
:10CD800004EB53F055B900BF0000344200A08C45BD
:10CD900000A08CC5F8B52DED088B00F5005600F508
:10CDA000A04596F95E3A13F0040F03F0010203F078
:10CDB000020440F0F580D5F8807F7B1E5F425F4122
:10CDC000002A00F0EF804D2053F046F94E20F0EE9F
:10CDD000409A53F041F9B0EE408AB6F97632DFED71
:10CDE00087AA0AEE103A1520B8EECAAA53F034F911
:10CDF0002AEE2AAA20EE0AAA002C00F0DB80F0EE30
:10CE0000488AB0EE699AB5EEC0AAF1EE10FA40F386
:10CE1000D6809FED7B1ADFED7B0A38EE0A0A4FF4CD
:10CE200080701BF0D7FF9FED761ADFED760AB0EE2B
:10CE3000408A40F2011038EECA0A1BF0CBFFF0EE38
:10CE4000408A96F95F3A632B15DC07EE903A9FED26
:10CE50006E7AF8EEE77AB4EEC79A67EEAA7AF1EE48
:10CE600010FAF4EEC78A98BF29EE279AF1EE10FA6D
:10CE700098BF68EEA78AD5F8803F96F95C4A96F984
:10CE80005D6A022B00F0B48024B2002C01DC002E7D
:10CE90006EDD032053F0F0F8DFED5C7AB4EEE70AC4
:10CEA000F1EE10FAB0EE40AA62DB002F00F0A28093
:10CEB0009FED571ADFED570A40F2271030EE000AB7
:10CEC0001BF088FF9FED541ADFED520AB0EE40BA16
:10CED0004FF494703AEE410A1BF07CFF70EE007A3A
:10CEE000B0EE4BAA07EE104AF8EEC7AA9FED4BBA78
:10CEF0009FED431ADFED430A6AEEA7AAB0EE690A76
:10CF000040F22B10AAEE8B0A1BF064FF07EE906A2A
:10CF1000F0EE409AB8EEE70A9FED391ADFED390AD4
:10CF20002AEE40AAB0EE490A4FF49670AAEE0B0A18
:10CF30001BF050FFB0EE409AB0EE480A9FED301A59
:10CF4000DFED300A40F22D10AAEE8B0A1BF042FFF3
:10CF5000B0EE408AB0EE680AAAEE0B0A4FF4977062
:10CF60009FED271ADFED270A1BF034FFF0EE408A11
:10CF7000B0EE690A102053F05BF8B0EE490A562073
:10CF800053F056F8B0EE480A112053F051F8B0EEC5
:10CF9000680ABDEC088B5720BDE8F84053F048B84C
:10CFA00001270DE7042053F057F8B0EE408AF1EE68
:10CFB000409A12E7DFED178AB0EE689A23E79FEDFB
:10CFC000101ADFED100A39EECA0A4FF482701BF016
:10CFD00001FF9FED0B1ADFED0B0AF0EE409A40F2D5
:10CFE000051039EE0A0A1BF0F5FEB0EE409A28E76C
:10CFF00000244CE7F0EE407A74E700BF0AD7233CE8
:10D0000000A08C4500A08CC5000000B400000034D6
:10D010000000C84200000000000048426666E63E8C
:10D0200038B52DED028B00F500550446D5F8A00A61
:10D03000A0B304F5804393F8582C7ABB93F85E3C78
:10D0400063BB51F0ABFD07EE900AB8EE678A46204D
:10D0500095F9D85153F000F8002DF0EE408A20DA0F
:10D0600004F5B940203075F071FDE8B99FED101A54
:10D07000DFED100A40F25110B1EE680A1BF0AAFE73
:10D08000B4EE408AF1EE10FAC8BFB0EE480ABDEC2B
:10D09000028B6E20BDE8384052F0CABF9FED058A72
:10D0A000D5E79FED040AEBE79FED010AE8E700BF33
:10D0B0000000C8420000000010B52DED028B43694E
:10D0C000002B4AD0037C0BB101330374037C002B8B
:10D0D00041D0182B1FD803EB4303C3EB03139B0072
:10D0E0001CB2002307EE903AB8EEE78A0420B0EEB7
:10D0F000480A52F09DFF07EE904A1320B8EEE70A67
:10D1000052F096FFB0EE480ABDEC028B1520BDE848
:10D11000104052F08DBF4A2B02D8C3F13203DAE738
:10D12000632B01D8643BD6E77C2B08D8643B03EB28
:10D130004303C3EB03139B001BB20024D2E7AE2BC7
:10D1400002D8C3F19603F2E7C72B01D8C83BEEE73C
:10D1500000230374F1E71C46C4E7BDEC028B10BD4D
:10D1600010B59FED1C7AD0ED017AF4EEC77A00235A
:10D17000F1EE10FA044643722BDB90ED007AB4EE28
:10D18000E77AF1EE10FA24D908F022FA217A07F0B2
:10D1900073FED4ED010AF5EE007A60EEA77AB4EEE4
:10D1A000E70AF1EE10FA14D494ED001A40F2A5103B
:10D1B0001BF010FEF7EE007AB4EEE70AF1EE10FA7B
:10D1C00007D494ED007AC7EE007A01236372C4EDB0
:10D1D000037A10BD00000034437A7BB391F900302C
:10D1E00090ED037A07EE903AF8EEE77A67EE877AE9
:10D1F0009FED137AF4EEC77AF1EE10FAD8BFF0EE95
:10D20000477AFDEEE77A17EE903A0B7092F900300C
:10D2100090ED037A07EE903AF8EEE77A67EE877AB8
:10D220009FED087AF4EEC77AF1EE10FA58BFF0EEEF
:10D23000477AFDEEE77A17EE903A1370704700BF19
:10D240000000C8C20000C842437AF0EE407A5BB1E9
:10D2500090ED030A9FED051ADFED050A27EE800A1F
:10D260004FF4E6701BF0B6BD704700BF0000C84227
:10D270000000C8C2F8B504460E46174677F052FEC5
:10D28000054604F59940103007F080FF04F5A044EE
:10D29000D8B3462052F0E0FEDFED3D7AB4EEE70A67
:10D2A000F1EE10FA10DB97F9002094F9C132193A27
:10D2B000934209DAD4F8C422AA4205D0C4F8C45271
:10D2C000013384F8C13244E0462052F0C5FEDFED60
:10D2D000317AB4EEE70AF1EE10FA3AD896F9002066
:10D2E000002A36DAC2F1FF2294F9C23202F57F0237
:10D2F000E73293422DDAD4F8C422AA4229D0C4F8E6
:10D30000C452013384F8C23223E0D4F8C432EB1A99
:10D31000B3F57A7F1DD3462052F09EFE94F9C132B8
:10D3200007EE903AF8EEE77AB4EEE70AF1EE10FA7B
:10D3300001DD002B22DC462052F08EFE94F9C23231
:10D3400007EE903AF8EEE77AB4EEE70AF1EE10FA5B
:10D3500018D497F9000094F9C1220021821A1BF019
:10D36000E9FD387096F90000002806DA94F9C21237
:10D37000002201441BF0DEFD3070F8BDC4F8C45239
:10D38000013B9EE7002BE4DDC4F8C452013BB9E742
:10D3900000000034000000B410B52DED028B00F544
:10D3A000005284B092F9D83192F8D9218DF80E301C
:10D3B000002B0446B0EE408A8DF80F2004DAFFF708
:10D3C000C1F908B98DF80E0004F5A043D3F8C822BE
:10D3D000012A4BD0072A49D004F5B940203075F016
:10D3E000B5FB002853D104F529500DF10E010DF1C4
:10D3F0000F022030FFF7F0FE2046FFF73BFF9DF9BC
:10D400000E309DF90F20DFED238A9342A8BF13460B
:10D4100007EE903AB8EEE70A04F52D5020EE280A00
:10D420008DF80E30019074F089FD9DF90F30019850
:10D4300000EE103AB8EEC00A20EE280A74F088FD1B
:10D440009DF90F3001EE103A9DF90E3000EE903A42
:10D45000B8EEC11AF8EEE00A40F24D20B0EE480AEC
:10D460001BF0B8FC04B0BDEC028B10BDD3ED897A83
:10D47000FDEEE77A17EE902AD3ED8A7A8DF80F2029
:10D48000FDEEE77A17EE903A8DF80E30ABE7002309
:10D49000FAE700BF0AD7233C70B5044600F52955CA
:10D4A000203504F580462846FFF75AFED6F8440C8E
:10D4B00003685B6D984740B1462052F0CDFD284689
:10D4C000FFF7C2FE462052F0B3FDD6F8440C0368C5
:10D4D0001B6D984740B1462052F0BEFD2046FFF735
:10D4E0005BFF462052F0A4FD2046FFF7E3FA10B39D
:10D4F00004F5005595F9443243B101212046FFF768
:10D50000E7F9BDE87040462052F092BD04F5B944F9
:10D510002034204675F01AFB50B1204675F09EFC71
:10D5200030B195F9D83100EE103AB8EEC00AE8E70C
:10D530009FED010AE5E770BD0000000010B504464C
:10D540002DED028B462052F087FD2046B0EE408A3A
:10D55000FBF7E8FD80BB04F5BD4054306FF08AFD59
:10D5600050B304F5A153D3ED008A1AF0B7FE90F83A
:10D57000EC349FED137A0C2202FB0300D0ED807A8D
:10D58000E8EEC77AF4EEC77AF1EE10FA0CDC04F597
:10D59000005494F9DB3107EE903AF8EEE77AF4EEB6
:10D5A000C87AF1EE10FA07D5BDEC028B0548BDE84C
:10D5B0001040012104F0A6BDBDEC028B10BD00BFE0
:10D5C0000AE81C41603E00202DE9F04100F50055BD
:10D5D0000646D5F89C3AA3BB002706F58048D8F844
:10D5E000440C03689B6B98470446002852D006F50C
:10D5F0008E50083003F004F980B308F54763D3ED8B
:10D60000007A9FED3F7AF8EEE77A67EE877AFDEED3
:10D61000E77A17EE903A1BB295F98B220AB19A423B
:10D620001FDA95F98942FCB906F5A042D2F8C83252
:10D63000013B062B2ED8DFE803F01E2D24602D2D94
:10D640001E0051F0FFF80368DB6898470028C3D03C
:10D65000D5F89C0A51F0A2FA47B2BEE795F9DB3142
:10D66000DAE795F98A42DFE724B29C42ACBF95F92C
:10D6700088420024D8E795F98C32002B18BF1C464D
:10D6800008E095F98C322BB13046FBF769FD08B103
:10D6900095F98C4287EAE773A3EBE773DBB2A34209
:10D6A000C8BF3C4607EE904A0320B8EEE70A52F0A6
:10D6B000BFFC07EE907A0220B8EEE70A52F0B8FC01
:10D6C00095F9BD32D6ED460A00EE103A6421B8EE67
:10D6D000C00A032052F0A2FD95F9BD32D6ED460AEC
:10D6E00000EE103A0220B8EEC00A642152F096FD16
:10D6F0003046BDE8F041FFF709BB92F91B3DBCE79E
:10D700000AD7233C70B504462DED048B462052F019
:10D71000A3FC5B4BDFED5B7A93F9293A08EE903A74
:10D72000F8EEE88A152068EEA78AB0EE408A52F03B
:10D7300093FC9FED557A20EE280A04F5A045C0EE33
:10D74000077A05F5776604F5BA402C30C6ED007A05
:10D7500072F058FA08B100233360B5EEC08AF1EEDA
:10D7600010FA46D52046FFF7ADF8002800F0838078
:10D770002046FEF7E7FF00287DD005F57765D5ED5B
:10D78000007A9FED429A9FED421ADFED420AB0EE19
:10D79000480AA7EE890A4FF43B701BF01BFBD5ED3E
:10D7A000007A9FED3B1ADFED3B0AF0EE408A40F233
:10D7B000ED20B0EE480AA7EEC90A1BF00BFBB0EE55
:10D7C000408A04F5BD45543528466FF05DFCE0BB4A
:10D7D000284670F065FD022829D10321492052F026
:10D7E00081FFBDEC048B0321BDE870404A2052F05C
:10D7F00079BF40D905F57765D5ED007A9FED239A7D
:10D800009FED251ADFED220AB0EE480AA7EE890A3D
:10D8100040F2F2201BF0DEFAD5ED007A9FED1E1AE1
:10D82000DFED1B0AF0EE408A40F2F320C1E79FEDE6
:10D83000180A492052F0FCFBBDEC048B9FED140A42
:10D84000BDE870404A2052F0F3BBB0EE680A4920B0
:10D8500052F0EEFBB0EE480A4A2052F0E9FB2046B7
:10D860004921FFF7DFF8BDEC048B20464A21BDE8D3
:10D870007040FFF7D7B89FED068AF0EE488AA0E720
:10D88000984C00200AD7233C00A08C450000484259
:10D89000000000000000C8C20000C842F8B52DED2D
:10D8A000028B00F5A046044696F9193D002B32DDA7
:10D8B00000F5804200F59743D2F8442C58339A4241
:10D8C00029D196F9183D002B25DD00F5B94020300F
:10D8D00075F0AEF9F8B104F5BD4054306FF0CAFBF5
:10D8E000C8B9124F9FED128A04463D682D190ED01B
:10D8F000B5F9080052F0C2F948B196F9193D012B6B
:10D900000CD1B5F90800B0EE480A52F091FB14347E
:10D91000B4F5A07FE9D1BDEC028BF8BD022BF6D1A6
:10D92000B5F90800032152F0DDFEF0E77091002008
:10D930000000000037B500F5A043044693F82032FC
:10D940000BB39FED120A15204F2552F071FB2046B4
:10D950000095502313221521FFF774F9152052F07A
:10D9600009FE80B9284652F005FE60B99FED070A0E
:10D970004E2052F05DFB9FED050A4D2003B0BDE83F
:10D98000304052F055BB03B030BD00BF0000000076
:10D9900070470000F8B52DED048B00F58045044676
:10D9A000D5F8440C03689B6B984738B9D5F8442CDC
:10D9B00004F597432C339A4240F0BE8004F5BD40F5
:10D9C00054306FF061FB002800F0B6802046FBF772
:10D9D000A9FB002800F0B08004F5A045D5F8DC32A2
:10D9E000002BB8BF5B42B3F52F7F00F3A580D5F8BD
:10D9F000E032002BB8BF5B42B3F52F7F00F39C8071
:10DA000077F090FAD5F8403EC31AB3F5FA7F064690
:10DA1000C0F0928004F5AE5393ED037AF2EE007AF3
:10DA2000B4EEE77AF1EE10FA00F1868095EDBA7A5D
:10DA3000B4EEE77AF1EE10FA7ED404F5005707F65B
:10DA4000EC6393ED048A04F5405304F51854D3EDC8
:10DA5000168A1434B0EE480A0421204652F05EFBC8
:10DA6000B0EE680A1321204652F058FB78EEC89AAF
:10DA70004D21B0EE690A204652F050FB38EE289A4C
:10DA80004E21B0EE490A204652F048FBB0EE680A3B
:10DA90004F21204652F042FBB0EE680A502120464A
:10DAA00052F03CFBB0EE480A1821204652F036FBFB
:10DAB000B0EE480A1921204652F030FB97F95E3A41
:10DAC00003F00202DB075CBFF1EE489AB0EE489A21
:10DAD0006AB3B0EE498AF0EE698AB0EE690A1021A5
:10DAE000204652F01BFBB0EE680A5621204652F049
:10DAF00015FBB0EE490A1121204652F00FFBB0EEA3
:10DB0000480A5721204652F009FBD5F8443EC5F893
:10DB1000406EF31A42F2107293420DD9C5F8446E6A
:10DB2000BDEC048B2046BDE8F84052F0DDBE9FED11
:10DB3000048AF0EE488AD0E7BDEC048BF8BD00BF44
:10DB40000000000073B5044652F0E4FF054652F0B1
:10DB500077FF2046FFF7D6FD4E23009313224D2377
:10DB600004212046FFF76EF84F231521132200935E
:10DB700020465023FFF766F82046FFF70BF92046B2
:10DB8000FFF78CFE4FF400512046F4F7E7FC10B18C
:10DB90002046FFF7CFFE04F50056D6F82C0A50B108
:10DBA00004F5804204F59843D2F8442C14339A4289
:10DBB00001D152F017FA52F0D9FE52F02DF9284651
:10DBC00052F046FF96F9003A2BB1204602B0BDE86C
:10DBD0007040FFF7DFBE02B070BD000073B50446B1
:10DBE00004F5BA4552F096FF2C3552F029FF28462D
:10DBF00072F008F804F5A046002866D1D6F8C832BD
:10DC0000042B04D104F5B940203074F0CBFF20463A
:10DC1000FFF742FC04F5804204F59843D2F8442C07
:10DC2000143304F5BD459A4205F1540523D0284626
:10DC30006FF02AFAF8B99FED310A462052F0F8F950
:10DC40009FED2E0A492052F0F3F99FED2C0A4A204D
:10DC500052F0EEF9284670F023FB02280BD1032185
:10DC6000462052F03FFD0321492052F03BFD0321A5
:10DC70004A2052F037FD2046FFF760FC2046FFF7B0
:10DC8000A3FC2046FFF7CCF920464621FEF7CAFE4A
:10DC900028466FF0EFF990B90190284670F000FB2C
:10DCA00068B102281AD10199462052F087FC0199E7
:10DCB000492052F083FC01994A2052F07FFC204613
:10DCC00002B0BDE87040FFF73DBF2846F8F794F872
:10DCD00096F9363D2B2B91D002B070BD9FED070A0F
:10DCE000462052F0A5F99FED050A492052F0A0F90F
:10DCF0009FED020A4A2052F09BF9E0E70000000085
:10DD0000F6F796BE0148FAF7C1BF00BF982C002075
:10DD100008B5044A0F2343F0F1F880F00100C0B2C7
:10DD200008BD00BF18930C08F8B500F5405704462D
:10DD3000D7F8085477F0F6F804F5804304F5005658
:10DD4000B3F95C1C8A1E92B2012A73D904F5A04271
:10DD5000D2F8C822042A6DD0012993F8581CD3F8B0
:10DD6000642C08BFD3F8602CB1B1821A07EE902A58
:10DD700096ED967ADFED416AF8EE677A27EE267A1D
:10DD8000F4EEC77AF1EE10FA06DD032202212046F6
:10DD9000BDE8F840FAF732BE96F95C22032A1BD19F
:10DDA000D3F8443C04F597425832934265D1002D94
:10DDB00063D0401B07EE900ADFED306AB8EE677A59
:10DDC000D6ED967A67EEA67AB4EEE77AF1EE10FA1F
:10DDD00053DD05220321DAE7012A4CD0022A4CD177
:10DDE0008DB1431B07EE103AD6ED967ADFED236A2C
:10DDF000B8EE477A67EEA67AB4EEE77AF1EE10FA5B
:10DE0000E7DC022A39D197F8EC32B3B3D7F8F03215
:10DE10009BB31B4B1B6883B3C01A07EE900A96EDA9
:10DE2000967ADFED166AF8EE677A27EE267AF4EE38
:10DE3000C77ACBE796F95022D6ED967A032A18BF17
:10DE4000D6ED957A03290FD1FCEEE77A4FF47A7379
:10DE500017EE902A401B5A4390420ED205212046CD
:10DE6000BDE8F840FAF784BE022906D193F8583C81
:10DE70001BB90321F3E7002DB3D1F8BD00007A44AC
:10DE8000E490002070B500F50056044696F9503233
:10DE9000032B00F580450FD0B5F95C3C63B900F564
:10DEA000A043D3F8C832042B17D095F8583CA3B13F
:10DEB00003220121FAF720FDB5F95C3C012B0CD1BE
:10DEC00095F8583C1BB196F95032032B05D12046EA
:10DED0000321BDE87040FAF71DBE70BD70B500F5B6
:10DEE000B266044630461AF0C5F904F549531033BA
:10DEF00060B3174A04F58E5518460121083548F0DD
:10DF0000F1F8284602F022FB04F58053032283F83F
:10DF1000DC2340F20112A3F8D024B4F9A4301BB9D9
:10DF2000B4F8A230A4F8A430B4F8A41030461AF023
:10DF30007BFA284602F00AFC8023C4F8843204F5F8
:10DF40001C700121BDE8704006F0F4BA014AD1E727
:10DF500020920C084D920C0838B50B6805465B689A
:10DF600008460C469847074BD87023682046DB6864
:10DF70009847014605F58B501430BDE8384038F01D
:10DF800017BB00BFD58C00202DE9F74F00F5804767
:10DF90000446D7F8443C8B420D4616460CD100F59A
:10DFA000005494F89831934240F0B5804FF0010945
:10DFB000484603B0BDE8F08F0B6808465B69984798
:10DFC00004F5495808F110088146B0B143F048F90A
:10DFD00040F203124FF4801143F0FAF8524A06213E
:10DFE000404648F07FF81A2E1FBF504A137843F07E
:10DFF000040313704FF00009DAE74D4B1B68DB6A2E
:10E0000093F89C305BB304F5005393F8802032B34F
:10E01000B3F89C20D20722D593F8BC30FBB1204640
:10E02000FAF7E4FED8B1A6F12703DBB20A2B06D833
:10E03000012202FA03F340F2234213420FD12B686C
:10E0400028469B6898473B4A03460521404648F0CE
:10E0500049F8364A137843F004031370A8E7022EF8
:10E060002BD0D7F844BCD7F8483CC7F8445C04F53B
:10E070000059C7F848BC04F5A04A99F898210093C4
:10E0800028469AF8883F8AF8882F89F89861019382
:10E09000FBF72CFC38BB284A0421404648F022F804
:10E0A000009BC7F8483CC7F844BC9AF8883F89F8F9
:10E0B0009831019B8AF8883F95E72B6828465B6872
:10E0C000984701462046FFF723FE81460028C8D125
:10E0D0002B6828469B689847184A03460521404606
:10E0E00048F000F864E75846FBF7ECFBD7F8440C1F
:10E0F00003685B68984799F89821014604F6A86080
:10E1000044F088F8D7F8441C2046FFF725FF00218B
:10E1100040464FF0C1FC1A2E1FBF044A137843F04B
:10E120000203137042E700BF68920C08F48C0020D1
:10E13000942C002080920C08EC920C08AC920C08F5
:10E1400073B505460A4801920E46FAF7BDF9019AE1
:10E15000044630B10146284602B0BDE87040FFF7E2
:10E1600013BF2846314642F00FFE204602B070BD74
:10E17000982C0020FFF7E4BF4FF40023F7B50446C6
:10E18000C0F8803A00F53750043070F0ABFF04F56A
:10E190003C501C3070F022FD50F054FB9922292194
:10E1A00051F03AFC50F04EFB50F0F4FA04F58A506E
:10E1B00059F0DCFB04F58B50143038F0DDF904F530
:10E1C00080432046D3F8441CFFF7C6FE2046FDF7E7
:10E1D000B7FF04F51C7006F025FC4FF480431921AD
:10E1E000C4F8A43E04F6F8303DF036FC04F599403E
:10E1F000103006F091FD04F6D87053F0ADFD04F533
:10E20000495504F52B501035183053F027FA28469D
:10E210004CF0BAF904F55550103060F005FF0AF0E3
:10E2200065FC4FF4806343620AF060FC0BF05AFC1B
:10E2300004F5075104F5F6501831083001F0B6F82E
:10E2400004F5005380229A610423C4F85C3104F57C
:10E25000907011F0EDFA2046FDF758FF04F5BC4030
:10E26000503054F06BFB04F551503C3008F094F8FA
:10E2700004F528503C3060F0C7F9334B33491E6831
:10E28000B06A03684FF47A72DB6A984701203BF06A
:10E29000BFFA04F598411A220C312046FFF774FEAC
:10E2A0002B4A0621284647F01DFF2046FFF716FEA1
:10E2B00004F5A5406C301FF013F904F5A0434FF4AA
:10E2C0008072C3F8E023234B0093234B019302ABEE
:10E2D00013E9060004F6A86043F0B4FD76F022FED0
:10E2E00004F5405504F50057C5F808042046FDF72D
:10E2F00053FFD7F87C1A29B1706A03680222D3F859
:10E3000080309847706A154B1A68036892F8F113C9
:10E31000D3F8AC30984797F864121A222046FFF7DA
:10E320000FFF50F08FFA50F017FA95F901354BB105
:10E3300004F553504FF0FF313C3003B0BDE8F040DE
:10E3400039F022BB03B0F0BD942C002005DD01089C
:10E3500008930C08982C002001DD0108189100207A
:10E3600000F6A86044F0B4BB10B52DED028B044656
:10E3700082B0462051F070FE2046B0EE408AFEF793
:10E38000A1FAFDEEC87A0146CDED017A642240B9CA
:10E39000BDF904001AF0CEFD40B202B0BDEC028B14
:10E3A00010BD6FF06301F3E72DE9F04F054605F569
:10E3B000005985B076F0B6FD99F9988264231FFA6A
:10E3C00088F803FB08F8064643F29C1305F5BD40A8
:10E3D000984500F15400A8BF98466EF055FE05F52B
:10E3E000A044074698B9014605F5A4403022043000
:10E3F000A0F09EF895F88102242303FB0055D5F880
